:020000040800F2
:1040000000500020D1E400086DBC000871BC00081D
:1040100075BC000879BC00087DBC000800000000E9
:1040200000000000000000000000000085BC000847
:1040300081BC00080000000089BC0008CD8B00088E
:104040008DBC000891BC000895BC000899BC000814
:104050009DBC0008A1BC0008A5BC0008A9BC0008C4
:10406000ADBC0008B1BC0008B5BC000800000000F1
:104070000000000000000000000000000000000040
:104080000000000000000000D5BC0008D9BC0008FA
:10409000E9BC0008F9BC000809BD000819BD00080A
:1040A0001DBD000821BD000825BD000829BD000870
:1040B0002DBD000831BD000835BD000839BD000820
:1040C0003DBD000841BD000845BD000849BD0008D0
:1040D0004DBD0008418800087D87000859BD0008D3
:1040E0005DBD000861BD000865BD0008000000005E
:1040F00000000000000000000000000000000000C0
:0C41000000000000000000005FF800005C
:1041100030BF704720BF704740BF7047BFF36F8FFD
:104120007047BFF34F8F7047BFF35F8F704701DF5A
:104130007047EFF31480704780F31488BFF36F8FDC
:104140007047EFF30980704780F309887047EFF3F9
:104150000880704780F30888704772B6704762B66F
:10416000704771B6704761B6704780F31188704729
:10417000EFF31280704740BA704700BA70470000F2
:1041800037B508F077FE524B00254FF480301D7094
:1041900008F090FE08F0F4FF0128044626D1102014
:1041A00008F052F9284608F0D5FE284608F0E6FE49
:1041B000284608F0D9FE4FF480304FF4802108F0F3
:1041C000A5FE204608F0AEFE392008F0C3FF002807
:1041D000FAD0012008F020F9012008F0A9FE08F02B
:1041E000B1FE0428FBD13A4B01221A7004200121B0
:1041F00008F066FF03238DF80630153301A9354812
:104200008DF807304FF48073ADF8043008F050FBA0
:10421000062008F099FF0120014608F051FF4FF4F5
:1042200080414FF0006008F047FD4FF4407008F007
:10423000A5FC00F005FB00F01FFC2749274A284B8E
:104240001160284A284D136001222A70274A284C01
:10425000136000F0C7F804F0A5FD04F007FD04F0BA
:1042600067F900F049F8207804F0FCFBE07804F0EE
:10427000EDF9207804F03CFBE07804F00FFA2B789D
:104280000BB105F0D1F805F057FE00F07DF907F00D
:10429000BFFA01F0C5FC05F0E1F805F093FE154BFF
:1042A0004FF480625A6104F0DBFC03F0BBFA05F0C6
:1042B00097FE05F00DF900F0EBF800F0DDF80028AE
:1042C000F3D005F039FE01F0ABFC05F07BFEECE726
:1042D000580C002000080140C9920008680C00201A
:1042E000C98B0008F80B0020780B0020980B0020E9
:1042F00008000020000C0140144B82B01B7813B35F
:10430000134B4FF400725A614FF480721A6100230C
:1043100001E0019B01330193019A4AF69B539A42B3
:10432000F7D90B4B4FF400721A614FF480725A6147
:10433000002301E0019B01330193019A4AF69B534C
:104340009A42DDD8F6E702B0704700BFA40B002008
:10435000000C014010B1012805D101E0082200E065
:104360000422014B5A617047000C014010B1012832
:1043700005D101E0082200E00422014B1A617047D8
:10438000000C014038B50546002455FA04F2E3B2AA
:1043900012F0010F184602D0FFF7E8FF01E0FFF727
:1043A000D9FF0134082CF0D138BD00BF18B1012865
:1043B00006D0002008E0054BD868C0F3C00003E039
:1043C000024BD868C0F38000704700BF000C01406A
:1043D00008B1002003E0024B9868C0F3C03070477A
:1043E0000008014062B6704772B6704718B9024BB8
:1043F0004FF480625A617047000C014018B9024BBB
:104400004FF480621A617047000C014020B1054BE7
:104410004FF400521A6103E0024B4FF400525A610C
:10442000704700BF0010014020B1054B4FF480429F
:104430001A6103E0024B4FF480425A61704700BF9B
:104440000010014010B9024B09011960704700BF0C
:104450000400002008B9014B197070473002002099
:10446000044B58780138C0B201288CBF00200120CD
:10447000704700BF30020020044B5878012801D05B
:10448000002001E002225A70704700BF3002002075
:10449000082008B504F000FC592804D9064B5A78C6
:1044A0004AB9013206E0082004F0F6FB542802D88D
:1044B000014B00225A7008BD3002002008B50328C5
:1044C00003D8DFE800F0040D1217002016E00020EA
:1044D00004F0E2FBB0F5006F94BF002001200DE076
:1044E000074B9868C0F3801008E0054B9868C0F34C
:1044F000C01003E0024B9868C0F3401008BD00BF35
:10450000000C014038B500242546E0B2FFF7D6FF85
:1045100020B10123A34043EA0505EDB20134082C84
:10452000F3D1284638BD00BF70B50D4D0D4C2A683B
:104530000AB1606812E0FF21032000F021FAFF2198
:1045400006460122032000F01BFAA36840EA062079
:1045500003EA9000181A01232B60606070BD00BF51
:10456000E80600203002002008B5FFF7DDFF05282F
:1045700001D8012007E0FFF7D7FF40F2F933984256
:1045800094BF0020012008BD38B51E4C00202169D1
:104590004909FFF757FF2169002001F01F01FFF7CC
:1045A00059FFFE210022032000F0EAF940210122F8
:1045B000032000F0E5F900210A46032000F0E0F9AD
:1045C000002104460122032000F0DAF9082C0E4BEA
:1045D00005D14FF40062DA6040F6FF7204E04FF458
:1045E0000072DA6040F2FF329A60FFF79DFF064BDF
:1045F000040224464FEAE475C3E90845C3E90645C9
:10460000186138BDFC0B0020300200202DE9F84372
:1046100004F026FB624CA062FFF786FF2369E0628C
:1046200098423EDDE268C11A91420BDA5D4B256B80
:104630001A684D195143D4E90867721847EBE173C2
:1046400025632BE094F800C0564A1CF0040F12D0EA
:10465000A3681668C31A5E432CF0040C36464FEA72
:10466000E677236300220023C4E9086784F800C0CA
:10467000C4E906234EE0A56816685A190132121AD9
:104680007243D4E90867236BED43ED18B6EB0208DB
:1046900067EBE27942464B4669182163C4E9082377
:1046A00038E037DAE1681A1A8A420EDA3D4D216B9A
:1046B0002D68C91A6A43D4E90867B6EB020867EBAC
:1046C000E27942464B460918E7E72178354A11F06E
:1046D000040F0FD0126821F00401424312464FEA42
:1046E000E273C4E90823002200232170C4E90623F1
:1046F00020630FE0A16812680131CB1A1B185A43DE
:10470000D4E90867B61847EBE277226BC4E908677B
:104710009B182363224B1D6B5A6B996BAA1A82EA72
:10472000E27CACEBE27C8C452CD942F210714A431E
:104730009E6ADC6B3C21341B92FBF4F251434FF434
:10474000807C91FBFCF181EAE172A2EBE172596499
:1047500040F6B8318A42DE635D631C6401DDC82225
:1047600019E0B2F57A7F01DD642214E0322A01DD1E
:104770000A2210E00A2A01DD05220CE0012A0BDDE5
:10478000012208E0996ADA6B8A1AB2F5FA6F03D946
:1047900000225A6401329A63014B1861BDE8F88324
:1047A000300200200400002038B50D4618BB124C22
:1047B000FFF72CFFD4E90801002901DBA26803E020
:1047C000A268404261EB4101120212464FEAE273D5
:1047D0000CF09EFCC4E9062328464FEAE071064C23
:1047E0000B02020243EA1063D4E90601801841EB90
:1047F0000301C4E9080138BD3002002008B508B142
:1048000000200CE0FFF702FF054BD3E90601D3E9D6
:104810000823121A63EB0103100A40EA036008BD83
:104820003002002008B510B108F050FA01E008F09D
:1048300055FA08BD08B5C90804F0E8FF08BD00BF77
:104840002DE9F745DFF830814848012108F0C0F82C
:1048500001AE0420012108F033FC0325102440465A
:1048600042F212233146ADF804308DF806508DF82F
:10487000074008F01DF802233D4F4046C8F810409D
:104880004FF0040AC8F8143031464CF20043ADF83A
:1048900004308DF806508DF807A008F009F80820BC
:1048A000012108F00DFC41F61C7338463146ADF885
:1048B00004308DF806508DF8074007F0F9FF4FF4EB
:1048C000F8533B610C23384631467B614FF0E003DF
:1048D00008F50068ADF804308DF807A08DF8065093
:1048E00007F0E6FF2046012108F0EAFB4EF2000344
:1048F00031464046ADF804308DF806508DF807403B
:1049000007F0D6FF4FF42043C8F81030A3F5C0439A
:104910000121C8F81430174808F05AF800231A4645
:104920001946154C4FF4005565612046A4680133C3
:1049300014F4804F4FF400540461806808BF0131C3
:1049400010F4804F18BF01320A2BEAD10A2903D193
:104950000A2A01D1012200E00022084B03481A7004
:10496000012108F035F8BDE8FE8500BF00023000E7
:10497000000C01400004300000080140A40B00209E
:1049800070B504460D461646032868D8DFE800F0E7
:1049900002070A0E334B4FF480525A6112E0102284
:1049A000314B0DE04FF400622E4B09E02F4A138883
:1049B00023F002031B041B0C13802D4B4FF4004209
:1049C0005A6110E02B48022108F0DCFC0028F9D0E5
:1049D0002946284808F07AFC2648012108F0D2FC34
:1049E0000028F9D00FE02148022108F0CBFC002874
:1049F000F9D029461D4808F069FC1C48012108F03F
:104A0000C1FC0028F9D0EEB1032C28D8DFE804F06F
:104A100002070A0F134B4FF480521A6118E010225C
:104A2000114B02E00F4B4FF400621A6112E0104A82
:104A30000E4B4FF4004111611A8892B242F002020B
:104A40001A8007E0032C0AD8DFE804F0020404040B
:104A5000084800E0054808F03BFCC0B200E0002038
:104A600070BD00BF000C0140000801400030014053
:104A700000100140003800402DE9F04F01218BB0BB
:104A80004FF4804008F02AFB494C012009AF014651
:104A900008F016FB03264FF0180B204639464AF261
:104AA0000003DFF81491ADF824304FF0040A8DF8BC
:104AB00026608DF827B007F0FBFE204639464FF4FC
:104AC00080430DF11008ADF824308DF826608DF884
:104AD00027A007F0EDFE4FF48273002402224FF46A
:104AE000007C012548464146ADF812304FF00803DE
:104AF000ADF81620ADF81AC00392CDF808C0ADF895
:104B00001C30ADF81040ADF81440ADF81850ADF8B9
:104B10001E40ADF8204008F065FB4846294608F0E5
:104B20009DFB29464FF4805008F0CAFA09F5504918
:104B30002846214607F04CFF484639464FF0A0036F
:104B4000ADF824308DF827B08DF8266007F0B0FE60
:104B5000484639464FF04003ADF824308DF82660C2
:104B60008DF827A007F0A4FE039ADDF808C04FF4E3
:104B700082734146ADF812300E484FF01003ADF885
:104B80001620ADF81AC0ADF82040ADF81040ADF8D1
:104B90001440ADF81850ADF81C30ADF81E4008F0C8
:104BA00021FB0448294608F059FB0BB0BDE8F08F03
:104BB000000C01400030014000380040014B1878E3
:104BC000704700BF780200202DE9F84505461446DD
:104BD0000E4600294BD0002849D0814247D04FEAE9
:104BE00042185FFA88F848F006073946002006F0B8
:104BF0000BFB48F00C018246002006F005FB8046C6
:104C000028460CF047F8054630460CF043F80146BC
:104C100028460CF04BF9064650460CF03BF831465E
:104C20000CF044F90CF054FA054640460CF032F80A
:104C300031460CF03BF90CF04BFA0E49002814BF3A
:104C400080464FF001083046002D08BF01250CF0CA
:104C500017FA18B14146204606F050FD39462A465B
:104C6000002006F083FB044BE41801232371BDE808
:104C7000F88500BF0000A0417802002070B50D4DFE
:104C8000044645192B799BB1C6B20B4B710141F01B
:104C9000060153F8202001F0E601002006F0FAFB9F
:104CA000064B304653F8241006F028FD00232B71E4
:104CB00070BD00BF78020020740B00207007002038
:104CC00073B5A54CA578002D40F00C836378A42B18
:104CD00000F044825AD8842B00F0C68026D8062BD8
:104CE00000F00D8110D8022B00F0BE8006D8002BFA
:104CF00000F0AA80012B40F0F382ABE0042B00F01F
:104D0000D78000F2E780CDE0802B00F09D8007D8AF
:104D10000C2B00F00F810D2B00F02C81072B70E085
:104D2000822B00F0398100F2C38093E0942B00F0D5
:104D3000018116D88A2B00F03F8108D8862B00F01D
:104D4000C980C0F0AF80872B40F0CA822EE18D2B46
:104D500000F05181932B00F00D818C2B40F0C0822C
:104D60003EE1A02B00F0E58109D8992B00F0668187
:104D70009A2B00F07881952B40F0B28241E1A22B72
:104D800000F0E181744B00F2E481D7E1B62B00F032
:104D90006A8228D8AC2B00F0318210D8A82B00F002
:104DA0000F8205D8A62B00F0F68100F20382E3E122
:104DB000AA2B00F00F82684B00F2128205E2B02BA2
:104DC00000F0388206D8AE2B00F02882624B00F249
:104DD0002C821EE2B22B00F03882C0F03082B52B5C
:104DE00040F07E8237E2C82B00F06A8115D8C12BD3
:104DF00000F0528108D8B82B00F04E82C0F04782F4
:104E0000C02B40F06D8288E0C32B00F05181C0F0D0
:104E10004781C72B40F0648271E0D42B00F065819C
:104E200009D8D12B00F03E82D22B00F04482CC2B4B
:104E300040F0568251E1D62B00F06381C0F05C81D6
:104E4000FE2B40F04D8264E1434B00205A6801463E
:104E5000DB7804E0404B00205A68DB78022143EA0B
:104E6000022206F083FA40E23B4C0020E3786268BD
:104E7000082143EA022206F00DFBE378A17862687C
:104E8000490143EA0222002A41F00601B8BF52421A
:104E900001F0E601002006F0FDFA304AA378D318AD
:104EA0000122F7E12C4B00205A680A21DB7878E0D8
:104EB000294C0020E3786268062143EA022206F0CA
:104EC000E9FAE2786068A37842EA0020234A24499C
:104ED0009A180FE0204C0020E378616843EA012132
:104EE00006F00CFCE2786068A37842EA00201B4AD6
:104EF0001C499A1841F8230000231371F5E1164B61
:104F0000194AD978194B01201B781070184A022BC6
:104F1000517240F0EA810138B6E10F4B0122D97895
:104F2000124B1878104B1A70114B9972002840F0F0
:104F3000DC81A9E11421002001AA06F0B7F9064A94
:104F40009DF805305168D27852EA012114BF43F030
:104F5000020323F0020365E0EC0600207802002043
:104F6000740B002070070020600C0020640C0020EF
:104F7000FC0B00201421002001AA06F097F99B4A9F
:104F80009DF805305168D27852EA012114BF43F0F0
:104F9000010323F0010345E0944B00205A68DB78BD
:104FA000042143EA022206F075FA9EE18F4B0020AD
:104FB0005A680E21DB78F4E701AE32461421284608
:104FC00006F074F9A178E378490141F0140128460C
:104FD00001F0F40132468DF8063006F003FB84E15F
:104FE000824B834ADB780020C3F10801C9B2D37237
:104FF00004F026FF79E17D4B00205A681A21DB7806
:10500000CFE71421002001AA06F050F9774A9DF855
:1050100005305168D27852EA012114BF43F00403ED
:1050200023F004038DF80530704B0020997801AA15
:10503000490141F0140101F0F401CEE701AC224630
:105040001821002006F032F9684A9DF80530917861
:10505000D278490102F00F0223F00F0341F018014A
:1050600042EA030311E001AC22461821002006F0B9
:105070001DF95E4A9DF805309178D278490103F018
:105080000F0341F0180143EA021301F0F801224630
:1050900000208DF80530A0E7E278554B1A7224E124
:1050A000524B5A68DB7843EA0222514B1A601CE1EA
:1050B0004E4B5A68DB7843EA02224D4B5A6014E1AA
:1050C0004C4B4D4A1B780120E1781070484A032B65
:1050D000D17740F00A812846D6E0444B5A68DB7805
:1050E00043EA0222424BDA81FFE0E378626843EA56
:1050F00002223F4B5A61F8E03C4BDA783C4B9A77FE
:10510000F3E03A4B5A68DB7843EA0222384B9A8341
:10511000EBE0364B364A5968DB7843EA0121052932
:1051200004D818461373FFF77FF9DEE000231373EA
:10513000DBE02846E17804F075FED6E0D97800205F
:1051400004F066FED1E0294B0020D97804F040FD40
:10515000CBE0D978002004F02FFDC6E0284604F00B
:10516000EDF9E178A37818B9184604F00DFDBCE01C
:10517000184604F0D9FCB8E0002004F0DFF91B4B1E
:1051800020B9D978987804F0F3FCAEE0D978987813
:1051900004F0B2FCA9E0002004F0D0F9134B20B9D0
:1051A000D978987804F0D8FC9FE0D978987804F002
:1051B000AFFC9AE00D4B0020D97804F0C1FC94E0DC
:1051C0002846E17804F0C6FB8FE0D978002004F08F
:1051D000B5FB8AE0054B0020D97804F0A3FB84E0FE
:1051E000D978002004F092FB7FE000BFEC0600209D
:1051F000FC0B0020640C0020600C0020E1782846A5
:1052000004F078FBA178394BE27803EBC1035A71C3
:105210006BE0D978002004F011FB66E0344B0020ED
:1052200093F9031004F0FEFA5FE0D978002004F04F
:1052300093FD5AE02846E17804F082FD55E02C4BBE
:105240000020D97804F070FD4FE0294B0020D97878
:1052500004F05EFD49E0264B5A68DB7843EA0222FF
:10526000244B9A6141E06068E278204B42EA0020DA
:10527000186010B9597904F03DFB1D4B1E4A98780F
:10528000125C012A31D1D978FFF7D4FA2DE0184BFE
:10529000DA78164B1A7128E0154B0020D97804F003
:1052A0007FFC22E0124B00205968DB7843EA0121A1
:1052B000FFF77AFA19E00E4C0020E378626803F0F9
:1052C0001F0143EA02220B4B1A61FFF7C3F8E37890
:1052D0006168A07843EA01214911FFF7B3F804E0BF
:1052E000032200E00422054B1A707CBD880B0020CD
:1052F000EC060020FC0B0020640C0020640700205A
:1053000013B5A84CA078002840F05B826378A52BE9
:1053100000F0EE81A44C79D8842B00F0FB8036D8C5
:10532000082B00F00A8113D8032B00F0F68005D873
:10533000012B00F0E98000F2ED80E2E0052B00F0A7
:10534000F380C0F0EF80062B00F0F180072BA4E083
:105350000D2B00F005810BD80A2B00F02F81C0F037
:1053600009810B2B00F00B810C2B40F02782EDE024
:10537000812B00F0C98003D8802B40F01F82C0E051
:10538000822B00F02881832B40F01882CAE0992BF1
:1053900000F043811ED88C2B00F02D810BD8862B7A
:1053A00000F0C280C0F0B980872B00F019818A2BF1
:1053B00040F0048217E1932B00F0D28003D88D2BAC
:1053C00040F0FC811CE1942B00F0C080952B40F054
:1053D000F58118E1A02B00F06C810BD89B2B00F01D
:1053E000CE80C0F023819C2B00F0E8809D2B40F004
:1053F000E581A2E0A22B00F06381C0F05D81A32BC8
:1054000000F06281A42B40F0D98163E1B82B00F059
:10541000C68135D8AE2B00F0A08115D8A92B00F09D
:105420008A8105D8A72B00F07E8100F280816CE193
:10543000AB2B00F08781C0F08181AC2B00F086811E
:10544000AD2B40F0BB8184E1B32B00F09A810BD8E7
:10545000B02B00F08A81C0F08481B12B00F08981EB
:10546000B22B40F0AB8188E1B52B00F09081C0F009
:105470008B81B62B00F08E81B72B40F09F818BE1A2
:10548000CE2B00F0EF8020D8C42B00F0E0800ED8A7
:10549000C12B00F0D48003D8C02B40F08F8149E0AD
:1054A000C22B00F0CF80C32B40F08881CCE0C72B0B
:1054B0003DD003D8C52B40F08181CAE0C82B00F055
:1054C000CB80CC2B40F07A81C9E0D42B00F0E48073
:1054D0000BD8D02B00F0DE80C0F0C680D12B00F0BE
:1054E0006181D22B40F06A8160E1D62B00F0DB8035
:1054F000C0F0D680D72B00F05E81FE2B40F05E819D
:10550000D4E00020014601E00020022105F07CFEED
:10551000606059E1002008215FE000200A2105F0C9
:10552000ADFEF5E7214B00E0214B1B68B6E0214BB7
:105530005B7AB3E01F4B9B7AB0E0002005F07AFD68
:10554000184B9B785B0050FA03F310E00020142105
:1055500001AA05F0ABFE9DF80530C3F340039DE0C2
:105560000020142101AA05F0A1FE9DF8053003F0EA
:10557000010393E0104B9A68C2F3401218E17C21BA
:10558000002001AA05F092FE064B02219A789DF8B0
:105590000630520011FA02F21A420CBF0023012316
:1055A0007CE000BFEC06002064070020740B0020A4
:1055B00070070020FC0B0020000C014001AA002015
:1055C0007C2105F073FE894B9DF806209B785B00DB
:1055D00052FA03F3CBE70020042105F04FFE76E0FA
:1055E00000200E21F9E701AA0020142105F05EFE3B
:1055F0009DF80620DCE003F081FFC0F1080087E79A
:1056000000201A21E9E701AA0020142105F04EFE2E
:105610009DF80520C2F38002CAE0182101AA05F016
:1056200045FE9DF8053003F00F0337E001AA002086
:10563000182105F03BFE9DF805201209B8E06C4BDF
:105640001A7AB5E06A4B05E0694B5A68B0E0694BDD
:105650006BE7694B1A68ABE0654BDA7FA8E0644BF7
:10566000DA89A5E0654B60E7654A664B1278002150
:1056700059600AB101225A60634B614A1B780021CC
:10568000117023B15F4B5A6842F002025A60002247
:105690005D4B98E05D4B78E0554B5B69636093E050
:1056A000534B9A7F84E0524B9A8B81E0504B1A7B8C
:1056B0007EE003F02BFF2BE7002003F02FFF06E036
:1056C000002003F033FF02E0002003F037FF4D4BD2
:1056D000586079E0002003F031FF4A4C434B18B981
:1056E000987803F03BFF13E7987803F057FF0FE734
:1056F00003F024FFA378434C18B9184603F036FF93
:1057000006E7184603F05AFF02E7002003F016FFF1
:105710003C4C364B18B9987803F030FFF8E698788F
:1057200003F044FFF4E6002003F030FFCFE7002051
:1057300003F04CFFCBE703F051FFE9E6002003F054
:1057400055FFC4E7002003F059FFC0E7304B5A79FA
:105750002EE0002003F062FFB9E703F067FF40B2DC
:10576000D6E6002003F074FFB1E7002003F078FFD5
:10577000ADE7002003F07CFFA9E7002003F080FFE5
:10578000A5E703F08DFFC3E6224B1A7810E0184B13
:105790009A690DE01E4B5DE71D4B1A7908E003F096
:1057A000D5FEB5E60020FFF729F890E7104B1A69FF
:1057B000144B5A6008E0FEF7B7FE88E70323237016
:1057C00002E0104B04221A70134B1B786BB10D4B87
:1057D00012495A68124B0A601AB91A6842F0080254
:1057E00002E01A6822F008021A601CBDEC060020D4
:1057F000FC0B00207C0B0020200C0020A00B0020C4
:10580000F00B002064070020940B0020F40B002014
:10581000880B0020840B00205E0700204C0700202E
:10582000F406002010B51B4A5378142B2DD891781C
:1058300071B95468D078184A1849927E40EA042019
:1058400041F8230022B31BB303F5C270013013E00B
:10585000FF2918D163B94FF4C364114920460919CF
:105860000422043402F09CFCB4F5CD6FF5D10FE0B6
:1058700003F5C2700949013001EB83018000042265
:1058800002F08EFC04E0042200E00322054B1A70B3
:1058900010BD00BFEC06002008000020F806002024
:1058A000E40000206407002038B51F4C6578142DF3
:1058B00036D8A07810F0800F18D010F0010F06D065
:1058C0000020022105F0A0FC184B43F82500184BDE
:1058D0009B7E43B3144B5B782BB303F5C270134923
:1058E000013001EB83018000042214E0B0B90221F1
:1058F00005F08AFC0E4A0D4B927E43F8250092B1CA
:10590000617881B1A0780422091801F5C2700130D4
:1059100003EB8101800002F043FC04E0042200E07C
:105920000322044B1A7038BDEC060020F806002054
:10593000080000206407002038B56E4CA07808B13C
:105940000422D3E063789A2B22D8992B80F09B8095
:10595000822B00F081800BD8062B6ED003D8042B4D
:1059600038D0052B0AE0072B6DD00C3B012B0CE047
:105970008C2B75D005D8832B2CD0862B40F0B5808E
:105980003FE08D2B7DD0933B022B00F2AE8060E098
:10599000C72B52D00ED8C12B7AD005D8B52B74D0D6
:1059A000C02B40F0A2804EE0C22B77D0C32B40F03A
:1059B0009C8076E0D42B7DD005D8C82B74D0CC2B1E
:1059C00040F0938073E0D62B7CD077D3FE2B40F051
:1059D0008C807DE0474D0020062105F06DFEAC78FF
:1059E0000020610141F0060101F0E60105F046FCEE
:1059F000414AAB78D318414A42F8240000221A7178
:105A000076E03C4D00200C2105F056FEAC780020DD
:105A1000610141F00C0101F0EC0105F02FFCAB78C5
:105A2000374A354942F8240018465B1852F82010CE
:105A300000221A7105F062FE5AE0492002F098FB3C
:105A4000304B587254E04A2002F092FB2D4B987272
:105A50004EE00020142100E0042105F02DFE47E077
:105A60004B200122284902F05FFBA378254A184603
:105A700002EB4313D97AC1F10801C9B204F0E0F98D
:105A800036E01A21E9E71821E7E758201F4913E01B
:105A9000482002F06DFB1B4B187229E04020194989
:105AA0000AE044201A4907E05F201A4908E04E2026
:105AB000194909E019495420042206E018495E20DA
:105AC000012202E017495C20022202F02DFB0FE0C8
:105AD0004C200122144902F027FBA278094B03EB6A
:105AE0004213187BFEF7A0FC02E003220F4B1A7052
:105AF00038BD00BFEC06002078020020740B0020A7
:105B000070070020FC0B0020070C0020140C002064
:105B1000000C00201B0C00200A0C0020100C0020A0
:105B20001A0C0020180C0020080C0020640700202C
:105B300010B51E4A5378142B34D89278AAB91C4A4F
:105B40001C4952F823201C4B4A601B78002B2CD098
:105B50001A491B4B0A601AB91A6842F0080202E09F
:105B60001A6822F008021A601FE0FF2A18D163B9F0
:105B70004FF4C3641349204609190422043402F087
:105B8000D3FAB4F5CD6FF5D10FE003F5C270084933
:105B9000013001EB83018000042202F0C5FA04E029
:105BA000042200E00322034B1A7010BDEC06002013
:105BB000F8060020640700205E0700204C07002044
:105BC000F4060020E400002037B5134C657815B1C9
:105BD000012D1DD112E0042240F2FB7001A902F058
:105BE000A3FAE378626843EA0222019B9A420B4BD4
:105BF00002D101225A600EE05D600CE0A3782A2BEE
:105C000006D1E11C40F2FB70042202F0C9FA02E066
:105C1000024B03221A703EBDEC06002064070020F0
:105C2000374938B500230B603649374A0B6037498E
:105C300093740B609360D36013745374344A4FF0C1
:105C4000FF3142F82310334A0024D45401332F2B60
:105C5000F4D10731204605F0D7FA2F4B0C211860FC
:105C6000204605F0D1FA2D4D2D4BE97A1860C1F18F
:105C700008012046C9B204F0E3F8287BFEF7D4FB04
:105C8000284B0022E2500434B4F5806FF8D1264B43
:105C90009B7E5BB104F50674244920460919042251
:105CA000043402F041FAB4F5CD6FF5D11E4BDB7E22
:105CB0005BB94FF4A7641E49204609190422043435
:105CC00002F032FAB4F5C36FF5D1174B1B79012BF3
:105CD00003D0112B01D0212B01D1012200E00022A1
:105CE000094B83F8D020104B5B7D23B1FEF7B8FB46
:105CF00008B1012200E00022034B83F8D12038BD17
:105D00004C0700206C07002078020020F4060020D9
:105D10008C020020740C0020740B0020FC0B00206F
:105D2000700700207407002008000020E400002015
:105D30003C02002008B50B4B5A7892B9997881B98A
:105D40005A68DB7843EA022240F2D2439A4208D1F1
:105D500040F2FF7002F0A2FA02F064FB0120FEF7AD
:105D600061FD08BDEC06002010B5994B9A78022A17
:105D700000F05181032A00F05781002A40F0E781AA
:105D80005A784D2A00F0BC8023D8452A70D00ED80E
:105D9000422A56D005D8402A45D0412A40F0D58124
:105DA00046E0432A53D0442A40F0CF8156E0482AA7
:105DB0007BD005D8462A61D0472A40F0C6816AE0E8
:105DC0004B2A00F0848000F29480492A40F0BD8183
:105DD00071E0542A00F0DA8011D8512A00F0B08026
:105DE00006D84F2A00F09280502A40F0AE81A0E001
:105DF000522A00F0B780532A40F0A781BCE0832AE2
:105E000000F0EC8006D8552A00F0CD80572A40F0EB
:105E10009C81D5E0852A00F0F180C0F0E780FF2A60
:105E200040F09381F3E06A4B40F2FF70D97805E0CF
:105E3000674B684ADB7800201946137002F02EFA8F
:105E400088E1DB78634A194601205370F6E7604B1E
:105E5000604ADB78042019461371EFE75C4B5D491B
:105E60005A68DB781C2043EA022341F81C3F0EE00D
:105E7000DB78584A194605205371DFE7544B5549E2
:105E80005A68DB780C2043EA022341F80C3F0422D5
:105E900002F086F95EE14E4B4E495A68DB780820E5
:105EA00043EA022341F8083FF1E7DB78494926201D
:105EB00001F8263F75E0464A464BD27812B1464972
:105EC00001224A60DA75434B1720D97DB6E7404B73
:105ED000404CDB7803201946E37002F0DFF9E078EC
:105EE00002F0B4FBE07802F0B1FBE07802F0D6FB00
:105EF00030E1374B374ADB780220194693709DE733
:105F0000DB78344A19461520537597E7304B314CEE
:105F1000DB7819201946637602F0C0F9607E10F034
:105F2000010002D00020012100E0014605F0A0FAA6
:105F300010E1274B274ADB781620194693757DE739
:105F4000244A127D12F0010F05D0DB7813F0010F07
:105F500001D102F067FA1E4B1E4ADB781420194665
:105F600013756BE71A4B1B495A68DB78202043EA0C
:105F7000022341F8203F8AE7154B16495A68DB781F
:105F8000102043EA022341F8103F80E75A68DB788B
:105F900043EA0222012A00F2DA800E491A2001F8AF
:105FA0001A3F012274E70A4B5A68DB7843EA02225F
:105FB000012A00F2CC8007491B2001F81B3FF0E7C3
:105FC000034B0449DB78272001F8273FE9E700BFAE
:105FD000EC06002008000020640700205A68DB78E7
:105FE00043EA02225C4BC3F8D420B3E05B4B5A680F
:105FF000DB7843EA02225A4B1A60ABE0574B5A68EF
:10600000DB7843EA0222544BC3F8D820A2E0534B7A
:10601000DA78544B9DE05868D9785A78524B41EA67
:10602000002143F8221095E05A78272A59D00ED83B
:10603000022A33D004D8CAB1012A40F0868021E078
:106040001B2A3ED01C2A44D0092A7ED132E02B2ABA
:106050005FD005D8292A50D0D978444A54D847E08F
:106060002D2A64D05CD32E2A6FD167E05A68DB7882
:1060700043EA02223D4B1A6002F0F2FD364BC3F8B0
:10608000DC0067E05A68DB7843EA0222374B5A604B
:1060900002F0E6FD304BC3F8E0005BE05A68DB78C5
:1060A00043EA0222314B9A6002F0DAFD2A4BC3F830
:1060B000E4004FE05A68DB7843EA02222B4BDA60B7
:1060C00048E05968DB78002043EA012105F0CAFA6C
:1060D00040E05968DB78002043EA012105F096FA98
:1060E00038E05A68DB7843EA0222204B1A6131E03B
:1060F0005B6841EA032151612CE05A68DB7843EA8E
:1061000002221A4B9A6125E05B6841EA0321D161C2
:1061100020E05A68DB7843EA0222144B1A6219E045
:106120005A68DB7843EA0222104B5A6212E05A683E
:10613000DB7843EA02220D4B9A620BE05A68DB7867
:1061400043EA0222094BDA6204E0032200E004225F
:10615000074B1A7010BD00BF78020020EC0600202B
:10616000600700205D07002074070020240C002039
:106170006407002008B5824B9A78022A00F0B980A3
:10618000032A00F0BB80002A40F01E815B78502B70
:106190006ED022D8462B54D00ED8422B47D005D8EB
:1061A000402B3DD0412B40F00D813EE0442B43D0AD
:1061B000744B754A43D83DE04B2B4DD006D8482B45
:1061C00043D040D3492B40F0FD8042E04D2B49D0D5
:1061D00045D34F2B40F0F68047E0812B5FD010D89D
:1061E000542B4ED005D8522B47D0664B664A46D822
:1061F00041E0572B4BD0802B4DD0552B40F0E28007
:1062000042E0852B5DD004D8832B53D05D4B55D80D
:106210004DE0FE2B64D066D8F02B40F0D3805FE0D9
:1062200040F2FF7001F0A4FF9CE0574B59E0564B41
:106230005A78C4E01279C3E0534BDA69BFE052796F
:10624000BEE0514B85E0504B80E04F4B93F8262049
:10625000B5E04D4BDA7D48E04B4BDA78AFE04A4B86
:106260009A78ACE0484B5A7DA9E0474B5A7EA6E0AD
:10627000454B9A7DA3E0127DA2E0434B95E0126965
:106280009EE0414B9A7E9AE03F4BDA7E97E03E4B90
:1062900093F8272093E03D4B93F8D1208FE03B4BC0
:1062A00093F8D120042A14BF0022012287E0374A44
:1062B000926885E0354BD3F8D42080E0344A1268E8
:1062C0007EE0324A334BD2F8D8104B4303F54053AB
:1062D00039332C4923F000404860C2F8D83076E0CA
:1062E0002D4B1A786BE02D4B1A78003A18BF01221B
:1062F00065E05A782A4B53F8222060E05B78272B20
:1063000033D00DD8022B20D003D8C3B1012B59D1E3
:1063100018E01B2B1FD01C2B21D0092B52D117E0CA
:106320002B2B41D005D8292B24D0164B1D4A24D81D
:106330001EE02D2B3ED03AD32E2B43D13DE0194BFE
:106340001A683CE0174B5A6839E0164B9A6836E0F9
:10635000144BDA6833E0002004F0D2FF02E00020A2
:1063600004F0BAFF074B586031E00E4B1A6926E083
:10637000526925E00B4B9A6921E0D26920E000BF09
:10638000EC060020640700200800002078020020AE
:10639000600700206D4EC641580C00205D070020AC
:1063A00074070020240C0020124B1A6A07E0114BDE
:1063B0005A6A04E00F4B9A6A01E00E4BDA6A0E4B00
:1063C0005A6004E0032200E004220B4B1A700B4BCE
:1063D0001B786BB1084B0A495A680A4B0A601AB914
:1063E0001A6842F0080202E01A6822F008021A60F5
:1063F00008BD00BF240C0020640700205E070020B9
:106400004C070020F406002010B5154CA07818BBEE
:106410006378012B16D003D3022B124C19D114E050
:1064200004F0A0FAA17839B10F4A937FBBB102EB17
:106430004112927F9A4212D10C4B01221A71013AF9
:106440000B4B0BE004F096FA09E004F09BFA606055
:1064500005E00323237002E0024B04221A7010BDF2
:10646000EC06002064070020FC0B002078020020CE
:10647000940B002037B5504B1A7CA2B94F4948689D
:10648000CA7842EA0022B2F1FF3F04BF4C4A1268C8
:106490000A214A43C3F8E82002F0E2FB464B0122FE
:1064A0001A74C3F8EC00454B5B78042B00F2828031
:1064B000DFE803F003353F4F130002F0D1FB3E4B02
:1064C000D3F8EC10D3F8E820411A0029B8BF4942AC
:1064D00091426CD900221A746CE0384B364C987893
:1064E00004F050FA30B9374A2074136823F01003CF
:1064F00013605FE0D4F8E830002B57D002F0B0FB17
:10650000D4F8EC20D4F8E830821A002AB8BF5242FE
:106510009A424BD92B4B00211A68217442E000208B
:1065200004F088FD254B244C9D786D0050FA05F54C
:106530001CE000207C2101AA04F0B8FE1F4B0222BF
:106540009D789DF806306D0012FA05F51A4C1D4035
:106550000EE001AA00207C2104F0A8FE174A9DF855
:1065600006309578144C6D0053FA05F515F00105C9
:1065700006D0144B00211A68217422F0100213E097
:10658000D4F8E83093B102F06BFBD4F8EC20D4F8E7
:10659000E830821A002AB8BF52429A4206D9094B03
:1065A00025741A6842F010021A6003E0024B9A68E0
:1065B000013A9A603EBD00BF78020020EC06002040
:1065C0004C070020F406002008B5184B9A7812B149
:1065D000022A26D106E05868DB7843EA0020FDF75E
:1065E00015FF21E0587807280AD85A68DB7853EA63
:1065F000022202D1FDF7AEFE16E0FDF7B7FE13E072
:10660000FF280CD15868DB7843EA0020B0F1FF3F47
:106610000ABF074BC0B21878FDF7B4FE04E00322AE
:1066200000E00422034B1A7008BD00BFEC060020F6
:106630004C0700206407002010B5224B9A78012AED
:1066400023D003D3022A204C28D122E058780828EE
:1066500002D8FDF733FF15E00A2801D100220AE035
:106660000B2802D1FDF780FF0CE00C2806D1174B58
:106670009A68C2F34012144B5A6011E0FF280FD100
:10668000FDF740FF104B58600AE0587802F004FB19
:10669000F8E75878FDF78AFE606001E00423237074
:1066A0000B4B1B786BB1084B0A495A680A4B0A60BE
:1066B0001AB91A6842F0080202E01A6822F00802C9
:1066C0001A6010BDEC06002064070020000C014099
:1066D0005E0700204C070020F406002010B5204B78
:1066E0005A78812A3AD19A78922A37D19A79A32A6C
:1066F00034D15A79B42A31D11A79C52A2ED1DB780E
:10670000D62B2BD1174B4FF480621A6102F04CFE4E
:1067100002F0A6FA044602F0A3FA001B0028B8BF54
:106720004042B0F57A7FF6DBFDF75EFE06F0F4F945
:10673000002006F021FF00210B4805F0A3FD0A48C8
:1067400005F000FD094805F0D3FC05F0EBFD4FF026
:10675000804007F095FC0020FEF764F810BD00BFF4
:10676000EC060020000C014008000240002401401B
:106770002DE9F3479D4A9E4DD0785168137840EA41
:1067800001204FF0640C222B85F800C06B7068600C
:1067900000F0838554D80F2B00F03E8324D8072BBC
:1067A00000F00A8210D8032B00F0F88006D8012BE5
:1067B00000F0A680022B40F0B187C8E0052B00F066
:1067C000F38100F2F58101E10B2B00F0E88205D89E
:1067D000092B00F0DC8200F2DE82D4E20D2B00F007
:1067E000138300F21583F3E2192B00F0BD8412D855
:1067F000152B00F0C98306D8132B00F01183142B3E
:1068000040F08C8774E3172B00F08E84794B00F2F4
:106810009E8400F082BC1E2B00F0D08409D81B2B74
:1068200000F0C484C0F0B0841C2B40F0778700F0E7
:10683000C0BC202B00F0C88400F2C98400F0C1BCA9
:10684000812B00F0D8852ED8412B00F0BA8515D8C1
:10685000252B00F0688507D8232B00F02A85242BF0
:1068600040F05C8700F031BD272B00F09385C0F02D
:106870006585402B40F0528700F0A0BD452B00F00D
:10688000AC8506D8432B00F0A28500F2A38500F06A
:106890009BBD472B00F0A785C0F0A285802B40F060
:1068A0003D8700F0A3BD882B00F0478612D8842BCB
:1068B00000F0EC8507D8822B00F0B585832B40F0E3
:1068C0002D8700F0B5BD862B00F0FA8500F25586C5
:1068D00000F0F1BD8C2B00F09A8606D88A2B00F0D0
:1068E0007D8600F28F8600F076BEF22B00F0E78600
:1068F000FF2B00F005878D2B40F0108700F08ABE3B
:106900009378FBB93B4B4FF0010C83F804C03A4B32
:1069100000241C70394B21461C702046022204F0D2
:106920004DFC2046062140F2FF7204F0B3FD2F4BD0
:1069300020465A68DB78082143EA022204F0AAFDC7
:1069400000F0EFBE2A4B04221A7000F0EABE274D79
:10695000AC78F4B9274B4FF0010C83F804C0264BF8
:1069600021461C70254B20461C70022204F026FC98
:106970002046062140F2FF7204F08CFD6A68EB7835
:10698000204643EA02225242082104F083FD00F02F
:10699000C8BE174B04221A7000F0C3BE94788CB99D
:1069A000154B20461C70154B1C7003F0E3FF20466E
:1069B0002146022204F002FC2046082104F07EFD5C
:1069C00000F0AFBE04232B7000F0ABBE074B9A78EB
:1069D000002A40F0E4805B78032B00F2DB80DFE8E4
:1069E00013F00F0049009400BA0000BFEC0600202D
:1069F0006407002078020020F00B0020940B002098
:106A0000A64D0020FEF73AF9A54EAB780024686841
:106A1000EA78F454A34E590142EA0022F45401F0FA
:106A2000E001204604F0A2FCA9782246204604F0AA
:106A3000C5FBA9789C4A02EB41139B7F002B00F019
:106A40007086002900F06D86927F9A4240F0698638
:106A50002046FEF713F96A68EB78204643EA0222E3
:106A6000214604F083FC20462146224604F0A6FB82
:106A700000F057BE894D0020FEF700F9AB78884A38
:106A800000245901D454874A41F00201D45401F042
:106A9000E201204604F0B8FBEB786E68A97843EA7F
:106AA00006268619490101F0E0013246204604F02D
:106AB0005DFC2046A978224604F080FBA8787A4A3B
:106AC0007A4902EB40139B7F4E60002B00F0298631
:106AD000002800F02686927F9A4240F02286FEF738
:106AE000CDF80221204604F08FFB6A68EB7821463E
:106AF00043EA02228218204604F038FC2046214650
:106B0000224604F05BFB00F00CBE644CE378626844
:106B100043EA0223142B19DC654A002052F8236053
:106B2000FEF7ACF8A37832465D4E0025F5545D4E75
:106B30005901284601F0E001F55404F017FC2846FD
:106B4000A1782A4604F03AFB00F0EBBD574B042233
:106B50001A7000F0E6BD514C0020E3786268002511
:106B600043EA0222524B53F82260FEF787F8A378DB
:106B700032464B4E5901F5544A4E284601F0E00189
:106B8000F55404F0F3FB2846A1782A4604F016FBDE
:106B900000F0C7BD454B03221A7000F0C2BD434B45
:106BA00004221A7000F0BDBDFEF78AF800F0B9BDEE
:106BB000FEF7A6FB00F0B5BD907818B104232B704A
:106BC00000F0AFBD53789A2B21D8992B80F08480A8
:106BD000822B6FD00BD8062B4BD003D8042B3CD084
:106BE000052B0AE0072B4BD00C3B012B0CE08C2B28
:106BF00065D005D8832B30D0862B40F0BF8032E0A3
:106C00008D2B63D0933B022B00F2B8803FE0C82B62
:106C100000F083800FD8C12B6AD005D8B52B60D087
:106C2000C02B40F0AB802BE0C32B6FD067D3C72BBA
:106C300040F0A4801DE0D42B00F0848005D8CC2B3C
:106C400072D0D22B40F09A8075E0D62B00F088806D
:106C50007FD3FE2B40F0928089E00020062104F0D3
:106C600063FB00F05EBD00200C2104F05DFB00F032
:106C700058BD0D4B4920597A01F010FB00F051BD71
:106C8000094B4A20997A01F009FB00F04ABD002027
:106C9000142104F049FB00F044BD00BFEC060020C5
:106CA000940B0020F00B0020FC0B00206407002058
:106CB000F8060020042104F037FB00F032BD4B2021
:106CC000A149012201F06CFA00F02BBD00201A212D
:106CD00004F02AFB00F025BD182104F025FB00F08C
:106CE00020BD58209949042201F05AFA00F019BD3C
:106CF000974B4820197A01F0D1FA00F012BD4020DC
:106D00009349042201F04CFA00F00BBD4420914954
:106D1000042201F045FA00F004BD5F208E490122F3
:106D200001F03EFA00F0FDBC4E208C49022201F039
:106D300037FA00F0F6BC50208949042201F030FAFD
:106D400000F0EFBC54208749042201F029FA00F03A
:106D5000E8BC5E208449012201F022FA00F0E1BC87
:106D60005C208249022201F01BFA00F0DABC4C20C0
:106D70007F49012201F014FA00F0D3BC7D4B0322BD
:106D80001A7000F0CEBCFEF7D7FD00F0CABCFEF7CB
:106D9000EBFF00F0C6BCFFF7EDF900F0C2BC937842
:106DA000022B11D15378372B0AD8734903F5A770FA
:106DB00001EB83018000042201F0F2F900F0B1BC84
:106DC00003232B7000F0ADBC04232B7000F0A9BC92
:106DD0006A4B9A78022A12D15B78372B0AD8664917
:106DE00003F5A77001EB83018000023201F09CF9EA
:106DF00000F097BC5F4B03221A7000F092BC5D4B11
:106E000004221A7000F08DBCFFF7FEFA00F089BC76
:106E1000FFF7DAFB00F085BCFFF70EFC00F081BC49
:106E20005278574B092A53D8DFE802F0050D151D9B
:106E300026313941494C514A19685068D27842EAA2
:106E40000022521843E04D4A19685068D27842EA4D
:106E500000228A1A3BE0494A19685068D27842EA0F
:106E600000224A4333E0454A19685068D27842EA22
:106E7000002291FBF2F22AE0404819684468C27887
:106E800042EA042291FBF2F002FB10121FE03B4A9F
:106E900019685068D27842EA00220A4017E0374A5F
:106EA00019685068D27842EA00220A430FE0334A58
:106EB00019685068D27842EA00224A4007E01A680E
:106EC000D24304E02D4A5168D27842EA01221A6086
:106ED0002B4A2C4B12682AB91A6842F008021A6031
:106EE00000F01FBC1A6822F008021A6000F019BCFA
:106EF000224B234A5968DB78126843EA01239A42FD
:106F000006DD204B1A6842F0040222F003020CE076
:106F10001C4B05D11A6822F0060242F0010204E07F
:106F20001A6822F0070242F002021A60144A154B56
:106F3000126822B91A6842F008021A60F1E31A686E
:106F400022F008021A60ECE3070C0020140C002069
:106F5000FC0B0020000C00201B0C00200A0C002061
:106F60000C0C0020100C00201A0C0020180C002023
:106F7000080C00206407002074070020EC060020A5
:106F80004C070020F406002053780C2B00F2C98334
:106F9000DFE813F00D001B00290037004500530007
:106FA00061006F007D008B009900A700B500944B35
:106FB0001B6813F0080F00F0B483924B5A68DB781B
:106FC00043EA0222904B9A60ABE38D4B1B6813F0AF
:106FD000080F40F0A6838B4B5A68DB7843EA022205
:106FE000894B9A609DE3864B1B6813F0010F00F0FC
:106FF0009883844B5A68DB7843EA0222824B9A607A
:107000008FE37F4B1B6813F0010F40F08A837D4BA9
:107010005A68DB7843EA02227B4B9A6081E3784B23
:107020001B6813F0040F00F07C83764B5A68DB7802
:1070300043EA0222744B9A6073E3714B1B6813F0AE
:10704000050F00F06E836F4B5A68DB7843EA02222B
:107050006D4B9A6065E36A4B1B6813F0020F00F0FA
:107060006083684B5A68DB7843EA0222664B9A6079
:1070700057E3634B1B6813F0030F00F05283614B1F
:107080005A68DB7843EA02225F4B9A6049E35C4B23
:107090001B6813F0100F00F044835A4B5A68DB78DA
:1070A00043EA0222584B9A603BE3554B1B6813F0AE
:1070B000200F00F03683534B5A68DB7843EA0222F4
:1070C000514B9A602DE34E4B1B6813F0400F00F0BC
:1070D00028834C4B5A68DB7843EA02224A4B9A6079
:1070E0001FE3474B1B6813F0800F00F01A83454BDA
:1070F0005A68DB7843EA0222434B9A6011E3404B23
:107100001B6813F4807F00F00C833E4B5A68DB78D9
:1071100043EA02223C4B9A6003E33A4A5168D27830
:1071200042EA01229A60FCE2374BDA68072A00F251
:10713000F88234499C684868C97841EA0020511CAB
:1071400003EB8202C2F8F0409860D960E9E2DA68A5
:107150002D4B002A00F0E582013A03EB8201D1F8C1
:10716000F010DA609960DCE253782E2B03D8274ABE
:107170000121D154D5E2FF2B03D1234B01225A74B4
:10718000CFE203232B70CCE21E4B5B782E2B03D86F
:107190001E4A0021D154C4E2FF2B03D11A4B002216
:1071A0005A74BEE21A4B03221A70BAE2FFF762F970
:1071B000B7E2154B002283F8D120B2E2FEF732FB92
:1071C000AFE2FEF7B5FCACE2FEF76EFBA9E20D4ABA
:1071D000104B52780A2A52D8DFE802F0060B20251D
:1071E0002B33393F45494C000B491A6809688A1806
:1071F00003E0094A196812688A1A1A603FE000BF62
:10720000F4060020EC06002078020020740C002018
:10721000640700204C0700206C070020934A19687F
:1072200012684A43E9E7914A1968126891FBF2F241
:10723000E3E78E4A1968126891FBF2F002FB101224
:10724000DBE78A491A68096801EA0202D5E787493B
:107250001A68096841EA0202CFE784491A68096896
:1072600081EA0202C9E7814B1A68D243C5E71A686E
:107270007E4BC2E77D4A18681168106019607C4A2D
:107280007C4B126822B91A6842F008021A6048E280
:107290001A6822F008021A6043E2754B01F07F4140
:1072A00018681B7841EA10215160D370FDF708FD82
:1072B00037E26F4B01F07F4118681B7841EA1021DB
:1072C0005160D370FEF750FD2BE26B4B5B78052BC2
:1072D00000F22782DFE803F003090F151B21654B3D
:1072E0001A6802F00F021A601BE2624B1A6822F061
:1072F00010021A6015E25F4B1A6822F020021A6031
:107300000FE25C4B1A6822F040021A6009E2594B06
:107310001A6822F080021A6003E2564B1A6822F4BF
:1073200080721A60FDE153782E2B04D8534A02EB89
:1073300083035861F5E103232B70F2E14F4BDFF833
:1073400030C1D3F810914E4993F82C21D3F814A1F1
:10735000CCF80090DFF814C1D3F81871D3F81C8171
:10736000D3F82061D3F82451D3F82841CCF800A0F9
:10737000885CDFF800C19F60CCF800801E74C3F801
:10738000EC50C3F8E84008B101238B543B4B00227A
:107390009A74C6E193786BB9374B5B78142B05D898
:1073A000334A1168374A42F82310BAE1364B0322B8
:1073B0001A70B6E1344B04221A70B2E102F050F8B0
:1073C000AFE102F04FF8ACE102F04EF8A9E102F0B3
:1073D0004DF8A6E102F04CF8A3E102F04BF8A0E171
:1073E00002F04AF89DE102F049F89AE1234B0022AD
:1073F00083F8D12095E1537813B1012B10D104E02B
:107400001E4B012283F8D1208BE1B0F5006F04D22E
:107410001A4A906082F8D13083E104232B7080E116
:1074200003232B707DE1154B022283F8D12078E1F4
:10743000124B002199745974104A4FF0FF3402F135
:10744000140040F821400E480023435401312F29F5
:10745000F2D1084913740B60054982F8D1300B60F2
:10746000024993600B60D3605BE100BF6C070020B2
:107470004C070020F4060020EC06002078020020D3
:10748000740C0020F8060020640700208D4B1B7D43
:1074900013F0020F0CD1B0F5006F06D28A4B042214
:1074A000C3F8300183F8D1203BE104232B7038E18D
:1074B00008232B7035E1844B002283F8D12030E182
:1074C000804B01219A78814BB0F5006F1970804B89
:1074D0001A7028D27B4B1C7D0C4024D1694600F0E9
:1074E000E5FF7B4B9DF800709DF801609DF8025010
:1074F0009DF806C09DF805009DF804109DF8032036
:107500001C725F709E70DD7083F804C058719971B1
:10751000DA7101236E4A985C117A01334118082B05
:107520001172F7D1FDE00123694A0021995401331A
:10753000082BF9D113781372F3E053788BB9614AB1
:1075400001209178634A1468604A1070604A117093
:107550000133E21812F8011C5D4A082B9954F7D147
:10756000DFE0012B40F0DD801B222A710422EA714A
:107570006FF07602AA716B71D3E0574B5B78032BE7
:1075800000F2CF80DFE803F002101D224E4A534B79
:10759000D2F8301192F8D1C0107C0A0A197183F820
:1075A00007C098715A71BCE0474A4C4B916892F8F9
:1075B000D1C0107C0A0A197183F807C098715A71FA
:1075C000AFE0474B1A68454B5A60AAE0454B1A6832
:1075D000424B5A60A5E0FEF7ADFBA2E05278424B69
:1075E00002B101221A703C4B404AD878364B1070D9
:1075F00093F834113E4A002311703E4A13703E4AFC
:1076000013708EE0304B012283F8352189E0FEF7BC
:10761000DBFA86E0304B5B78032B4CD8DFE803F0D5
:107620000C023C472C4B28495A68DB78D1F83811BA
:1076300043EA022C00232BE0234BD3F83821092AFC
:107640000CD82549501C4C68C97803EB820241EAEA
:107650000421C2F83C11C3F8380162E01F4B092233
:107660001A705EE052F82340581C64450FD102EBBB
:107670008002013904E052F8040C013342F8080C8E
:1076800004328B42F7D3104BC3F8381149E003465C
:107690008B421A4AE6D344E00B4A0023C2F8383141
:1076A000164A0021D1500433282BF9D139E00B4B75
:1076B0000A225A6035E0094B03221A7031E0FFF7C5
:1076C0000DF82EE00800002078020020500700206E
:1076D0005407002000000020EC0600206407002072
:1076E0004C0700206C070020800B00209C0B002022
:1076F000620C0020A30C0020950B0020B403002096
:10770000094B5A68DB7843EA022240F2D2439A429C
:1077100007D1064B012283F8642102E0044B0222C8
:107720001A70BDE8FC8700BFEC060020780200203C
:107730006407002073B5204B024640781F4D187037
:10774000907800265870D078EC46987010790C46E6
:1077500098715079587192F806E095E8030083F823
:1077600004E0D2798CE80300DA70154B1E70FEF746
:10777000FFFF144B1B7873B9637023702B78A370D1
:107780006B78E370EB792371AB7963716B79A371DB
:107790002B79E37108E0012B06D10B4B9B195B7829
:1077A000A3550136082EF8D1044B6A4692E803002F
:1077B00083E803007CBD00BFEC06002064070020C6
:1077C0005E0700205007002054070020F7B5114D38
:1077D000114C6F684FF0000C07F07F4747EA132702
:1077E0006F600E4F6E4687F800C028706970AA70EF
:1077F00094E80300EB7086E80300FEF7B9FF96E813
:1078000003006368227884E80300054918460A707B
:10781000FEBD00BFEC060020640700205E070020CC
:10782000780200202DE9F04F7E4B93B01B781BB9F6
:107830007D4B93F865316BB17C4B1B78062B09D0DF
:107840000A2B07D00F2B05D01F2B03D0764B00221D
:1078500083F83421744A92F83431032B25D192F8FD
:10786000D040002C40F0D980714B1B7893B9714DFA
:10787000714CA8786E78227863788619B618E27908
:10788000F618A379B6186279F6182379B618F6189F
:10789000F6B219E0012B40F0FE80684BE05C013449
:1078A00000F040FF092CF8D1F5E0042B27D1614D01
:1078B000614CAB786E7818469E1901360023012280
:1078C00022706360F6B2637000F02CFF687800F0FD
:1078D00029FF207800F026FF607800F023FFE07990
:1078E00000F020FFA07900F01DFF607900F01AFF82
:1078F000207900F017FF304600F014FFCBE0052B95
:1079000025D192F8D040002C40F08780484B1B785E
:1079100093B9484D484CA8786E78227863788619D8
:10792000B618E279F618A379B6186279F6182379B1
:10793000B618F618F6B219E0012B40F0AC803F4BB8
:10794000E05C013400F0D2FE092CF8D1A3E0062B54
:1079500027D1384D384CAB786E7818469E190136D1
:107960000023012222706360F6B2637000F0BEFE55
:10797000687800F0BBFE207800F0B8FE607800F078
:10798000B5FEE07900F0B2FEA07900F0AFFE6079BC
:1079900000F0ACFE207900F0A9FE304600F0A6FE13
:1079A00079E0072B4ED192F8D030002B35D1204A08
:1079B000127822BB1F4A204B557896781C7893F892
:1079C00001C0AF19D879E719997967445A79C7196D
:1079D0001B79CF19D719DF198DF838708DF8306001
:1079E0008DF831508DF832408DF833C08DF8340069
:1079F0008DF835108DF836208DF8373008E0012AE3
:107A000006D10E4A995C0CAAD1540133092BF8D146
:107A10000B4B1B78002B3ED039E0074803F088FF62
:107A200039E000BF5D07002078020020EC0600204E
:107A300050070020080000206407002054070020A1
:107A4000780B0020082B26D1954B00225978987886
:107A5000944B45181C78944B4FF0010C01355A603B
:107A60008DF832C08DF8332016468DF834208DF80D
:107A700035208DF836208DF837208DF838505A7023
:107A800083F800C08DF830008DF831101CB10CA8BF
:107A9000092101F057FB854B1B78002B56D0844BF6
:107AA0001B78032B02D0072B4BD123E07C4C814D5C
:107AB000A07866782B7886190A36F61800F032FE20
:107AC000607800F02FFE802000F02CFE8A2000F06D
:107AD00029FE002000F026FE002000F023FE0020FA
:107AE00000F020FEF6B2287800F01CFE304600F0D0
:107AF00019FE26E06A4B6FF07F05597898786D4B38
:107B000000EB010C1A78674B0CF10A0C1C789444BA
:107B100000238DF826500A358DF827508DF82A302D
:107B20008DF82CC08DF824008DF825108DF82830A4
:107B30008DF829308DF82B201CB109A8092101F0FE
:107B400001FB5A4A002313705A4A13705A4B5B4880
:107B500093F864110022027083F8652183F83421C0
:107B600011B10120FCF75EFE534B93F8352152B161
:107B700093F8D0200021D2F1010238BF002283F80F
:107B8000351183F8D0204C4C94F8D050002D72D190
:107B90000DF1470000F044FD00286CD000F05CFDC2
:107BA00008B184F86651444B9DF8470093F866117C
:107BB0004A1CD2B2C918092A81F8680183F86621E3
:107BC00040F07681364993F8682148784FF0000CF0
:107BD000904283F866C107D091F82730002B00F05F
:107BE00067819A4240F064812D4B93F8273093428D
:107BF00003D1314B012283F8652100231A462E4C14
:107C000004F5B471C95C01335218082BD2B2F6D115
:107C100094F8703193422CD1294B94F86D1194F85B
:107C20006E2194F86F5194F8696194F86AE194F8C0
:107C30006BC194F86C01DD7059711A711E7083F874
:107C400001E083F802C0987101F00AF81D4D94F824
:107C5000D1302860591E1C480022C9B2027003208E
:107C6000012984F8340184F8662140F2EE80052B66
:107C7000A0E00423EDE0104C94F8D03033B310486A
:107C800003F09CFE10B300F0EBFF0E4994F8D130E6
:107C900008600D495A1E00200870D2B20321CEE0C0
:107CA00008000020780B002064070020A30C0020AF
:107CB000620C0020950B0020780200205007002065
:107CC000EC0600205C0C0020610C00206F4C94F846
:107CD000D050002D73D10DF1470000F0C7FC0028F3
:107CE0006DD000F0E1FC08B184F86651674B9DF857
:107CF000470093F866114A1CD2B2C918092A81F8C4
:107D0000680183F8662140F0D380614993F86821C7
:107D100048784FF0000C904283F866C107D091F884
:107D20002730002B00F0C4809A4240F0C180584BAD
:107D300093F82730934203D1544B012283F86521F5
:107D400000231A46514C04F5B471C95C0133521832
:107D5000082BD2B2F6D194F8703193422DD14D4B0D
:107D600094F86D1194F86E2194F86F5194F869614C
:107D700094F86AE194F86BC194F86C01DD70597164
:107D80001A711E7083F801E083F802C0987100F048
:107D900067FF414D94F8D1302860591E3F480022BA
:107DA000C9B202700520012984F8340184F86621E3
:107DB0004BD9834249D0013248E0062349E0334B96
:107DC00093F8D040002C47D1354B1B78002B43D083
:107DD0000FA801F0A1F900283ED0234622460FA9A2
:107DE000C95C01335218082BD2B2F8D19DF8441067
:107DF000264C91422DD1274B9DF841109DF84220F1
:107E00009DF83D609DF83EE09DF83FC09DF8400024
:107E10009DF8435059711A711E70DD7083F801E0AE
:107E200083F802C0987100F01BFF1B4994F8D13011
:107E300008601A495A1E00200870D2B20721012A90
:107E400084F8341101D9052B1ED10022154B1A706C
:107E50002EE084F834312BE00C4C94F8D130013B07
:107E6000DBB2012B24D8A368B3F5006F1CD2FCF75A
:107E7000F7FAC8B1A368074918460133A36000F0B8
:107E800015FB092384F834310122DFE77802002052
:107E900008000020EC0600205C0C0020610C002093
:107EA000780B00205E070020964B002283F8D1203B
:107EB000944C94F8D130042B05D1934E327812F0C3
:107EC000800F00F0EF808F4B93F834313BB1042BDF
:107ED00005D0082B03D0062B01D0FEF749FC894CB6
:107EE00094F83431092B40F0B28000F0B9FED4F898
:107EF000DC30864AC31A002B1268B8BF5B4293423B
:107F00000AD9834B1A78012A01D101321A7000F084
:107F1000A7FE7C4BC3F8DC0000F0A2FE794BD3F83F
:107F2000E0207A4B821A002A5B68B8BF52429A421C
:107F30000AD9774B5A78012A01D101325A7000F0E0
:107F40008FFE704BC3F8E00000F08AFE6D4BD3F853
:107F5000E4206E4B821A002A9B68B8BF52429A42B4
:107F60000AD96B4B9A78012A01D101329A7000F03C
:107F700077FE644BC3F8E400624A537C002B66D062
:107F8000937C002B63D19C46624B92F82C011B68BA
:107F900002900793604BD2F8E8001B6803900693A9
:107FA0005E4BD2F810811B68D2F814710593D2F899
:107FB000EC30D2F818410493D2F81C619368107C1D
:107FC000D2F82051D2F824B1D2F828210192624689
:107FD000DFF83C91194619F802A0BAF1020F18D146
:107FE0004F4951F82210B1F1FF3F0ED00546D0B2F3
:107FF00002900398DDF810B00190059E069FDDF811
:108000001C804FF0010C002004E0002109F8021050
:108010001946234601322F2A02D01C460B46D7E7C9
:10802000384AC2F818311074019B029882F812C0C5
:10803000C2F81081C2F814719160C2F81C61C2F8D4
:108040002051C2F824B1C2F8283182F82C012D4BFE
:1080500093F83421092A06D193F8D120022A02D1BB
:10806000033283F8D120274BD3F83811002946D0AA
:1080700093F83421092A42D193F8D120012A3ED124
:108080009868002308E054F823400133A04203D14C
:10809000052382F8D13032E01A4A8B4202F59E74F1
:1080A000F1D32CE094F834314BB3042B27D0082BB8
:1080B00025D0062B23D0F3787168D4F83001194D00
:1080C00043EA0123B0F5006F6A706B6012D231464B
:1080D00000F01CF93146D4F8300100F03FF930B11E
:1080E000D4F830310133C4F83031652300E0072380
:1080F0002B7004E007232B70002384F8D13013B0D9
:10810000BDE8F08F78020020EC060020240C00204F
:10811000740C00204C0700206C070020F40600209F
:108120008C0200206407002070B5044600200E4633
:10813000154603210246FCF723FC0020C4F3072167
:108140000246FCF71DFC0020E1B20246FCF718FCD9
:10815000002407E0944214BF00220122FCF710FC27
:108160003055013400206A1EAC420146F2D370BD86
:1081700010B50446002003210246FCF701FC002054
:10818000C4F307210246FCF7FBFB0020E1B20246E4
:10819000FCF7F6FB002001460122FCF7F1FB10BDC5
:1081A0002DE9F04104460F46164600200621012223
:1081B000FCF7E6FB002005210246FCF7E1FB00206E
:1081C00001220146FCF7DCFB10F0020FF2D0002088
:1081D00002210246FCF7D4FB0020C4F3072102462B
:1081E000FCF7CEFB0020E1B20246FCF7C9FB0025FC
:1081F00043E0013414F03F08795D01D1012204E02D
:10820000721E954214BF002201220020FCF7B8FB29
:10821000B8F1000F30D1731E9D422DD200200521F0
:108220000246FCF7ADFB002001220146FCF7A8FB4B
:1082300010F00100F2D106210122FCF7A1FB002081
:1082400005210246FCF79CFB002001220146FCF7B9
:1082500097FB10F0020FF2D0002002210246FCF73B
:108260008FFB0020C4F307210246FCF789FB0020A6
:10827000E1B20246FCF784FB0135B542B9D30020D8
:1082800005210246FCF77CFB002001220146FCF799
:1082900077FB10F0010FF2D1BDE8F08138B5012273
:1082A00004460D4600200621FCF76AFB002005214C
:1082B0000246FCF765FB002001220146FCF760FB4B
:1082C00010F0020FF2D0002002210246FCF758FB0A
:1082D0000020C4F307210246FCF752FB0020E1B264
:1082E0000246FCF74DFB294600200122FCF748FB23
:1082F000002005210246FCF743FB00200122014635
:10830000FCF73EFB10F0010FF2D138BD38B5072560
:10831000454305F500650C46284609780135FFF709
:10832000BDFF284661780135FFF7B8FF2846A178E0
:108330000135FFF7B3FF2846E1780135FFF7AEFFBF
:10834000284621790135FFF7A9FF28466179FFF713
:10835000A5FF681CA179FFF7A1FF38BD2DE9F34700
:108360000725454300200C4602460321FCF708FB85
:1083700005F500650020C5F307210246FCF700FB68
:108380000020E9B20246FCF7FBFA00200146024653
:10839000FCF7F6FA8246002001460246FCF7F0FAA6
:1083A0008046002001460246FCF7EAFA0746002014
:1083B00001460246FCF7E4FA8146002001460246E7
:1083C000FCF7DEFA0646002001460246FCF7D8FA22
:1083D0000546002001220146FCF7D2FA23785345D6
:1083E0001DD1637843451AD1A378BB4217D1E378F6
:1083F00021798DF804608DF805508DF806006279BA
:1084000043EA012343EA0243A079019A43EA006068
:1084100049EA0229814514BF0020012000E0002024
:10842000BDE8FC8738B54FF4006400200621012226
:10843000FCF7A6FA002005210246FCF7A1FA00206D
:1084400001220146FCF79CFA10F0020FF2D0002046
:1084500002210246FCF794FA0020C4F307210246E9
:10846000FCF78EFA0020E1B20246FCF789FA0025FB
:1084700000203F2D14BF0022012201460135FCF7E8
:108480007FFA402DF4D1002005210246FCF778FA4E
:10849000002001220146FCF773FA10F0010FF2D11F
:1084A0004034B4F5804FC0D138BD00BF38B5072582
:1084B000454300200C4602460321FCF761FA05F50E
:1084C00000650020C5F307210246FCF759FA002099
:1084D000E9B20246FCF754FA002001460246FCF7D6
:1084E0004FFA2070002001460246FCF749FA6070FE
:1084F000002001460246FCF743FAA0700020014626
:108500000246FCF73DFAE070002001460246FCF707
:1085100037FA2071002001460246FCF731FA6071FB
:10852000002001460122FCF72BFAA07138BD00BFE4
:1085300037B5002005210246FCF722FA002001226F
:108540000146FCF71DFA10F07104F2D100F088FB2F
:10855000054605E0FFF70CFE422814BF0024012465
:1085600000F07EFB431B002BB8BF5B42B3F5FA6FF4
:1085700040F2FF7002DA002CECD000E01CB1234B7B
:108580001B78002B36D040F2FF700021FFF786FEEB
:10859000FFF748FF00201E494022FFF701FE4FF47D
:1085A00080701C49B422FFF7FBFD40201A492022AD
:1085B000FFF7F6FD002301934FF4C36401AD20469D
:1085C000042204342946FFF7EBFDB4F5FF6FF5D123
:1085D00000230193A4F53074204604220434294674
:1085E000FFF7DEFDB4F5C36FF6D140F2FF70422114
:1085F000FFF754FE002040220549FFF795FD40207B
:1086000006492022FFF790FD3EBD00BFA40B0020CD
:10861000080000200018010830180108FC0B002099
:10862000094B19685A68914201D100200BE01A6881
:10863000D118097A013201701A601A68202A01D112
:1086400000221A6001207047EC030020014B986261
:10865000704700BFEC030020034B1A78104612B19C
:1086600000221A7001207047B40C00200A4BD96A0E
:108670001A6B914201D100200CE0DA6AD11891F80E
:10868000341001320170DA62DA6A202A01D1002244
:10869000DA620120704700BFEC030020014B5865EF
:1086A000704700BFEC030020034B1A78104612B14C
:1086B00000221A7001207047B50C002008B5FBF7A6
:1086C00093FE034B0022DA621A63FBF78BFE08BDB0
:1086D000EC03002008B5FBF787FE034B00221A606D
:1086E0005A60FBF77FFE08BDEC03002038B50B4B4A
:1086F00084469C6DDA6D0134202C08BF002494421E
:108700000AD09D6D0648ED1885F860C040F22771CB
:1087100001229C6505F04CFD38BD00BFEC03002034
:108720000044004038B50D4B8446D3F88040D3F860
:1087300084200134202C08BF002494420CD0D3F8AC
:1087400080500748ED1885F888C040F22771012253
:10875000C3F8804005F02CFD38BD00BFEC030020BD
:108760000038014038B50546002401E0FFF7DAFF84
:108770002B5D01341846002BF8D138BD2B4910B5BC
:108780000B8813F0200F1DD0294BDB6813F0020F6C
:1087900001D08B8816E0274B1A6BD86A0132202A49
:1087A00008BF0022824206D01C6B8888E118C0B244
:1087B00081F834001A63204B0A221A601D4B5A6D4F
:1087C0001E4B1A601948038813F0800F1BD01B4BF7
:1087D0001A68C2B9174B9C6DD96D8C420FD01449E1
:1087E00002240C61D96DCC1894F860C00131A0F856
:1087F00004C0D965D96D202905D1DA6503E040F2BE
:10880000277105F0D5FC0948038813F0400F0BD001
:1088100040F2266105F0C4FD064BDA6D9B6D9A426D
:1088200002D1034B02225A6110BD00BF0044004038
:1088300000080140EC030020A40C0020AC0C002038
:10884000274910B50B8813F0200F15D0254B5A6817
:1088500018680132202A08BF0022824205D05C68D5
:108860008888E118C0B208725A601F4B0A221A6049
:108870001C4B9A6A1D4B1A601948038813F0800F2D
:108880001ED01A4B1A68DAB9164BD3F88040D3F8C9
:1088900084108C4210D0D3F88410CC1894F888C07F
:1088A0000131A0F804C0C3F88410D3F88410202943
:1088B00006D1C3F8842003E040F2277105F078FC6C
:1088C0000748038813F0400F08D040F2266105F0F6
:1088D00067FD044BD3F88420D3F8803010BD00BF6F
:1088E00000380140EC030020B00C0020A80C002050
:1088F00030B5054687B0564805F0A2FD4FF400306C
:10890000012104F0EBFB0420012104F0D9FB042039
:10891000002104F0F1FB0820002104F059F806AC16
:108920004FF0040324F8083D03234A4821468DF8FC
:10893000123015338DF8133003F0BAFF4823454841
:108940008DF8133021464FF00803ADF8103003F0D6
:10895000AFFF684605F0F6FB0B2D25D8DFE805F0E4
:108960002406090C0F1215181B1E20224FF4615308
:108970001CE04FF4964319E04FF4E14316E04FF446
:10898000164313E04FF4614310E04FF496330DE0CB
:108990004FF4E1330AE04FF4613307E02E4B05E07A
:1089A0002E4B03E02E4B01E04FF416530093009B37
:1089B00006A95B0841F8183D2548694605F0F8FC12
:1089C00026230024012505A88DF8143007238DF8EF
:1089D00015308DF816408DF8175004F0D9F81C4862
:1089E00040F2FF3105F0B8FC28212246184805F076
:1089F000DFFB2A46164840F2277105F0D9FB2A46CC
:108A0000134840F2266105F0D3FB2A46104840F295
:108A1000255105F0CDFB22460D4840F2244105F0DA
:108A2000C7FB22460A4840F6460105F0C1FB224634
:108A3000074840F66A1105F0BBFB60212246044856
:108A400005F0B6FB2946024805F0A4FB07B030BD8F
:108A5000004400400008014090D0030020A107001E
:108A600040420F0030B5054687B0524805F0E8FC9B
:108A70004FF48040012104F023FB0420002103F087
:108A8000A7FF06AC4FF4007324F8083D03234A48BF
:108A900021468DF8123015338DF8133003F008FF9E
:108AA000482345488DF8133021464FF48063ADF8D4
:108AB000103003F0FDFE684605F044FB0B2D25D871
:108AC000DFE805F02406090C0F1215181B1E2022E2
:108AD0004FF461531CE04FF4964319E04FF4E14327
:108AE00016E04FF4164313E04FF4614310E04FF4E7
:108AF00096330DE04FF4E1330AE04FF4613307E0C1
:108B00002E4B05E02E4B03E02E4B01E04FF41653A5
:108B10000093009B06A95B0841F8183D254869466B
:108B200005F046FC25230024012505A88DF8143006
:108B300007238DF815308DF816408DF8175004F086
:108B400027F81C4840F2FF3105F006FC2821224698
:108B5000184805F02DFB2A46164840F2277105F00B
:108B600027FB2A46134840F2266105F021FB2A46DE
:108B7000104840F2255105F01BFB22460D4840F2FB
:108B8000244105F015FB22460A4840F6460105F04F
:108B90000FFB2246074840F66A1105F009FB6021E9
:108BA0002246044805F004FB2946024805F0F2FA83
:108BB00007B030BD003801400008014090D00300EC
:108BC00020A1070040420F00704700BF1B4B1A78DE
:108BD000AAB159681A4A013159601168194B01311B
:108BE00011601A6812B11A68013A1A60164B1A68B5
:108BF00012B11A68013A1A600022104B00E00122FB
:108C00001A70124B1A683AB11A68013A1A601B6856
:108C100013B90F4B01221A700E4B1A683AB11A6839
:108C2000013A1A601B6813B90B4B01221A700B4BE7
:108C30001A6812B11A68013A1A6070479404002049
:108C400060070020A80C0020AC0C0020B00C002015
:108C5000B40C0020A40C0020B50C0020E806002075
:108C6000014B5868704700BF9404002008B50420E9
:108C700004F056FC4FF4FA5004F062FC012004F0BA
:108C800065FC04480321002204F050F8012004F0A0
:108C900073FC08BD9AC302000828F8B508D009285B
:108CA0000ED008B100205AE03B4B188880B256E045
:108CB000394B588840F26B1380B2584300134EE092
:108CC000354B988880B207F0E5FF07F0C7FB00221C
:108CD000324B07F017FC22A3D3E9002306460F46C8
:108CE00007F010FC20A3D3E9002307F059FA1EA3D4
:108CF000D3E9002304460D463046394607F002FC0E
:108D00001BA3D3E9002307F027FD02460B462046AC
:108D1000294607F021FD07F0B7FE07F09FFB002270
:108D20001F4B07F019FD06F041FE13A3D3E9002302
:108D300007F0E8FB12A3D3E9002307F031FA02465B
:108D40000B4611A1D1E9000107F006FD10A3D3E9FC
:108D5000002307F023FA07F097FE08F0B9F9F8BDF1
:108D60006666666666660AC06666666666660A4027
:108D70009A99999999990140C3F5285C8FA27240FC
:108D80000000000000FEAA409A999999FD6F2F41BA
:108D9000C3F5285C8F1271409C0400200000303F16
:108DA00000002440F0B593B011AF01240025032644
:108DB00040483946ADF844408DF846608DF847503C
:108DC00003F076FD39463C48ADF844608DF84660C6
:108DD0008DF8475003F06CFD2046214604F062F9FF
:108DE00021464FF4007004F06BF9344803F0AAF9FF
:108DF000334B32480193334B01A9029380230693EE
:108E0000DB18079303F540730893A3F57873099370
:108E100003F5FF530A930395049605950B9503F00C
:108E200001FA2648214603F02DFA4FF46023264824
:108E30000CA90E938DF834400C958DF835400F95A4
:108E40008DF8406002F0B2FF1F48082122463346E9
:108E500003F02EF81C4829460222334603F028F876
:108E6000334632461848092103F022F82A461648AC
:108E70004FF4FC6102F0DEFF1348214602F0D0FF00
:108E80001148214602F0C2FF0F4802F0DDFF0E48F4
:108E900002F0E0FF0028FAD10B4802F0DFFF0A4899
:108EA00002F0E2FF0028FAD10748012102F0E0FFBA
:108EB00013B0F0BD00080140000C01400800024062
:108EC0004C2401409C04002000240140AFF30080AA
:108ED000014B03221A607047A4040020044A054B8A
:108EE000927A0AB1052200E001221A60704700BFA1
:108EF000C40C0020A4040020704700BF014B0022D6
:108F00005A607047A404002008B5074B1A6892B253
:108F100042F008021A601A6892B242F004021A6023
:108F2000FFF7D6FF08BD00BF405C004010B5064CFF
:108F30004FF6FB73226802EA03032360FFF7CEFFBC
:108F40004FF40643236010BD405C0040072818BF63
:108F50001F4B10B51E4C18BF18702378052B33D843
:108F6000DFE803F003060A0E1621FFF7DFFF2BE010
:108F7000FFF7DCFF042328E002236370013324E0C1
:108F80006378013BDBB263706378FBB9042218E0BD
:108F9000104B1A6892B242F010021A600523237037
:108FA000DB18637012E06378013BDBB263706378B7
:108FB00063B9084A4FF6EF73116801EA03031360BF
:108FC0000622034B1A7001E00623237010BD00BF78
:108FD000280D0020405C0040034B9B7A13B1034BEB
:108FE00005221A60704700BFC40C0020A4040020B2
:108FF000014B04221A607047A4040020034B1A7A24
:10900000202A01D100221A72704700BFA404002058
:10901000704700BF212808B508D1124B1B681B7888
:1090200003F07F03212B1AD10F4B0EE0202816D11D
:109030000C4B0E4A1B681B7810720D4A03F07F031D
:10904000212B0CBF134600234BB1064A4FF0000101
:1090500012680020518293619847002000E00220AE
:1090600008BD00BF240D0020A9900008A404002022
:10907000C5900008074B1B681B7803F07F03212B6A
:1090800005D1022801D0222801D1002000E00220D1
:10909000704700BF240D002019B9012801D80846E7
:1090A00000E00220704700BF28B9044B4FF00802CF
:1090B0001B681A8200E00248704700BF240D0020A0
:1090C0004800002028B9044B4FF008021B681A82A0
:1090D00000E00248704700BF240D00204800002037
:1090E0000B4B10B5DA6882B11B68052B01D000224A
:1090F0000BE0002303E00749595CC15401330449E4
:10910000CC68A342F7D30023CB60104610BD00BF4C
:10911000A40400202C0D0020084BDB68082B01D88C
:1091200000200AE00023064A9A5CC2540133092B4E
:10913000F9D1024B0022DA6001207047A40400201C
:109140002C0D002010B5074C0B468AB2C02163607D
:1091500005F052FF0120A18806F05CF9012006F01D
:1091600027F810BDA404002007B5142200238DF8B1
:10917000042001A801228DF806308DF807208DF813
:10918000053003F005FD0EBD07B5142200238DF850
:10919000042001A801228DF806308DF807208DF8F3
:1091A000053003F0F5FC0EBD08B5064B1B68DB78F7
:1091B000042B01D9002004E0034901EBC30105F0B1
:1091C000C3FA08BD240D00205000002008B5024954
:1091D00005F0BAFA08BD00BF7000002008B50249CA
:1091E00005F0B2FA08BD00BF78000020334B10B57F
:1091F0001B686FF03F0200245A72DC729C7220469A
:1092000005F04EFF20464FF4007105F067FF102176
:10921000204605F079FF4021204606F0CFF8802156
:10922000204606F0BBF8204605F0F8FF244B204608
:1092300093F8641006F010F9204605F0C7FF0120EE
:10924000214605F04BFF0120C02106F0A7F80120C0
:10925000202105F059FF0120214605F06DFF022075
:109260004FF4C06105F03AFF02204FF4807106F020
:1092700095F80220214605F05FFF0220202105F02D
:1092800043FF0320214605F029FF03204FF4887196
:1092900006F094F80320402106F0DEF803204FF496
:1092A000405105F049FF2146032005F02DFF2046DF
:1092B00005F058FA034B01221A6010BD240D00205E
:1092C00048000020A404002008B5174B174A19686D
:1092D00089B2118016491288098801EA020212F443
:1092E000806F05D04FF6FF321A60124BDB6B984748
:1092F0000E4B1A880E4B1B8803EA020212F4007F01
:1093000008D009490C4A4FF6FF500860117C013122
:10931000C9B21174054A1288134013F4004F01D0EA
:1093200005F0A6FD08BD00BF445C0040BA0C00205B
:109330006C0D002048000020A404002010B503207C
:1093400006F0BAF8064C034602464FF48871054809
:10935000E36005F069FE032005F038FF10BD00BF93
:10936000A40400202C0D002008B520B104481021D1
:1093700003F004FB03E00248102103F001FB08BDE9
:10938000000C014038B5064D01232B60054B00242D
:1093900020461C60FFF7E8FF03232B60204638BD02
:1093A000405C0040445C004008B5FFF7EBFF08BD9F
:1093B00008B50120FFF7D8FF064B012119600649C7
:1093C0004FF4E0520A8005490020186008601A60D6
:1093D00008BD00BF405C00406C0D0020445C0040B4
:1093E000084B10B51B6800249C72FFF7E1FF064A8A
:1093F0004FF406431460043A1360044A1460044AAC
:10940000138010BD240D0020445C0040A404002003
:109410006C0D0020012008B503F0C8FD4FF40000DA
:10942000012103F05BFE08BD07B5FFF7F3FFFFF76F
:10943000ABFE05F0BFFC0820012103F041FE102324
:109440000322054801A98DF806208DF80730ADF8F4
:10945000043003F02DFA0EBD000C0140704700BF30
:10946000704700BF704700BF704700BF704700BF24
:10947000704700BF704700BF704700BF08B5FBF7DB
:1094800053F8052805D9FBF74FF840F2F933984215
:1094900001D9012200E00022094B5A60094B1B78D8
:1094A0006BB1074B08495A68084B0A601AB91A6829
:1094B00042F0080202E01A6822F008021A6008BDB1
:1094C000640700205E0700204C070020F4060020FF
:1094D00010B5FFF7C5FB074C2368C31AB3F5FA7F35
:1094E00007D9054BDA6882F40072DA60FFF7B8FB3F
:1094F000206010BD700D0020000C0140024B03EBFA
:10950000C003D879704700BFB8040020024B03EBBA
:10951000C0035879704700BFB8040020024B03EB2A
:10952000C0039879704700BFB8040020024B0B229B
:1095300002FB0033187A7047B8040020024B0B225C
:1095400002FB0033587A7047B8040020024B0B220C
:1095500002FB0033D87A7047B8040020024B0B227C
:1095600002FB0033987A7047B8040020024B0B22AC
:1095700002FB0033187B7047B8040020024B0B221B
:1095800002FB0033587B7047B8040020024B0B22CB
:1095900002FB0033987B7047B8040020024B0B227B
:1095A00002FB0033187C7047B8040020024B0B22EA
:1095B00002FB0033587C7047B8040020024B0B229A
:1095C00002FB0033987C7047B8040020024B052250
:1095D00002FB0033187D7047B8040020024B0522BF
:1095E00002FB0033587D7047B8040020024B05226F
:1095F00002FB0033987D7047B8040020024B05221F
:1096000002FB0033D87D7047B8040020024B0522CE
:1096100002FB0033187E7047B8040020024B03227F
:1096200002FB0033187F7047B8040020034B03226D
:1096300002FB003393F91D00704700BFB8040020FF
:10964000024B032202FB0033987F7047B8040020CE
:10965000024B03EBC00393F820007047B8040020CE
:10966000024B03EBC00393F821007047B8040020BD
:10967000024B03EBC00393F822007047B8040020AC
:10968000024B03EBC00393F823007047B80400209B
:10969000024B03EBC00393F824007047B80400208A
:1096A000024B03EBC00393F825007047B804002079
:1096B000024B03EBC00393F826007047B804002068
:1096C000024B03EBC00393F827007047B804002057
:1096D00006281AD8DFE800F004070A0D1013160058
:1096E0000A4B9B6A10E0094BDB6A0DE0074B1B6BD2
:1096F0000AE0064B5B6B07E0044B9B6B04E0034BFB
:10970000DB6B01E0014BDB7B0B607047B804002092
:1097100070B5C0F30741054600220120FBF730F980
:109720000A4C0602C5F3072100220120A662FBF7BE
:1097300027F9064301203602E9B20246A662FBF78A
:109740001FF906433609A66270BD00BFB8040020A9
:109750002D4B032202FB003310B51C3393F901207B
:109760003F2A01DD3F225A70274B032202FB0033C0
:109770001C3393F9012012F13F0FBCBF6FF03E0282
:109780005A70214B032202FB00331C339A781F2AA4
:1097900001D91F229A701C4B032202FB00324FF4A6
:1097A00040211964127F012A04BF4FF450221A6429
:1097B000154B03EBC00292F827203AB9033202FBA3
:1097C0000032527F196C02F07F020BE0032101FB93
:1097D000003191F81DC002F003020CF07C0C196CF2
:1097E0004CEA0202084C41EA02221A64032303FBFA
:1097F0000040236C827F42EA030318462364FFF78C
:1098000087FF236CA36310BDB804002008B5044B88
:10981000032202FB00339977FFF79AFF08BD00BFD0
:10982000B804002008B5044B032202FB003359772B
:10983000FFF78EFF08BD00BFB804002008B5044B39
:10984000032202FB00331977FFF782FF08BD00BF38
:10985000B8040020264B052210B502FB00331A7D08
:10986000012A01D901221A75214B052202FB00337E
:1098700014335A78032A01D903225A701C4B05224B
:1098800002FB003314339A780F2A01D90F229A7001
:10989000174B052202FB00331433DA78032A01D96F
:1098A0000322DA70124B052202FB003314331A79BB
:1098B0000F2A01D90F221A710D4C052303FB00401A
:1098C00000F114021379017D43F42023507843EA18
:1098D000C133917843EA4033D27843EA012343EA23
:1098E000421318462364FFF713FF236C636310BD14
:1098F000B804002008B5044B052202FB003319769A
:10990000FFF7A8FF08BD00BFB804002008B5044B4E
:10991000052202FB0033D975FFF79CFF08BD00BF8D
:10992000B804002008B5044B052202FB00339975EA
:10993000FFF790FF08BD00BFB804002008B5044B36
:10994000052202FB00335975FFF784FF08BD00BFF5
:10995000B804002008B5044B052202FB003319753A
:10996000FFF778FF08BD00BFB8040020514B0B2261
:1099700010B502FB00331A7A032A01D903221A72A6
:109980004C4B0B2202FB003308339A78032A01D98F
:1099900003229A70474B0B2202FB003308331A79DB
:1099A0000F2A01D90F221A71424B0B2202FB0033FE
:1099B00008335A79072A01D907225A713D4B0B22E5
:1099C00002FB003308339A790F2A01D90F229A71CA
:1099D000384B0B2202FB003310335A780F2A01D97F
:1099E0000F225A70334B0B2202FB003310339A784C
:1099F0000F2A01D90F229A702E4B0B2202FB003244
:109A0000117AC90341F400241C64527A12B141F462
:109A100004211964274B0B2101FB0031C97A19B1CC
:109A2000196C41F400511964224B8AB90B3202FBC4
:109A30000032083292F804C091784FEACC1C1C6CBA
:109A40004CEAC12C51794CEA040242EA01121DE0B1
:109A50000B2202FB0032127C1AB11A6C42F48052C3
:109A60001A64144B0B2101FB0031103191F801E015
:109A70001A6C897842EACE1201F0070C42EA0C1205
:109A800011F0080F1A6402D042F400621A64094B04
:109A90000B2202FB00300830C27922B981791A6C9E
:109AA00041EA02021A64034C206CFFF731FE236C7A
:109AB000236310BDB804002008B5064B0B2202FB3F
:109AC00000330833DA791AB10022DA71FFF74EFF5A
:109AD00008BD00BFB804002008B5064B0B2202FBEE
:109AE00000330833DA791AB90132DA71FFF73EFF31
:109AF00008BD00BFB804002008B5044B0B2202FBD0
:109B000000339974FFF732FF08BD00BFB80400208E
:109B100008B5044B0B2202FB00335974FFF726FFF4
:109B200008BD00BFB804002008B5044B0B2202FB9F
:109B300000331974FFF71AFF08BD00BFB8040020F6
:109B400008B5044B0B2202FB00339973FFF70EFF9D
:109B500008BD00BFB804002008B5044B0B2202FB6F
:109B600000335973FFF702FF08BD00BFB80400209F
:109B700008B5044B0B2202FB00331973FFF7F6FE06
:109B800008BD00BFB804002008B5044B0B2202FB3F
:109B900000339972FFF7EAFE08BD00BFB804002049
:109BA00008B5044B0B2202FB0033D972FFF7DEFE2F
:109BB00008BD00BFB804002008B5044B0B2202FB0F
:109BC00000335972FFF7D2FE08BD00BFB804002071
:109BD00008B5044B0B2202FB00331972FFF7C6FED7
:109BE00008BD00BFB804002010B5254B4FF460221B
:109BF0001A6403EBC00292F8272012B14FF47022CE
:109C00001A641F4B03EBC00292F8211092F820C097
:109C10001C6C090341EA8C312143196492F822201B
:109C2000012A04BF41F480611964154B03EBC001A4
:109C300091F823C01A6C42EA0C221A6491F824109D
:109C4000012904BF42F080021A640D4B03EBC002ED
:109C500092F82520012A03D11A6C42F040021A64BE
:109C6000074C04EBC00090F82620236C43EA021353
:109C700018462364FFF74CFD236CE36310BD00BF5F
:109C8000B804002008B5044B03EBC00383F826108A
:109C9000FFF7AAFF08BD00BFB804002070B50F4B46
:109CA000064603EBC00393F82650032D02D0032190
:109CB000FFF7E8FF3046FFF797FF084B9C6A14F464
:109CC000002F1CBF6FEA04346FEA1434032D03D055
:109CD00030462946FFF7D6FF204670BDB804002065
:109CE00008B5044B03EBC00383F82510FFF77CFF96
:109CF00008BD00BFB804002008B5044B03EBC00347
:109D000083F82410FFF770FF08BD00BFB8040020DF
:109D100008B5044B03EBC00383F82310FFF764FF7F
:109D200008BD00BFB804002008B5044B03EBC00316
:109D300083F82210FFF758FF08BD00BFB8040020C9
:109D400008B5044B03EBC00383F82110FFF74CFF69
:109D500008BD00BFB804002008B5044B03EBC003E6
:109D600083F82010FFF740FF08BD00BFB8040020B3
:109D7000064B10B503EBC003044683F82710FFF72A
:109D800033FF2046FFF7E4FC10BD00BFB8040020FD
:109D900010B5144B00221A6403EBC002527912B1C1
:109DA0004FF400721A640F4B03EBC00292791AB1A0
:109DB0001A6C42F480721A640A4B03EBC003DA791E
:109DC0000F2A01D90F22DA71064C04EBC000C279C8
:109DD000236C42EA030318462364FFF799FC236CC3
:109DE000E36210BDB804002070B5084D9DF810E086
:109DF0009DF8146005EBC00426716270A37084F8AE
:109E000003E005F83010FFF7C3FF70BDB804002071
:109E100008B5034B03EBC0039971FFF7B9FF08BD09
:109E2000B804002008B5054B03EBC003597109B114
:109E30000422DA71FFF7ACFF08BD00BFB8040020B0
:109E400008B5054B042903EBC003D97101D00022EA
:109E50005A71FFF79DFF08BDB80400202DE9F047B7
:109E6000344D0446401990F844000E461746984673
:109E7000DDF82090DDF824A004281FD8DFE800F0EA
:109E800003090F151B002046FFF770FD651901231C
:109E900016E02046FFF7A8FE6519022310E02046D1
:109EA000FFF7D8FC651903230AE02046FFF750FCB2
:109EB0006519042304E02046FFF76AFF65190023B3
:109EC00085F844301B4B03EBC40494F82620012A88
:109ED0000DD002D3022A23D111E016B19B6A9B0C4C
:109EE0003370EFB1134B9B6A9B0A3B7018E0B8F1DB
:109EF000000F15D09B6A9B0AC8F8003010E0B8F13B
:109F0000000F04D09B6ADB0B5B01C8F80030B9F18D
:109F1000000F05D0074B9B6AC3F3842389F80030F8
:109F2000BAF1000F03D0034B9B6A8AF80030BDE8FA
:109F3000F08700BFB8040020214B10B50322002495
:109F40004FF0050C02214FF0010E83F825E0197344
:109F500083F80EC09A745C7483F81CE083F81DC00B
:109F600083F81EC083F8202083F8212083F8224044
:109F700083F8234083F8244083F8261083F8274091
:109F80001C755C759C75DC751C765C719C71DC7154
:109F900019725C72DC729C725A73DC731C742046FA
:109FA000FFF758FC2046FFF7D3FB2046FFF71CFEC7
:109FB0002046FFF7EDFE2046FFF7D8FC10BD00BF9E
:109FC000B804002008B5044A0023917A034A1846D1
:109FD0001370FAF72FFC08BDFC0B0020640C002066
:109FE0002DE9FF417F4B1A7822B901321A706FF0C8
:109FF00000425A607B4B1C7A5CB9E0B2FAF75EFA19
:10A00000784B03F10C0210550134082CF5D10122D4
:10A010001A7227240025E8B2FAF750FA724A535D03
:10A02000834219D0714B291D53F821305055022B12
:10A0300005D0032B0AD0012B0ED168B106E058B928
:10A040006B4A115D012907D1135505E0684B1A5D74
:10A05000012A01D101321A5501350134082DDAD116
:10A06000644EF36993B1644C25787DB9FEF7F8FD31
:10A07000624AF3691268821A002AB8BF52429A42B1
:10A0800004D9284601F038FA01232370594E336A67
:10A0900093B15B4C25787DB9FEF7E2FD594A336AEE
:10A0A0001268821A002AB8BF52429A4204D928463E
:10A0B00001F022FA012323704A4D534C2A7D93006C
:10A0C00004EBC3010E7B002E00F028814F48504F57
:10A0D000504E0021C318BF18B61810460A46009704
:10A0E0000196FFF7BBFE2B7D04EB4314227B013A64
:10A0F000042A00F20281DFE812F005004E00D300CE
:10A100004E00D300444A374D926812F0200F1BD006
:10A110005D192A7E022A04D1404AD25C002A00F04E
:10A12000EC80394A2F4C02EB43121846517AFAF769
:10A1300081FB207DFFF7C0FC237D384A0021E41815
:10A14000D15402232376D8E05D192A7E012A04D156
:10A15000324AD25C002A00F0D0802B4C184604EB27
:10A160004313997AFAF766FB1E4B187D04EB4014F3
:10A17000A37A13B9FFF7B0FC04E0284B1B5C0BB1CA
:10A18000FFF79AFC174A2549137D0020D218C854BE
:10A1900001231376B1E01F4A124DD256002A3FDB4D
:10A1A0005D192A7E022A02D11C4AD25C8AB1164A63
:10A1B0000C4C02EB43121846517AFAF73BFB207D18
:10A1C000FFF77AFC237D154A0021E418D1540223BD
:10A1D0002376044C257DFEF743FD04EB8504606087
:10A1E00056E000BF000500200C050020240C0020D4
:10A1F000740C002008000020610C00205C0C002082
:10A20000790B0020540C0020FC0B0020A00B002038
:10A21000840B0020F40B0020000C0140600C002097
:10A220005B191B7E012B11D0FEF71AFD2B7D894A8D
:10A2300005EB830502EB43139B8B0A2253436A68A9
:10A24000821A002AB8BF52429A4204DC824B834AE7
:10A250001B7DD35CE3B1804D7E4C287D04EB401325
:10A26000997AFAF7E7FA287D04EB4014A37A13B938
:10A27000FFF732FC04E0794B1B5C0BB1FFF71CFCD1
:10A28000754A7649137D0020D218C85401231376ED
:10A29000714B1A7D6F4B03EB42131B7B042B20E0A9
:10A2A0006D4A9A18127E022A02D16C4AD25C8AB197
:10A2B000684A694C02EB43121846517AFAF7BAFA27
:10A2C000207DFFF7F9FB237D644A0021E418D15477
:10A2D00002232376604B1A7D5E4B03EB42131B7BFC
:10A2E000052B0AD15E4B9A6812F0200F15BF4FF470
:10A2F00080624FF480625A611A61FEF7B1FC564CDD
:10A30000E369C31A002BB8BF5B420A2B40F31A83E0
:10A31000FAF77CF9FEF7A4FCE06113E3FAF776F9AB
:10A32000FEF79EFCEB69C31A002BB8BF5B420A2BF9
:10A3300040F30883297D3046490141F00A0101F0CC
:10A34000EA0100F09BFF0446287D01F0F9F82B7D1F
:10A350000C20584343494218157A0DB1455800E086
:10A360005568414AD25C032A00F2E480DFE802F03B
:10A3700002801C4B002C00F0DD80364A364D02EB8B
:10A380004311C97F384E29B11846FAF753FA2B7D8D
:10A39000032207E002EB43121846517AFAF74AFA11
:10A3A0002B7D0222F254C5E04CB95B0143F0080159
:10A3B00001F0E801204600F061FF002862D0264E3F
:10A3C000244B307D03EB4013D97F002900F0AB8094
:10A3D000002D84EAE472B8BF6D42A2EBE472AA4297
:10A3E00002D0002C40F09980204B53F830108A4264
:10A3F00080F0998003EBC0031979FAF71BFA164B2A
:10A4000001211B7D8DE0002D84EAE471B8BF6D420F
:10A41000A1EBE471A94202D0002C40F08480134AE1
:10A420000D4D52F83300104E814208D202EBC302A8
:10A4300018461179FAF7FEF92B7D012208E0054A4A
:10A44000184602EB4313597AFAF7F4F92B7D0222EE
:10A45000F25468E0FC0B002000050020600C002096
:10A46000000C0140A80B0020640C0020880B002089
:10A4700044BB5B0143F0080101F0E801204600F015
:10A48000FDFEF8B9FEF7ECFB1F4D204A2B7D4FF087
:10A490000A0E02EB4311B1F81CC099004E19766800
:10A4A0000EFB0CFC861B002EB8BF7642664541DDD4
:10A4B00002EBC1021846917AFAF7BCF92B7D144AD7
:10A4C000D45437E0104E114A337D02EB4312D17F52
:10A4D00049B3002D84EAE472B8BF6D42A2EBE47286
:10A4E000AA4200D0C4B90B4951F833108A421AD39A
:10A4F000064A184602EB4313597AFAF79BF9024BC6
:10A5000002211B7D0DE000BF00050020FC0B002098
:10A51000640C0020880B00201846FAF78BF9337D75
:10A520000321A34AD154A34D2E7DFEF799FB05EBE1
:10A53000860568609F4DA04F2B7DA04E1846F618EB
:10A54000FF189F4B002103EB80030A4601960097FA
:10A550009C4EFFF783FC287D06EB40139B6943B3B9
:10A56000F9F736FF28B3287D84EAE47206EB40133E
:10A570009B69A2EBE4729A421BD900F0BDFF2A7DD1
:10A58000914906EB42139B7F0120885443B1B27F6F
:10A590009A4205D1013800F0AFFF002000F0EAF93F
:10A5A000844B8A4A1B7D0F33D15C012901D10131D3
:10A5B000D154804D2B7D022B25D8002000F03AFD90
:10A5C00095F8203010F0010F03F0F80385F82030E3
:10A5D0001CBF43F0010385F8203010F0040F8DF804
:10A5E0000C0006D0734B93F8202042F0020283F84F
:10A5F000202010F0100F06D06E4B93F8202042F070
:10A60000040283F82020724A137853B1694991F803
:10A6100020100B4205D16F496F480978037001B9CA
:10A6200011706D4B1B784BB1624A92F8202003EAFF
:10A6300002029A4202D1694B01221A705D4B93F8D3
:10A64000202012F0010F0AD093F8213013F0010FEF
:10A6500005D15E4BDA78012A01D10132DA70554B0F
:10A6600093F8202012F0020F0AD093F8213013F053
:10A67000020F05D1554B1A79012A01D101321A7105
:10A680004C4B93F8202012F0040F0AD093F821309D
:10A6900013F0040F05D14D4B5A79012A01D1013233
:10A6A0005A71444D03222B7D04A8B3FBF2F28218A9
:10A6B00012F9042C95F82010002A85F821104ADAA6
:10A6C0005B0143F01601002001F0F60102AA00F040
:10A6D000EDFD9DF80A3013F0400F08D02A7D3B496C
:10A6E00052001B32885C012801D10130885413F0DC
:10A6F000800F0AD02F49354A097D0E3112F811001A
:10A70000012802D1013002F8110013F0100F09D016
:10A71000284A2E49127D52001B32885C012801D143
:10A720000130885413F0200F0AD0224A274B127DA3
:10A730000E3213F81210012902D1013103F8121060
:10A740001C4B0020197D02AA490141F0160101F0BD
:10A75000F60100F047FF174F1A4E3B7D06EB431200
:10A760005269002A00F082801D4AD55C002D7DD1FF
:10A77000002C7CD05B0143F0020101F0E20128468D
:10A7800000F042FD8046387DFAF738F8397DC0EB9D
:10A79000080806EB41135B69B8F1000F83EAE37226
:10A7A000B8BFC8F10008A2EBE372904568DD19E07C
:10A7B000640C002000050020840B0020F40B002016
:10A7C000A00B0020FC0B0020F00B0020740C0020DC
:10A7D0009C0B0020800B0020950B0020A30C002078
:10A7E000940B0020002B0EDD084600F085FE3B7D1B
:10A7F00006EB43139B7F3BB3B27F9A4224D128469A
:10A8000000F07AFE1DE02846022200F0D7FC397DD8
:10A810002846490141F0080101F0E80100F04EFE30
:10A820003B7D06EB43139B7F73B1B27F9A420BD102
:10A8300029462846022200F0C1FC2846082100F0E3
:10A840003DFE284600F096F83F4B404A1B7D1533ED
:10A85000D15C012901D10131D1543B4B3C4A1B7DD4
:10A8600001211846D15400F085F809E044B95B0194
:10A8700043F0080101F0E801002000F0FFFC20B1E6
:10A88000314D344B2E7D9B5D43B32F4B324A1B7DA4
:10A8900002EB4312D28912B92E4AD35C1BB3FEF7E6
:10A8A000DFF9294D2C492B7D4FF00A0C9A0001EB62
:10A8B000C201C9895219526A0CFB01F1821A002A9D
:10A8C000B8BF52428A420EDD244EF25C5AB9184695
:10A8D000FFF702F92B7D0122F25404E0FEF7C0F9E4
:10A8E00005EB86056862184E1D4D307D002C55F82D
:10A8F0003030B8BF64429C420AD2FEF787FE337DF7
:10A9000005EBC3056A7982420DD11846002108E0A3
:10A91000FEF77CFE337D05EBC3056979884202D0E2
:10A920001846FEF7E7FF084C207D00F031F8237D44
:10A930000133DBB223750BB100232375FEF790F9C9
:10A94000014BD861BDE8FF8100050020740C002098
:10A95000940B00206C0C0020FC0B0020700C0020DD
:10A96000880B0020024B1A5C0AB901321A54704756
:10A9700028050020024B1A5C0AB10F221A547047B6
:10A9800028050020014B185C704700BF28050020F7
:10A990002DE9F3474601F5B2044645F07C0100205D
:10A9A00001AA00F083FCB74A610002EB4413187A55
:10A9B00006EB020710F0400F9DF8063012D04FF062
:10A9C00001084FF0020C08FA01F80CFA01FCB1582A
:10A9D0007E680CEA030208EA0307C1F10009C6F128
:10A9E000000A0FE04FF0010C4FF002080CFA01FCD6
:10A9F00008FA01F156F80290D7F804A00CEA030215
:10AA000001EA030710F0800F00F03F0606D09E4BCE
:10AA10009B6883F02008C8F3401803E09A4B9B68BA
:10AA2000C3F34018731E072B00F2D182DFE813F046
:10AA300008000800080008006E016E016E016E013A
:10AA4000924B1B5D013B0E2B00F2C182DFE813F03D
:10AA50000F003D00530062007A0082008E00A000CB
:10AA6000D10014012401BF0243014E01A60201AA34
:10AA700045F014010020854F00F018FC9DF80530CA
:10AA800045F0060507EB8408C8F804302946002085
:10AA900000F0F4FB0222C8F808002146002000F074
:10AAA0008DFB023E0020294640F2FF7200F0F2FCCE
:10AAB000F6B200200322214600F05AFB012E01D8F5
:10AAC000022300E004233B5581E2704E002006EB98
:10AAD00084035A68214602F00402824214BF052210
:10AAE000012200F045FB45F008014A46002000F035
:10AAF000D1FC032324E0002A00F0698245F0020122
:10AB0000002000F081FB614B04221A55604B43F892
:10AB100024005CE25D4E002006EB84035A68214667
:10AB200002F00402824214BF0622022200F020FB3F
:10AB300045F00801C9F10002002000F0ABFC05233C
:10AB4000335544E2002F00F04282204600F0D4FC4E
:10AB500006222FE200202146032200F009FB45F0E7
:10AB600008015246002000F095FC68E1002F40F0FB
:10AB70002E8245F008053A463846294600F08AFC00
:10AB8000CAF100023846294600F084FC082211E28E
:10AB9000002F00F01C8245F00201002000F034FB81
:10ABA00006460020024645F0080100F073FC384BD1
:10ABB000002053F824702146BF1B43F82470032261
:10ABC00000F0D6FA8AEAEA7245F00601A2EBEA72D0
:10ABD000002000F05FFC610101F0E001324600203E
:10ABE00000F0C4FB00200246214600F0E7FA0922EB
:10ABF000E0E1002000F01EFA630050FA03F313F0C6
:10AC0000010F00F0E48145F002073946002000F012
:10AC1000FBFA204B45F0080543F8240000200246CB
:10AC2000294600F037FC00200222214600F0C6FA37
:10AC300000200246394600F099FB002061010246DF
:10AC400001F0E001033E00F091FBF6B20021204646
:10AC5000F9F7AAFD012E0D4E0CD800202146022244
:10AC600000F0ACFA2946CAF10002002000F012FC04
:10AC70000A2365E70E2363E7002F00F0A8810B226B
:10AC800098E100BFFC0B0020000C014028050020CB
:10AC90007C0B0020200C0020002F40F0988145F014
:10ACA0000201384600F0B0FA45F0080106463A467F
:10ACB000384600F0EFFB6101022296FBF2F201F050
:10ACC000E001384600F052FB3A463846214600F093
:10ACD00075FA0D226EE1002000F0ACF9630050FA25
:10ACE00003F313F0010F00F0728162E1A84E45F00A
:10ACF000060106EB84050020AA6800F0CBFB2A7948
:10AD00000020214600F034FA002319E7A04B1B5D18
:10AD1000013B0E2B00F25B81DFE813F00F003400E3
:10AD20005200620081005901930059015901CC0081
:10AD3000DC00AD0008014F01400145F0140101AAFB
:10AD40000020934F00F0B2FA9DF805C007EB840392
:10AD500000200222C3F804C0214600F02FFA002090
:10AD600045F0060140F2FF7200F094FB0020032240
:10AD7000214600F0FDF9062E02D0082E7FF4A2AE87
:10AD8000022217E1062E0CD1814B002003EB840335
:10AD90005A68214602F00402824214BF05220122B1
:10ADA00004E0082E04D100202146032200F0E0F93F
:10ADB0004A4645F00801002000F06CFB0322F9E050
:10ADC000731FDBB2012B05D822B1062E704E30D195
:10ADD0000423B5E6B8F1000F00F0F9800C22E9E099
:10ADE000052E0CD16A4B002003EB84035A682146E0
:10ADF00002F00402824214BF0622022204E0072E5F
:10AE000004D100202146032200F0B2F9C9F100026A
:10AE100045F00801002000F03DFB0522CAE0731F49
:10AE2000DBB2012B07D837B1052E594E01D10223D1
:10AE300086E60F2384E6B8F1000F00F0C8800722F1
:10AE4000B8E0B8F1000F40F0C280073EF6B2012E24
:10AE50000DD94F4B404603EB84035A68214602F05C
:10AE60000402002A14BF0522012200F081F945F0F6
:10AE70000801524619E0B8F1000F40F0A880073EE3
:10AE8000F6B2012E0DD9424B404603EB84035A68BB
:10AE9000214602F00402002A14BF0622022200F01A
:10AEA00067F945F00801CAF10002002000F0F2FA4B
:10AEB0000A227FE0B8F1000F00F0898045F002011E
:10AEC000002000F0A1F9324B0B2103EB840219554D
:10AED000D0607CE0B8F1000F79D145F00201404626
:10AEE00000F092F92B4BA700294E03EBC7038AEA27
:10AEF000EA72814645F00601A2EBEA72404683F809
:10AF00000D80BF1900F032FAFB68610199440223F9
:10AF100099FBF3F201F0E001404600F027FA4046C9
:10AF20002146424600F04AF90D2309E6002000F0D0
:10AF300081F8630050FA03F313F0010F47D0144B6C
:10AF40000E2245F002061A553146002000F05CF949
:10AF5000114B45F0080143F824000020024600F0A0
:10AF600099FA21460020022200F028F900203146FB
:10AF7000024600F0FBF900206101024601F0E00109
:10AF800000F0F4F920460021F9F70EFC1FE000BFA5
:10AF900028050020FC0B0020200C0020002021466A
:10AFA000022200F00BF9002045F00801024600F0F3
:10AFB00071FA0E22074B1A5509E0064D002005EBE9
:10AFC00084031A79214600F0D3F800232B55BDE8FD
:10AFD000FC8700BF28050020154B10B503EB0012BD
:10AFE000926891420EDD8A1AC2F18074A2424FEA41
:10AFF000001C03DC63445C6812190EE063445A6869
:10B00000141B0FE00FDA521AC2F18074A2424FEA09
:10B01000001C04DC63445C68A21A5A6003E06344C9
:10B020005A68A4185C60024B03EB0010816010BDED
:10B03000740D0020012108B502200A46F9F7A0FC92
:10B0400008BD00BFF8B51378144613F0600F06462C
:10B050000D4627D1414A127B22BB13F0010F21D1AB
:10B060005F2B1FD83E4A1278E2B913F09F0301D03C
:10B07000082B17D13B4F387860B9384BD97F19B1BD
:10B08000F9F7D8FB032304E00846597AF9F7D2FB15
:10B0900002233B70344F3B7823B10020FEF70CFDB8
:10B0A00000233B70002221780220F9F769FC287008
:10B0B000002261780220F9F763FC68700022A17811
:10B0C0000220F9F75DFCA87001220220E178F9F76F
:10B0D00057FCE870237813F0010F3ED15F2B3CD86A
:10B0E00003F01E02082A04D0142A2CD0062A34D1D8
:10B0F0001BE0242171435B090C2000FB0313A5789E
:10B1000094F803C0194A4CEA05259D50A37813F022
:10B11000080F22D02678760900FB0616B3586FEA8E
:10B1200003536FEA1353B35017E0242256435B09CD
:10B130000C22A17802FB0363E27842EA01220B4968
:10B140005B185A6009E0242256435B090C2202FB7B
:10B1500003630649E2785B181A72F8BDFC0B002005
:10B160006C0C0020640C0020700C0020A80B002048
:10B170002DE9F3414901CEB201AC46F01503174663
:10B18000694622468DF804308046FFF75BFF9DF844
:10B1900001C09DF8033046F0140640466946224639
:10B1A0006D468DF804608DF805C08DF806708DF839
:10B1B0000730FFF747FFBDE8FC8100BF2DE9F341F1
:10B1C0004901CEB201AC46F0150317466946224646
:10B1D0008DF804308046FFF735FF9DF801C09DF8DB
:10B1E000023046F014064046694622466D468DF808
:10B1F00004608DF805C08DF806308DF80770FFF7F4
:10B2000021FFBDE8FC8100BF37B541F001030C46CA
:10B210006A4601A98DF800300546FFF713FF9DF837
:10B2200006009DF8052000029DF8073040EA024024
:10B23000184310F4000F18BF40F07F405F2C1AD85D
:10B24000C4F3411314F01E0402D0022C13D106E003
:10B25000032202FB0535084A2D01A8580BE0032202
:10B2600002FB053520F07F41E8B2FFF7B5FE024B47
:10B2700003EB051568683EBD740D002007B541F06D
:10B2800001036A4601A98DF80030FFF7DBFE9DF847
:10B2900006009DF8073043EA002010F4006F1CBF41
:10B2A0006FEA00506FEA10500EBD00BF13B541F0B9
:10B2B0000103144601A96A468DF80030FFF7C2FE6B
:10B2C0009DF805109DF806309DF807202170A270AA
:10B2D00063709DF804001CBD07B5410141F01601E3
:10B2E00001F0F601002001AAFFF7E0FF9DF805300C
:10B2F000D80913F0200F18BF40F002000EBD00BFA8
:10B3000007B5410141F0160101F0F601002001AA44
:10B31000FFF7CCFF9DF80530C3F3801013F0100F3A
:10B3200018BF40F002000EBD37B50C4641EA40118F
:10B3300001AA0546C9B20020FFF7B8FFB4235D4358
:10B340006408032305F5807503FB04549DF804107D
:10B350002046FCF7A3FF601C9DF80510FCF79EFF3C
:10B36000A01C9DF80610FCF799FF3EBD5F292DE952
:10B37000F3410D460646144662D8C1F3411811F058
:10B380001E0102D002295BD11EE0032202FB0088CD
:10B39000344A4FEA081083185B688450E01A00288A
:10B3A000B8BF4042B0F5000F0ADB9C42CCBF2E4C28
:10B3B0002E4C2C4A1C1902EB0812012313733FE098
:10B3C00002EB081211733BE0032707FB0087254BB4
:10B3D0003801C1587A00C4EB010C0132BCF1000FF6
:10B3E000B8BFCCF1000C00EB030EBCF5000F24F04D
:10B3F0007F40CEF8044043F832001DDBA142CCBFB1
:10B40000194B1A4B4FEA4818E3184FEA234E4FEAFC
:10B41000232C3046694601AA8DF807308DF8048048
:10B420008DF805E08DF806C0FFF70CFE0D4B03EB21
:10B43000071701233B7303E003EBC20300221A71D9
:10B440004FEA244C23123046694601AA8DF8045075
:10B450008DF805C08DF806308DF80740FFF7F2FD36
:10B46000BDE8FC81740D0020FFFF7F00010080FF1C
:10B4700038B50D4668210446FFF7C6FE15B140F009
:10B48000010201E020F0010220466821FFF76EFF73
:10B4900038BD00BF07B513464FEA222C8DF80410C3
:10B4A0004FF0000E694601AA8DF805E08DF806C040
:10B4B0008DF80730FFF7C6FD0EBD00BF07B50B4680
:10B4C00011F01E01024601D0022905D1104619468D
:10B4D0000022FFF74BFF0DE04FF0000C694601AA78
:10B4E0008DF804308DF807C08DF805C08DF806C0C2
:10B4F000FFF7A8FD0EBD00BF10B5C4B22146640120
:10B5000000200222E4B2FFF759FE002044F00801B7
:10B51000FFF7D4FF44F00A010020FFF7CFFF10BD72
:10B5200007B59DF810C08DF804108DF80520694608
:10B5300001AA8DF806308DF807C0FFF783FD0EBD18
:10B5400030B5430185B0044643F00303002003A94E
:10B5500002AA8DF80830FFF775FD9DF80E109DF8D2
:10B560000D209DF80F30090241EA0241194320469F
:10B57000FFF732FD174B03EB041108310A7932B3A0
:10B58000154A0C2000FB0422107A00BB2201D518BA
:10B59000D2586B68C3EB020CBCF1000FB8BFCCF102
:10B5A000000CBCF5000F05DB9A42CCBF0B4A0C4ADD
:10B5B0009A1800E008716101C2F30723D4B201F0C8
:10B5C000E0010020C2F307420094FFF7A9FF05B095
:10B5D00030BD00BF740D0020A80B0020FFFF7F00CE
:10B5E000010080FF07B5937892F800E092F801C05F
:10B5F0008DF8041001AA69468DF805E08DF806C0A3
:10B600008DF80730FFF71EFD0EBD00BF37B54401B2
:10B6100044F01604E4B20D4601AA21460020FFF7CB
:10B6200045FE9DF8053015F0010F1ABF6FEA436320
:10B630006FEA536303F07F038DF805309DF8053002
:10B6400015F0020F14BF43F0200323F020038DF800
:10B65000053000231846214601AA8DF80630FFF771
:10B66000C1FF3EBD37B5440144F01604E4B20D46B7
:10B6700001AA21460020FFF719FE9DF8053015F0BC
:10B68000010F14BF43F0400323F040038DF8053051
:10B690009DF8053015F0020F14BF43F0100323F09E
:10B6A00010038DF8053000231846214601AA8DF8B5
:10B6B0000630FFF797FF3EBD73B5B42545434B08F1
:10B6C000032205F5807502FB0355044628460E4605
:10B6D000FCF74EFD8DF80400681CFCF749FD8DF861
:10B6E0000500A81CFCF744FD46EA44148DF806004A
:10B6F000E1B2002001AAFFF775FF7CBD2DE9F74FED
:10B700004001C7B24C05002047F0180101AAFFF71D
:10B71000CDFD9DF80560640D06F00F053609B542B4
:10B720000EDB204604F078FEAD1B80460120A840C9
:10B73000894604F081FE0022334B04F0E3FE0FE063
:10B74000204604F069FE751B80460120A84089460A
:10B7500004F072FE02460B4600202B4904F0FCFF69
:10B7600002460B464046494604F0F6FF05F08CF9C8
:10B7700004F074FE22A3D3E9002304F0C3FE05F015
:10B7800083F904F06BFE0022204B04F0BBFE4FF067
:10B79000FF36B046002582468B460120A84004F0C3
:10B7A0004BFE02460B465046594604F0ABFE05F0F0
:10B7B00043F9A0F180027F2A98BF2E46034605F187
:10B7C000010588BF43460E2D01D09846E5E70025C8
:10B7D00047F0120101AA28468DF805308DF8066061
:10B7E0008DF80450FFF7FEFE284647F00C01224674
:10B7F000FFF750FE2846BDE8FE8F00BFAFF3008084
:10B8000004560E2DB29DEF3F000060400000204026
:10B8100013B5154B587E10F0010003D000206821AD
:10B82000212201E0682120220024FFF79FFD20460D
:10B830007E21202223460094FFF772FEE1B2002011
:10B840000134FFF739FF1D2CF8D10C210020FFF740
:10B85000DBFC01460020FFF751FF0020162143F2D8
:10B86000FF12FFF717FE1CBD08000020AFF3008099
:10B87000084B1868034605E02C2A02D100221A70F2
:10B8800003E001331A78002AF6D1024A013313602B
:10B89000704700BF3805002010B50E4B02461B78DC
:10B8A000ABB10D4B1C7994B19C68601CE4180D2A57
:10B8B0002273986002D03F2800D851B9064C014647
:10B8C00004F10C00FDF73EFC0023A36001E0FCF74F
:10B8D00029FF10BD780B00203805002030B501216C
:10B8E000044687B02020FFF7D7FF002C04DA2D2074
:10B8F0000121FFF7D1FF644200230A2194FBF1F2FA
:10B9000001FB124101AD3031E954591C141E01DD17
:10B910000B46F2E7ED181C460121013C15F8010920
:10B92000FFF7BAFFB4F1FF3FF6D107B030BD00BF5B
:10B9300038B50C4D0446A87801214030C0B2FFF75D
:10B94000ABFF687801214030C0B2FFF7A5FF207837
:10B95000FFF7C4FF6068FFF7C1FF0D200121FFF76B
:10B960009BFF38BD0800002070B5124B06461B78BF
:10B97000EBB1FCF755FE104C054618B100232371BE
:10B98000012016E0E36C226D934208D21A1992F856
:10B990005420013301203270E364207109E004F186
:10B9A0005400FDF79DFBE5642065284601E0FCF7A7
:10B9B00037FE70BD780B0020380500202DE9F341DB
:10B9C00004460DF10700FFF7CFFF002800F0CB8001
:10B9D0008B4B8C4A93F8941019BB51789DF8070053
:10B9E000403188420DD1D3F89810002940F0BB8037
:10B9F0001179012231F0010183F8942040F0B380E5
:10BA0000AFE00D2801D01B2802D100227C4B05E0BD
:10BA1000D3F898207E2A00F2A6800132C3F898203D
:10BA2000A1E0117931F0010103D19DF80700FFF782
:10BA300033FF9DF807301F2B0BD9714AD2F89810AD
:10BA40007E297FD8481C891881F89C30C2F898005C
:10BA500078E0082B08D16A4BD3F89820002A71D0DF
:10BA6000013AC3F898206DE00D2B6BD1644BD3F8ED
:10BA70009830002B66D0634B1A79112A15D158786B
:10BA800001214030C0B2FFF707FF002503E0585DF9
:10BA9000FFF702FF01355A4B0121D3F898209C3360
:10BAA0009542F4D30D20FFF7F7FE554A00231568A1
:10BAB000D2F8987019461A4633E001290FD002D304
:10BAC00002292DD122E04E4E06F19C00805C2028F8
:10BAD00026D09E1986F81C010133012120E0484838
:10BAE00000F19C0C1CF802C0BCF1200F0AD1012B04
:10BAF00004D91818002180F81C110133424D02218D
:10BB0000ED180DE0181880F81CC108E03C4E06F155
:10BB10009C00805C202803D09E1986F81C0101330C
:10BB20000132BA42C9D3364A0021981880F81C1154
:10BB30000120C2F89810156082F8A001C2F89C316B
:10BB400082F894109DF807301B2B0CD12D4A2C4BFA
:10BB500012790021012A83F89410C3F8981002D1B9
:10BB60000D20FFF799FE264B93F8A001002878D00E
:10BB70000022164683F8A0211546DFF8A880072783
:10BB800007FB058720483946013503F023FE30B90D
:10BB9000BE797B7916F0010F237049D007E018F8C1
:10BBA00006300736002B5ED0FF2DE6D15BE0FFF7B5
:10BBB0005FFE23780546042B0CD1144903F00AFEDE
:10BBC0000346D8B12846124903F004FE70B1284656
:10BBD00010490FE00D2B28D10F4903F0FBFD034660
:10BBE00060B128460D4903F0F5FD08B9012305E0D1
:10BBF0000B49284603F0EEFDB0B90223637017E04D
:10BC0000380500200800002054060020091B010808
:10BC10000D1B0108111B0108171B01081D1B010842
:10BC2000221B010808190108284603F0CDFD6070A9
:10BC300016F0020F04D0FFF71BFE03F0C5FDA07045
:10BC400016F0040F0CD0FFF713FE03F0BDFD010E3C
:10BC5000C0F30722C0F30743A17122716371E07042
:10BC60000120BDE8FC8100232370F9E7704700BF85
:10BC7000FEE700BFFEE700BFFEE700BFFEE700BF34
:10BC8000704700BF704700BF704700BF704700BFDC
:10BC9000704700BF704700BF704700BF704700BFCC
:10BCA000704700BF704700BF704700BF704700BFBC
:10BCB000704700BF704700BF704700BF704700BFAC
:10BCC000704700BF704700BF704700BF704700BF9C
:10BCD000704700BF704700BF08B5024B1B6898470C
:10BCE00008BD00BF980B002008B5024B1B689847A1
:10BCF00008BD00BF680C002008B5024B1B689847C0
:10BD000008BD00BFF80B002008B5024B1B68984720
:10BD100008BD00BF1C0C0020704700BF704700BF6B
:10BD2000704700BF704700BF704700BF704700BF3B
:10BD3000704700BF704700BF704700BF704700BF2B
:10BD4000704700BF704700BF704700BF704700BF1B
:10BD5000704700BF704700BF704700BF704700BF0B
:10BD6000704700BF704700BF704700BF704700BFFB
:10BD7000704700BF704700BF704700BF704700BFEB
:10BD8000704700BF704700BF704700BF704700BFDB
:10BD9000704700BF704700BF704700BF704700BFCB
:10BDA000704700BF704700BF704700BF436830B5A1
:10BDB00023F470230C680A7923F48073234343EA45
:10BDC0000223436082688D68CC680A4B45EA040C04
:10BDD00002EA03034A794CEA030343EA420383601D
:10BDE0000B7CC26A013B22F47002DBB242EA0353CD
:10BDF000C36230BDFDF7F1FF002301220274C3606E
:10BE00000360037143718360704700BF19B1836899
:10BE100043F0010302E0836823F00103836070476D
:10BE200019B1836843F4807302E0836823F480735C
:10BE300083607047C9B212B14368194302E0436896
:10BE400023EA010141607047836843F0080383607F
:10BE5000704700BF8068C0F3C0007047836843F03C
:10BE600004038360704700BF8068C0F380007047A0
:10BE700019B1836843F4A00302E0836823F4A003AC
:10BE8000836070478068C0F3805070474368013911
:10BE900023F4604343EA41334360704719B1436878
:10BEA00043F4006302E0436823F400634360704797
:10BEB000092930B511D94FF0030C0CFB01FC072503
:10BEC000ACF11E0C05FA0CF503FA0CFCC46824EA6C
:10BED000050343EA0C03C3600EE04FF0030C0CFBB8
:10BEE00001FC072505FA0CF503FA0CFC046924EAA9
:10BEF000050343EA0C030361062A0DD80523013A22
:10BF00005A434FF01F0C0CFA02FC9140436B23EA9A
:10BF10000C020A4342631CE00C2A0DD805235A4345
:10BF20004FF01F0C233A0CFA02FC9140036B23EAFA
:10BF30000C020A4302630CE005235A434FF01F0C26
:10BF4000413A0CFA02FC9140C36A23EA0C020A430C
:10BF5000C26230BD19B1836843F4801302E0836884
:10BF600023F4801383607047C06C80B2704700BFB9
:10BF7000014B1868704700BF4C24014019B1436859
:10BF800043F4806302E0436823F4806343607047B6
:10BF900019B1436843F4805302E0436823F48053AB
:10BFA00043607047836823F4E04341EA03038360FE
:10BFB000704700BF19B1836843F4004302E083680F
:10BFC00023F400438360704719B1836843F402137C
:10BFD00002E0836823F40213836070478068C0F333
:10BFE00040507047092930B511D94FF0030C0CFBB4
:10BFF00001FC0725ACF11E0C05FA0CF503FA0CFC4C
:10C00000C46824EA050343EA0C03C3600EE04FF062
:10C01000030C0CFB01FC072505FA0CF503FA0CFCDC
:10C02000046924EA050343EA0C030361836BC3F349
:10C03000015CCCEB020202324FF0050CD2B20CFBD9
:10C0400002F20CF11A0C0CFA02FC914023EA0C03E8
:10C050000B43836330BD00BF836B013923F440136E
:10C0600043EA0153836370470A50704728304058B1
:10C0700080B27047436823F4400323F4007341EA1D
:10C0800003034360704700BF41628262704700BF94
:10C09000436823F01F0341EA03034360704700BF76
:10C0A00020B1054B9A6842F4000203E0024B9A6803
:10C0B00022F400029A60704700240140036819428C
:10C0C0000CBF002001207047C9430160704700BFCA
:10C0D0004368006810EA112004D0C9B219420CBFAD
:10C0E00000200120704700BF6FEA112101607047F6
:10C0F00008B5134B98420FD003F5A053984213D0C4
:10C10000A3F5C053984219D14FF40070012100F0FB
:10C11000F3FF4FF400700EE04FF48060012100F057
:10C12000EBFF4FF4806006E04FF40040012100F087
:10C13000E3FF4FF40040002100F0DEFF08BD00BF28
:10C14000002801400268002322F00102026003601F
:10C1500043608360C3602D4B984233D011D83C3B81
:10C16000984229D006D8283B984221D014339842CF
:10C170004BD11FE0264B984220D01433984244D133
:10C180001EE0244B98422CD008D8A3F56773984240
:10C190001DD003F56273984237D11DE01E4B9842C3
:10C1A00029D0143398422BD0283B98422DD11DE042
:10C1B0001A4B12E0194B15E0184B18E0174B1BE017
:10C1C000164B1EE0154B5A6842F470021CE0134BEC
:10C1D0005A6842F0706217E0114B5A6842F00F0241
:10C1E00012E00F4B5A6842F0F0020DE00C4B5A6817
:10C1F00042F4706208E00A4B5A6842F4704203E06D
:10C20000074B5A6842F470225A6070476C00024033
:10C21000440002401C04024044040240000002406A
:10C22000000402408A6870B50C6A0B6944EA020295
:10C230004C691A438B692243CC6905684E6A42EA0D
:10C24000030323438C6A334325F4FE4C23432CF031
:10C25000F00C43EA0C030360CB6843600B68836017
:10C260004B68C36070BD00BF0023836203604360FE
:10C270008360C360036143618361C361036243629E
:10C28000704700BF19B1036843F0010302E003687F
:10C2900023F001030360704712B10368194302E001
:10C2A000036823EA01010160704700BF406880B263
:10C2B000704700BF10F0805F14BF044B044B1B6835
:10C2C00003420CBF00200120704700BF0004024061
:10C2D0000000024010F0805F14BF024B024B586018
:10C2E000704700BF000402400000024010F0805F71
:10C2F00014BF044B044B1B6803420CBF00200120F9
:10C30000704700BF000402400000024010F0805F50
:10C3100014BF024B024B5860704700BF000402403C
:10C3200000000240044B00221A605A609A60DA60F2
:10C33000024A5A61704700BF00040140FFFF070036
:10C34000837930B5016802794BB3184BCC431D6833
:10C3500090F805C004EA05051D605D682C405C602E
:10C36000D45844EA0101D15002689868D14301EAE7
:10C3700000009860D8680140BCF1100FD96007D167
:10C38000996811439960D96841EA0202DA600BE0CA
:10C390005CF8031041EA02024CF8032004E0034B6E
:10C3A000D05820EA0101D15030BD00BF0004014047
:10C3B00000230C228371427103600371704700BF38
:10C3C000024B1A6940EA02021A61704700040140F8
:10C3D000034B5B6918420CBF00200120704700BF6F
:10C3E00000040140014B5861704700BF0004014048
:10C3F000054B1A685B69034001D1184603E01042FF
:10C400000CBF00200120704700040140014B58611F
:10C41000704700BF00040140044B1A6802F0380264
:10C420001A601A6840EA02021A607047002002404F
:10C43000044B1A6822F008021A601A6840EA0202E5
:10C440001A60704700200240044B1A6822F0100264
:10C450001A601A6840EA02021A607047002002401F
:10C46000034B044A5A6002F188325A60704700BF99
:10C470000020024023016745024B1A6942F0800206
:10C480001A61704700200240014BD869800870474C
:10C4900000200240014B186A704700BF0020024094
:10C4A000024BD869C0F34000704700BF0020024033
:10C4B000024B1868C0F34010704700BF00200240D4
:10C4C00019B1054B1A69104303E0034B1A6922EABC
:10C4D00000001861704700BF00200240012804D10D
:10C4E000054BD86900F0010005E0034BDB681842FA
:10C4F0000CBF00200120704700200240014BD86093
:10C50000704700BF00200240094BDA6812F0010FAB
:10C5100001D001200BE0DA6812F0040F01D00220F4
:10C5200005E0DB6813F0100F14BF032004207047F0
:10C530000020024013B504460AE000230193FF33B4
:10C5400001E0019B013B0193019B002BF9D1013CD0
:10C55000FFF7DAFF012802D1002CEED100E004B988
:10C5600005201CBDF8B5124C124B0546A36003F123
:10C5700088330F20A3600E461746FFF7DBFF042821
:10C5800014D1236945F0F80543F0100323612E43CD
:10C59000094B37430B305F80FFF7CCFF012805D0F4
:10C5A000226941F6EF7302EA03032361F8BD00BF7D
:10C5B000002002402301674500F8FF1F38B50546FB
:10C5C00040F6FF70FFF7B6FF04283CD11E4C1F4B0E
:10C5D00040F6FF70A36003F18833A360236943F042
:10C5E00020032361236943F040032361FFF7A2FF87
:10C5F000042820D1226941F6DF7302EA0303236194
:10C60000236943F0100323611DB1114B4FF0000269
:10C6100002E00F4B4FF0A5021A8040F6FF70FFF7C3
:10C6200089FF01280FD0084A41F6EF73116901EA2A
:10C630000303136107E0012805D0226941F6DF7387
:10C6400002EA0303236138BD00200240230167454D
:10C6500000F8FF1F10B504460F20FFF76BFF0428FA
:10C660003DD11F4A1F4BE443936003F1883393602D
:10C670001169E3B241F01001FF2B116106D01A4A93
:10C680000B301381FFF756FF04281FD1C4F3072393
:10C69000FF2B06D0144A0F205381FFF74BFF0428CD
:10C6A00014D1C4F30743FF2B06D00F4A0F20938108
:10C6B000FFF740FF042809D1240EFF2C01D10420EC
:10C6C00006E0094B0F20DC81FFF734FF012806D07C
:10C6D000034A41F6EF73116901EA0303136110BDC8
:10C6E000002002402301674500F8FF1F70B5044693
:10C6F0000F200E46FFF71EFF042815D10B4D0C4BE3
:10C700000B30AB6003F18833AB602B6943F010034F
:10C710002B612680FFF70EFF012805D02A6941F61C
:10C72000EF7302EA03032B6170BD00BF00200240DB
:10C730002301674570B504460F200E46FFF7FAFE49
:10C74000042810D1084D0B302B6943F001032B61F5
:10C750002680FFF7EFFE012805D02A6941F6FE7317
:10C7600002EA03032B6170BD0020024070B504464D
:10C770000F200E46FFF7DEFE042818D10C4DB3B291
:10C780002A690B3042F001022A612380FFF7D2FEB2
:10C79000042804D1360C66800B30FFF7CBFE01284D
:10C7A00005D02A6941F6FE7302EA03032B6170BDCE
:10C7B0000020024010B540F6FF70FFF7BBFE0428D2
:10C7C0002CD1174C174B40F6FF70A36003F1883350
:10C7D000A360236943F020032361236943F04003EE
:10C7E0002361FFF7A7FE042810D1226941F6DF7309
:10C7F00002EA0303236123694FF0A50243F010030B
:10C800002361094B0B301A80FFF794FE012805D0F5
:10C81000226941F6EF7302EA0303236110BD00BFF2
:10C82000002002402301674500F8FF1F10B540F6C5
:10C83000FF70FFF77FFE042814D10B4C40F6FF7009
:10C84000236943F004032361236943F04003236118
:10C85000FFF770FE012805D0226941F6FB7302EA5A
:10C860000303236110BD00BF0020024038B5054618
:10C8700040F6FF70FFF75EFE042815D10B4C40F622
:10C88000FF70236943F0020323616561236943F06C
:10C8900040032361FFF74EFE012805D0226941F6CF
:10C8A000FD7302EA0303236138BD00BF002002408C
:10C8B000CB78F0B513F0100F18BF8A78098803F011
:10C8C0000F0C18BF4CEA020C11F0FF0F1AD00468CD
:10C8D00000220126964006EA0105B5420ED19600D7
:10C8E0000F27B7400CFA06F624EA07043443282B36
:10C8F00001D1456102E0482B08BF05610132082AD9
:10C90000E7D10460FF291CD94468002202F1080520
:10C910000126AE4006EA0105B5420ED196000F276A
:10C92000B7400CFA06F624EA07043443282B01D159
:10C93000456102E0482B08BF05610132082AE5D1B4
:10C940004460F0BD0423C370022383704FF0FF33B3
:10C9500003807047836819420CBF00200120704794
:10C96000806880B2704700BFC36819420CBF0020C6
:10C9700001207047C06880B2704700BF01617047F6
:10C98000416170470AB1016100E04161704700BF39
:10C99000C160704741F48033836181618361836941
:10C9A00083697047064A10B514684FF6807341EAF0
:10C9B000001104EA030341EA0303136010BD00BF42
:10C9C00000000140014B1860704700BF1C0020426E
:10C9D0000304154A00F4401C1B0CBCF5401F30B585
:10C9E000546806D1556824F0706425F07065556070
:10C9F00011E010F4801F06D0C0F303424FF0030C87
:10CA00000CFA02F203E0420D120113FA02F224EAD8
:10CA1000020444F0706419B1400D000183401C43CE
:10CA2000014B5C6030BD00BF0000014001F003031A
:10CA30009B000F229A4010FA03F310B58908074CA7
:10CA4000023154F8210020EA020244F8212054F86F
:10CA50002120134344F8213010BD00BF00000140E5
:10CA60000120014608B500F047FB0120002100F03D
:10CA700043FB08BD08B5264B98422BD00CD8A3F534
:10CA8000006398421AD003F5806398421CD0A3F546
:10CA9000006398423AD10BE01E4B984226D003F532
:10CAA0008063984228D0A3F5006398422ED117E006
:10CAB0000420012100F020FB042024E008200121B3
:10CAC00000F01AFB08201EE01020012100F014FBEA
:10CAD000102018E02020012100F00EFB202012E0A1
:10CAE0004020012100F008FB40200CE080200121C3
:10CAF00000F002FB802006E04FF48070012100F07E
:10CB0000FBFA4FF48070002100F0F6FA08BD00BF78
:10CB100000140140001C01400B4B4FF0FF316FF03F
:10CB20007042C3F88010C3F88420C3F88011C3F8A2
:10CB30008421002303F1C001034A013300200F2B9D
:10CB400042F82100F6D1704700E100E0094B4FF0B8
:10CB500020605860084800224FF0FF319A60D8608A
:10CB60001A615A619A61DA611A625A629962D962EB
:10CB70001963704700ED00E00000FA0540F0BE6068
:10CB8000024B40F42020D860704700BF00ED00E069
:10CB900030B5C27803787AB31C4A4178D2684FF036
:10CBA0000F0CD243C2F302222CFA02FCC2F104029F
:10CBB0009140807803F003020CEA000C4CEA010C6F
:10CBC000D2004FEA0C1CFF2090400CFA02FC01241A
:10CBD00003F01F02944099080D4AC03152F82150C9
:10CBE0000CEA000C25EA00004CEA00005B0942F860
:10CBF000210042F8234008E003F01F020121914088
:10CC00005B09034A203342F8231030BD00ED00E0F9
:10CC100000E100E00023C37003704370837070472D
:10CC2000024B5868C0F30930704700BF00ED00E0C8
:10CC3000012200F01F0312FA03F34009044A4030B6
:10CC400052F820001840984214BF0020012070477D
:10CC500000E100E0014B1860704700BF00EF00E00A
:10CC600000F01F0301229A404009024B603043F854
:10CC70002020704700E100E0024B58688005800DDD
:10CC8000704700BF00ED00E0012200F01F0312FA20
:10CC900003F34009044A803052F8200018409842BB
:10CCA00014BF00200120704700E100E0014B18682C
:10CCB000704700BF00ED00E021F0604121F07F01EE
:10CCC000014B01439960704700ED00E0014A024BBF
:10CCD000DA6070470400FA0500ED00E0014A024BFB
:10CCE000DA6070470100FA0500ED00E019B1054B6C
:10CCF0001A69104303E0034B1A6922EA0000186125
:10CD0000704700BF00ED00E000F01F00012313FAA0
:10CD100000F019B1044B5A6A104303E0024B5A6AFF
:10CD200022EA00005862704700ED00E0144B70B535
:10CD3000DC684FF0FF0CE443C4F302242CFA04F542
:10CD4000C4F1040411FA04F4C0F30126F6000CFA4D
:10CD500006FC02EA050545EA0404240114FA06F675
:10CD6000C0F38110063053F8202022EA0C0243F869
:10CD7000202053F82020164343F8206070BD00BFE8
:10CD800000ED00E0C0F3832001238340044A506A91
:10CD900003EA0000984214BF00200120704700BF42
:10CDA00000ED00E000F01F0001228240024B5968B4
:10CDB0000A435A60704700BF00ED00E000F01F0218
:10CDC0000123013A13FA02F2024B59680A435A60EE
:10CDD000704700BF00ED00E0C0F3833001238340C3
:10CDE000044A506A03EA0000984214BF0020012060
:10CDF000704700BF00ED00E0C0F3814313B90A4B58
:10CE0000D86A10E0012B0CD1074AC0F30153906A95
:10CE1000DA00D040022B14BF00F00F0000F0FF003A
:10CE200001E0014B186B704700ED00E010F4800F3B
:10CE30000BBF024B014B586B986B704700ED00E045
:10CE400008B5F7F795F908BD08B50001F7F78DF9B2
:10CE500008BD00BF08B5F7F786F908BD08B5F7F7B4
:10CE600080F908BD08B5F7F77AF908BD08B5F7F7F6
:10CE700074F908BD0D4B0E4A196841F001011960A3
:10CE8000596801EA02025A601A6822F0847222F498
:10CE900080321A601A6822F480221A605A6822F4DA
:10CEA000FE025A6000229A60704700BF00100240E4
:10CEB0000000FFF80C4BB0F5803F1A6822F4803276
:10CEC0001A601A6822F480221A6003D0B0F5802F0D
:10CED00008D103E01A6842F4803202E01A6842F492
:10CEE000A0221A60704700BF00100240034B1A686E
:10CEF00022F0F80242EAC0021A60704700100240B5
:10CF0000014B1860704700BF00004242044B5A6852
:10CF100022F47C1240EA02020A435A60704700BFC2
:10CF200000100240014B1860704700BF6000424291
:10CF3000034B5A6822F0030240EA02025A6070472B
:10CF400000100240024B586800F00C00704700BF10
:10CF500000100240034B5A6822F0F00240EA02023D
:10CF60005A60704700100240034B5A6822F4E06296
:10CF700040EA02025A60704700100240034B5A68B0
:10CF800022F4605242EAC0025A6070470010024028
:10CF900019B1054B1A78104303E0034B1A7822EAC3
:10CFA00000001870704700BF09100240014B186064
:10CFB000704700BFD8004242034B5A6822F44042F7
:10CFC00040EA02025A60704700100240064B0022FD
:10CFD00001281A701A7002D0042804D101E01870D8
:10CFE00001E005221A70704720100240014B1860C2
:10CFF000704700BF80044242024B1A6A40EA0202B4
:10D000001A62704700100240014B1860704700BF61
:10D010003C0442421F4B10B55A6802F00C02042A2D
:10D0200013D0082A11D15A685968C2F383420232D8
:10D0300011F4803F03D05B6813F4003F01D0164B1E
:10D0400000E0164B5A43026001E0144B0360114AA2
:10D05000134B51680468C1F30311595C34FA01F1B0
:10D0600041605468C4F3022C13F80C4031FA04F404
:10D0700084605468C4F3C22C13F80CC021FA0CF17C
:10D08000C1605268C2F381329B181B7CB1FBF3F183
:10D09000016110BD0010024000093D0000127A003D
:10D0A000E819010819B1054B5A69104303E0034B15
:10D0B0005A6922EA00005861704700BF0010024020
:10D0C00019B1054B9A69104303E0034B9A6922EAB0
:10D0D00000009861704700BF0010024019B1054B75
:10D0E000DA69104303E0034BDA6922EA0000D861F1
:10D0F000704700BF0010024019B1054BDA681043B9
:10D1000003E0034BDA6822EA0000D860704700BFF2
:10D110000010024019B1054B1A69104303E0034B9C
:10D120001A6922EA00001861704700BF001002402F
:10D13000014B1860704700BF40044242014B186029
:10D14000704700BF4C004242014B1870704700BF4F
:10D15000071002404309012B02D1084B1B6805E070
:10D16000022B0BBF054B054B1B6A5B6A00F01F00CF
:10D1700033FA00F000F00100704700BF00100240D9
:10D1800008B53120FFF7E6FF094B18705A680132E5
:10D190005A601A7822B95A6840F2FF139A42F0D1C5
:10D1A0003120FFF7D7FF003818BF012008BD00BFAE
:10D1B000DC060020024B5A6A42F080725A627047C5
:10D1C00000100240034B9B6818420CBF0020012056
:10D1D000704700BF00100240014B1870704700BF3D
:10D1E0000A1002400B884A88B1F804C01A43CB8861
:10D1F00042EA0C02B1F808C01A434B8930B542EA42
:10D200000C028D89B0F800C0CC891A432A4322430E
:10D210000CF4415313439BB20380838B23F40063CC
:10D220001B041B0C83830B8A038230BD00234FF049
:10D230000702C3810282038043808380C38003810D
:10D2400043818381704700BF002343810380438073
:10D250008380C3804FF002030381704721B10388AC
:10D260009BB243F0400304E0038823F040031B0417
:10D270001B0C0380704700BF21B1838B9BB243F42A
:10D28000806304E0838B23F480631B041B0C838383
:10D29000704700BF0909012313FA01F189B21AB1DD
:10D2A00083889BB2194303E083889BB223EA010180
:10D2B000818070471AB183889BB2194303E0838849
:10D2C0009BB223EA01018180704700BF81817047D2
:10D2D000808980B2704700BF4FF6FF63994205D046
:10D2E00003889BB243F48073038002E003881940F3
:10D2F0000180704721B183889BB243F0040304E0AE
:10D30000838823F004031B041B0C8380704700BF39
:10D31000038823F400631B041B0C038003889BB267
:10D3200041EA03030380704703889BB243F48053B0
:10D330000380704721B103889BB243F4005304E09B
:10D34000038823F400531B041B0C0380704700BFA9
:10D35000012914BF008B808A80B27047008A80B296
:10D36000704700BFB1F5804F04D103889BB243F4EE
:10D37000804304E0038823F480431B041B0C0380D8
:10D38000704700BF038919420CBF0020012070477D
:10D39000202906D1038903889BB243F04003038010
:10D3A00008E0402901D0082901D1038902E0C943DE
:10D3B00089B20181704700BF012301F00F0213FA07
:10D3C00002F2B0F804C000891FFA8CFC80B2104051
:10D3D00006D009098B401CEA030F0CBF0020012076
:10D3E000704700BF552906D1038903889BB243F0DB
:10D3F000400303800DE0562901D0532901D1038950
:10D4000007E001F00F01012313FA01F1C94389B2CA
:10D4100001817047838BF0B523F47A6323F01F03F7
:10D420001B041B0C83834FF0020303840B89868B40
:10D43000022B87B004460D46B6B201D1002225E08A
:10D4400001A88F88FFF7E6FDEB88002F0CBF0127AE
:10D450000227B3F5007F2989019A06D1A3F5FB7352
:10D4600053430902B3FBF1F305E00A2349015A4390
:10D470004F43B2FBF7F305330A229BB2B3FBF2F33F
:10D4800003F001021202C3F34F0392B2991E89B254
:10D49000FE2928BF002228BF0223E98842EA0303AD
:10D4A0000B439BB223842B886A8846EA0303A9882E
:10D4B00043F4006313436A890B4313439BB2A38372
:10D4C00007B0F0BD08B5154B98421BD003F5744367
:10D4D000984204D0A3F5784398421DD10AE0012177
:10D4E0004FF48050FFF708FE4FF480500021FFF703
:10D4F00003FE11E04FF480400121FFF70BFE4FF4D3
:10D50000804006E04FF400400121FFF703FE4FF496
:10D5100000400021FFF7FEFD08BD00BF003C0040B9
:10D52000042804D1054B1A6842F0040203E0034BBF
:10D530001A6822F004021A60704700BF10E000E091
:10D54000014B5860704700BF10E000E0012804D193
:10D55000084B1A6842F0010206E010F1020F05D1F3
:10D56000044B1A6822F001021A6002E0014B00220B
:10D570009A60704710E000E020B1054B1A6842F055
:10D58000020203E0024B1A6822F002021A6070479E
:10D5900010E000E0014B9868704700BF10E000E029
:10D5A000C308022B0BBF044B034B1B68DB6833FA29
:10D5B00000F000F00100704710E000E0038803F085
:10D5C0008F0303800388B1F806C04A889BB243EA00
:10D5D0000C0313439BB203808B8883850B880385E0
:10D5E000064B984203D003F50063984201D10B7AB1
:10D5F00003864FF001038382704700BF002C014077
:10D60000038C2DE9F04123F001031B041B0C038460
:10D61000038C0A894C8823F002031C4E14431B041C
:10D620008288B1F806C0058B1B0CA4B2B04244EA54
:10D63000030392B20C88ADB2A0F834C003D006F553
:10D640000066B04218D18E894F89B1F80E804FF62E
:10D65000F77C03EA0C0C4CEA070748EA06064FF68B
:10D66000FB73898847F6FF4C02EA0C0C07EA0303B8
:10D67000B2B20B4342EA0C024FF68F7105EA010188
:10D680002143828001830384BDE8F081002C0140A6
:10D69000038C2DE9F04123F010031B041B0C0384C1
:10D6A000028CB1F808C022F0200212048488120C07
:10D6B0004B8842EA0C1242EA0313A2B21B4C068BBF
:10D6C000B1F806C0A0420D88B6B29BB2A0F838C02F
:10D6D00003D004F50064A0421BD1B1F80A804FF6D4
:10D6E0007F748F8903EA040447F2FF3C02EA0C0CC2
:10D6F00044EA0814CA894FF6BF73898804EA030311
:10D700004CEA870C43EA01134CEA82023C469BB286
:10D7100092B248F6FF7106EA010141EA052189B299
:10D72000828001830384BDE8F08100BF002C0140AA
:10D73000038C2DE9F04123F480731B041B0C03843C
:10D74000028CB1F808C022F4007212048488120C12
:10D750004B8842EA0C2242EA0323A2B21A4C868B7F
:10D76000B1F806C0A0420D88B6B29BB2A0F83CC08A
:10D7700003D004F50064A0421BD1B1F80A804FF237
:10D78000FF748F8903EA040444F6FF7C02EA0C0C60
:10D7900044EA0824CA894FF6FF33898804EA030360
:10D7A0004CEA071C43EA01234CEA02123C469BB2B6
:10D7B00092B24FF68F7106EA01012943828081837C
:10D7C0000384BDE8F08100BF002C0140038CF0B55C
:10D7D00023F480531B041B0C0384B1F806C0078C90
:10D7E0000C8882880D89868B4B88A0F840C0DFF8B2
:10D7F00048C0BFB2604592B2B6B203D00CF5006C1F
:10D80000604505D192048989920C42EA811292B254
:10D810004DF6FF7C07EA0C0C48F6FF7106EA0101A1
:10D820004CEA053C41EA04214CEA033389B29BB23D
:10D83000828081830384F0BD002C0140B1F802C0D6
:10D840000B888A884CEA0303B1F806C013430A899F
:10D8500043EA0C03B1F80AC013438A8943EA0C0374
:10D8600013439BB2A0F84430704700BF00234FF031
:10D87000FF320372438082800380C380704700BF01
:10D880000023C381038043808380C380038143815D
:10D890008381704700234FF001020381038043809E
:10D8A0008280C380704700BF002383810380438050
:10D8B0008380C38003814381704700BF21B1038807
:10D8C0009BB243F0010304E0038823F001039B05AE
:10D8D0009B0D0380704700BF39B1B0F844306FEA48
:10D8E00043436FEA53439BB203E0B0F844305B0418
:10D8F0005B0CA0F8443070471AB183899BB219437E
:10D9000003E083899BB223EA01018181704700BF54
:10D91000818270470A43A0F8482070471AB1838972
:10D920009BB2194303E083899BB223EA0101818101
:10D93000704700BF038923F007031B041B0C0381FE
:10D94000704700BFB0F808C05FFA8CFC41EA0C0CCD
:10D9500042EA0C0C4CEA032C1FFA8CFCA0F808C01D
:10D96000704700BF10B50446FFF7ECFF23899BB258
:10D9700043F48043238110BD10B50446FFF7E2FF56
:10D98000238923F077031B041B0C43F077032381C7
:10D9900010BD00BF01858282704700BF038823F05D
:10D9A00070039B059B0D41EA03030380704700BF92
:10D9B000038923F070031B041B0C41EA030303815A
:10D9C000704700BF10B50446FFF7F2FF23899BB2F2
:10D9D00043F00703238110BD30B50489B0F818C0A7
:10D9E000058C2CF4407CADB22CF0030C24F0070421
:10D9F0004FEA0C4C25F0220542EA050524044FEAC3
:10DA00001C4C45EA0315240C4CF4807C21434CF05B
:10DA1000010CADB20181A0F818C0058430BD00BF73
:10DA2000038B23F070031B041B0C41EA03030383E5
:10DA3000704700BF038B23F4E0431B041B0C43EA35
:10DA400001239BB203837047838B23F070031B0475
:10DA50001B0C41EA03038383704700BF838B23F4CD
:10DA6000E0431B041B0C43EA01239BB283837047F2
:10DA700021B103889BB243F0800304E0038823F0C4
:10DA800080039B059B0D0380704700BF21B18388F5
:10DA90009BB243F0040304E0838823F004031B04D7
:10DAA0001B0C8380704700BF21B183889BB243F079
:10DAB000080304E0838823F008031B041B0C838005
:10DAC000704700BF21B183889BB243F0010304E09B
:10DAD000838823F001031B041B0C8380704700BF65
:10DAE000038B23F008031B041B0C41EA030303838D
:10DAF000704700BF038B23F400631B041B0C43EA35
:10DB000001239BB203837047838B23F008031B041C
:10DB10001B0C41EA03038383704700BF838B23F40C
:10DB200000631B041B0C43EA01239BB283837047F1
:10DB3000038B23F004031B041B0C41EA0303038340
:10DB4000704700BF038B23F480631B041B0C43EA64
:10DB500001239BB203837047838B23F004031B04D0
:10DB60001B0C41EA03038383704700BF838B23F4BC
:10DB700080631B041B0C43EA01239BB28383704721
:10DB8000038B23F080031B041B0C41EA0303038374
:10DB9000704700BF038B5B045B0C43EA01239BB21D
:10DBA00003837047838B23F080031B041B0C41EA23
:10DBB00003038383704700BF838B5B045B0C43EAE2
:10DBC00001239BB283837047038C23F002031B0461
:10DBD0001B0C41EA03030384704700BF038C23F04E
:10DBE00008031B041B0C41EA03030384704700BFB6
:10DBF000038C23F020031B041B0C43EA01139BB28C
:10DC000003847047038C23F080031B041B0C43EA3E
:10DC100001139BB203847047038C23F400731B042D
:10DC20001B0C43EA01239BB203847047038C23F44B
:10DC300000631B041B0C43EA01239BB2038470475F
:10DC4000038C23F400531B041B0C43EA01339BB2E7
:10DC50000384704701238B408A40018C89B221EAFA
:10DC600003030384018C0A4392B20284704700BF0D
:10DC700004238B408A40018C89B221EA0303038488
:10DC8000018C0A4392B20284704700BF01238B408B
:10DC9000B0F820C010B51FFA8CFC2CEA03030384F3
:10DCA00009B1082909D11830490844584FF68F7333
:10DCB00004EA0303435043580CE004391830C1F31D
:10DCC0004E01445848F6FF7304EA0303435012021E
:10DCD000435892B243EA0202425010BD21B1038878
:10DCE0009BB243F0020304E0038823F002039B0588
:10DCF0009B0D0380704700BF21B103889BB243F0A6
:10DD0000040304E0038823F004039B059B0D0380B8
:10DD1000704700BF21B183889BB243F0800304E0C9
:10DD2000838823F080031B041B0C8380704700BF93
:10DD3000038823F008039B059B0D038003889BB297
:10DD400041EA030303807047838823F070031B04B8
:10DD50001B0C838083889BB241EA03038380704756
:10DD6000038923F007031B041B0C038103899BB267
:10DD700041EA030303817047038923F080031B04F6
:10DD80001B0C038103899BB241EA030303817047A3
:10DD9000818470478185704781867047018770470D
:10DDA00081877047A0F84010704700BF038B23F0B5
:10DDB0000C031B041B0C0383038B9BB241EA03037C
:10DDC00003837047038B23F440631B041B0C038302
:10DDD000038B9BB243EA01239BB20383704700BFCE
:10DDE000838B23F00C031B041B0C8383838B9BB25C
:10DDF00041EA030383837047838B23F440631B044E
:10DE00001B0C8383838B9BB243EA01239BB28383E6
:10DE1000704700BF0388DBB2038003889BB241EAEE
:10DE200003030380704700BF808E80B2704700BF3D
:10DE3000008F80B2704700BF808F80B2704700BFF4
:10DE4000B0F8400080B27047808C80B2704700BF4D
:10DE5000008D80B2704700BF038A19420CBF0020BA
:10DE600001207047C94389B201827047038A8289C1
:10DE700011EA030092B203D011420CBF002001202E
:10DE8000704700BFC94389B201827047B0F820C013
:10DE900010B52CF0010C4FEA0C4C4FEA1C4CA0F8CA
:10DEA00020C0048BB0F820C0A4B21FFA8CFC24F070
:10DEB000F30442EA04042CF0020C44EA03144CF08C
:10DEC000010C4CEA010CA4B20483A0F820C010BDE0
:10DED000B0F820C010B52CF0100C4FEA0C4C4FEAF3
:10DEE0001C4CA0F820C0B0F818C0048C2CF4407C66
:10DEF000A4B24FEA0C5C4FEA1C5C24F020044CEA0C
:10DF0000022C44F010044CEA033C44EA01141FFACA
:10DF10008CFCA4B2A0F818C0048410BD38B50D461E
:10DF2000602D1146044603D10122FFF7D1FF02E024
:10DF30000122FFF7ABFF29462046FFF739FD238971
:10DF40009BB243F00703238138BD00BFF8B50C46F0
:10DF5000A2884988B4F800C0054600290CBF0227F2
:10DF60000027012A0CBF022601262389BCF1000FDD
:10DF700010D1FFF78BFF2846E188FFF717FF2846EF
:10DF8000394632462389FFF7A3FF2846E188FFF789
:10DF900019FF0FE0FFF79CFF2846E188FFF712FF0B
:10DFA0002846394632462389FFF770FF2846E18824
:10DFB000FFF7FCFEF8BD00BF38B50B880C460546E0
:10DFC0004BB94988A2882389FFF760FF2846E1887A
:10DFD000FFF7ECFE53E0042B09D14988A28823897E
:10DFE000FFF776FF2846E188FFF7ECFE47E0082BB5
:10DFF000B1F802C0B1F804E0098920D1028C22F402
:10E0000080721204120C0284838B028C9BB292B237
:10E0100023F0F30322F4007243EA011142EA0C2CCC
:10E0200089B21FFA8CFC41EA0E0E4CF4807CA0F8F9
:10E030001CE0A0F820C0E188FFF7D2FE1FE0028CB0
:10E0400022F480521204120C0284838B028C23F47B
:10E05000407392B21B051B0D22F4005243EA0E23BB
:10E0600042EA0C3C43EA01331FFA8CFC9BB24CF4AD
:10E07000805C8383A0F820C0E188FFF7BDFE38BD37
:10E0800008B52D4B984237D00BD8A3F500639842C2
:10E0900026D003F58063984228D0B0F1804F4AD152
:10E0A00018E0264B984233D004D8A3F580639842F9
:10E0B00041D127E0224B984204D003F500639842F7
:10E0C00039D12EE04FF400600121FFF715F84FF42D
:10E0D00000602DE001200146FFF71CF801201CE044
:10E0E00002200121FFF716F8022016E0042001218A
:10E0F000FFF710F8042010E008200121FFF70AF8CC
:10E1000008200AE010200121FFF704F8102004E0A5
:10E1100020200121FEF7FEFF20200021FEF7FAFF5C
:10E1200009E04FF400500121FEF7E6FF4FF40050E4
:10E130000021FEF7E1FF08BD000C00400014004084
:10E14000002C0140002383814FF416528380C3804A
:10E1500003814FF00C030260438170470A8810B5B9
:10E160004C88B1F804C0038AC98844EA020242EA32
:10E170000C0223F470630A431B041B0C92B242EAA4
:10E180000303038210BD00BF0023C38003804380CC
:10E190008380704721B183899BB243F4005304E02C
:10E1A000838923F400531B041B0C8381704700BF39
:10E1B00001F01F034FF0010CC1F3421161450CFA4D
:10E1C00003F301D10C3004E0022901D1103000E04A
:10E1D00014301AB1026842EA030302E0026822EA3C
:10E1E00003030360704700BF1AB1838A9BB21943CF
:10E1F00003E0838A9BB223EA01018182704700BF5A
:10E20000038A23F00F031B041B0C0382038A9BB2B7
:10E2100041EA030303827047838923F400631B04EC
:10E220001B0C838183899BB241EA0303838170477E
:10E2300021B183899BB243F0020304E0838923F078
:10E2400002031B041B0C8381704700BF038A23F069
:10E2500020031B041B0C0382038A9BB241EA0303C5
:10E260000382704721B1038A9BB243F4804304E0E8
:10E27000038A23F480431B041B0C0382704700BFF6
:10E28000C905C90D818070478088C005C00D7047E1
:10E2900083899BB243F0010383817047038BDBB218
:10E2A0000383038B9BB243EA01230383704700BFC0
:10E2B000038B03F47F430383038B9BB241EA030385
:10E2C0000383704721B1838A9BB243F0200304E0AB
:10E2D000838A23F020031B041B0C8382704700BF3A
:10E2E00021B1838A9BB243F0100304E0838A23F0B8
:10E2F00010031B041B0C8382704700BF21B1838A6B
:10E300009BB243F0080304E0838A23F008031B0454
:10E310001B0C8382704700BF838A23F004031B0415
:10E320001B0C8382838A9BB241EA0303838270477A
:10E3300021B1838A9BB243F0020304E0838A23F075
:10E3400002031B041B0C8382704700BF0388194221
:10E350000CBF002001207047C94389B2018070477B
:10E360004FF0010CC1F3421201F01F0362450CFA99
:10E3700003F301D1828903E0022A0CBF028A828A58
:10E3800092B21340028892B20BB9184607E0090A0C
:10E39000012313FA01F111420CBF00200120704744
:10E3A000090A01238B40DB439BB20380704700BF07
:10E3B000038ACA8823F440531B041B0C13430382B3
:10E3C00083898A8830B5044608890D4623F4B05302
:10E3D000498940EA020223F00C030A431B041B0C88
:10E3E00092B242EA0303A381A38AAA8923F4407369
:10E3F0001B041B0C134387B0A38201A8FEF70AFE7F
:10E400000E4B2A689C420CBF049B039B1921594365
:10E4100092006423B1FBF2F1B1FBF3F21201100997
:10E4200003FB101109013231B1FBF3F303F00F03C9
:10E4300043EA020292B2228107B030BD00380140A7
:10E4400008B5214B98422BD008D8A3F50063984219
:10E4500016D003F58063984234D119E01B4B9842E3
:10E4600026D003F5684398422CD101214FF4804017
:10E47000FEF742FE4FF480400021FEF73DFE21E012
:10E480004FF400300121FEF745FE4FF4003016E056
:10E490004FF480200121FEF73DFE4FF480200EE076
:10E4A0004FF400200121FEF735FE4FF4002006E076
:10E4B0004FF480100121FEF72DFE4FF48010002153
:10E4C000FEF728FE08BD00BF004C00400050004091
:10E4D000684620F007018D4601B5002303E00B4993
:10E4E0005958995004330A4A0A4998188842F6D371
:10E4F000094B02E0002243F8042B084A9342F9D367
:10E50000F5F73EFEBDE8014085467047401B010817
:10E510000000002030020020300200208C0D00207E
:10E5200010B5074C20B922684FF00103138205E0B3
:10E53000044B1B681B68984720680A3010BD00BF59
:10E54000240D0020E00C002010B50A4B0A4A1B687D
:10E550005178DA7891420AD3997841B99C8834B9D4
:10E560009A72064B1B685B689847204600E00220C1
:10E5700010BD00BF240D002004010020E00C00208D
:10E5800010B5074C20B922684FF00103138205E053
:10E59000044B1B689B68984720680C3010BD00BF77
:10E5A000240D0020E00C002038B50E4C0E4B2268E4
:10E5B0001B68D1789B695079984723689A7A7AB119
:10E5C00070B91A7962B99D7855B9084B1B68DB6838
:10E5D0009847236828465979DA78D9721A7300E087
:10E5E000022038BD240D0020BC0C0020E00C0020CF
:10E5F00008B50246244B20B91B684FF0020119826E
:10E6000040E0224A4FF000011B681180197811F098
:10E610007F0113D15B7A13F0200F03D0117841F002
:10E620000201117013F0400F184B15BF1A781A78B9
:10E6300022F0010242F001021A701EE0012921D0ED
:10E64000022901D000221DE0597911F0800F01F05C
:10E650000F0306D00E4951F8233003F03003102B7E
:10E6600006E00B4951F8233003F44053B3F5805FC3
:10E6700003D1137843F001031370064B1B681B6929
:10E680009847024A104608BD240D0020840D002042
:10E69000005C0040E00C002010B51E4B19684A7960
:10E6A00012F0800F22F0800305D01B4850F82300A1
:10E6B00000F0300004E0184850F8230000F4405007
:10E6C000164C94F800C0634522D24C8804BBF8B1C4
:10E6D000897AE9B112F0800F09D00F4948F6BF726C
:10E6E00051F8230000EA020282F0100208E00A4911
:10E6F0004BF68F7251F8230000EA020282F4805236
:10E7000041F82320064B1B689B699847002000E0D6
:10E71000022010BD240D0020005C004004010020F8
:10E72000E00C002008B5064B1B685A7A42F0200224
:10E730005A72044B1B68DB699847002008BD00BF74
:10E74000240D0020E00C0020054B1A68538A18B9EC
:10E750008988CB1A138201E008681818704700BF37
:10E76000240D002030B50E4B1C78002310E05FFA1A
:10E7700083FC4FEA8C0202F1804202F5B842156830
:10E7800048F68F7105EA010141EA0C01116001337D
:10E79000A342ECD3034B40F08000186030BD00BFB3
:10E7A000040100204C5C0040704700BF08B50C4BD2
:10E7B000002093F82C1000F04FFE0A4B1B68187ACB
:10E7C000082807D1084B4FF480521A80074B4FF0AE
:10E7D00010021A80092814BF0020012008BD00BFC4
:10E7E00080000020240D0020860D0020880D0020D0
:10E7F00070B52D4B1C68237A032B01D0052B46D115
:10E80000A369228AABB1A2B1A58A954228BF154659
:10E8100028469847228A638A521BEB1806462282B2
:10E820006382002000F0E8FD2A460146304600F0F1
:10E83000FBFB238A5BB11D4B4FF4405200201A8032
:10E84000014600F0E7FD1A4B4FF030021A80A28A11
:10E85000238A9A4203D8144B03221B6803E0124A0E
:10E860001BB1136805221A720DE01268062111729D
:10E87000104A1168104A89B28A18520013600C4B72
:10E880004FF030021A80084B1B681B7A06E0072BFA
:10E8900003D10A4B1B68DB6898470823024A1268B9
:10E8A0001372FFF783FF70BD240D0020860D00203A
:10E8B000880D0020505C004002300020BC0C00207D
:10E8C000F8B5244B1C68238A267ABBB9042E15D1CF
:10E8D000214822490278012A0BD1214C214A24687F
:10E8E0000370A0B28218520013604FF030020A8009
:10E8F0002BE04FF010030B80072626E0A68AA269C2
:10E900009E4234BF35461D462846B34294BF042676
:10E91000022690470746002000F060FD2A46014687
:10E92000384600F069FB2946002000F073FD638A39
:10E93000228AEB186382094B551B4FF03002258267
:10E940001A80094B4FF440521A80024B1B681E720A
:10E95000F8BD00BF240D0020E4060020880D002033
:10E96000505C004002300020860D002008B5144B9A
:10E970001B681A7A022A01D0042A05D1FFF7A0FFEA
:10E980000F4B1B681B7A14E0062A11D15A78052A0E
:10E990000AD11A7812F07F0F06D1D878FFF7E2FE7D
:10E9A000084B1B681B6A9847074B1B689B68984776
:10E9B0000823034A12681372FFF7F8FE08BD00BF70
:10E9C000240D0020E00C0020BC0C002038B5324B98
:10E9D0001B68187810F07F0004D15A7A22F02002C8
:10E9E0005A7258E0022855D15A88002A52D11A7911
:10E9F000002A4FD15A7912F0800F22F0800405D0FE
:10EA0000264951F8241001F0300104E0234951F85F
:10EA1000241001F440512248007884423AD200295F
:10EA200038D09B7A002B35D012F0800F0FD01B4BC3
:10EA300053F8243003F03003102B25D1E4B22046E4
:10EA400000F082FC2046302100F05EFB1CE0134DFC
:10EA500055F8243003F44053B3F5805F14D134B932
:10EA6000104B204693F82C1000F0F6FC02E02046F4
:10EA700000F056FC55F824204BF68F7302EA03038E
:10EA800083F4405345F82430074B1B685B69984773
:10EA9000002000E0022038BD240D0020005C004072
:10EAA0000401002080000020E00C0020F7B58D4B11
:10EAB0008D4E1A6835688D4B92B2D3182A7A5B0056
:10EAC000092A1B681BD09BB203F1005303F5405386
:10EAD0005B001C4614F8012B03F10A072A705B78CF
:10EAE0006B70B4F8030000F063FE6880B4F80700B0
:10EAF000346800F05DFEA08033687F88DF807A4C48
:10EB000001212368DA8819725D78002A62D11A78A7
:10EB100012F07F022ED1092D02D1FFF715FD3BE047
:10EB2000052D0DD193F90320002A4EDB9A78002A97
:10EB30004BD19A88002A48D19B7A002B37D044E0E9
:10EB4000032D0BD1DA78012A27D19A882ABB5B7A68
:10EB500013F0200F21D0FFF7E5FD1DE0012D1CD1A2
:10EB6000DA78012A19D19A88BAB95B7A13F0200FA2
:10EB700013D00AE0012A04D10B2D0ED1FFF714FDAA
:10EB80000AE0022A09D1012D02D1FFF71FFF03E09D
:10EB9000032D02D1FFF780FD48B1554B28461B6875
:10EBA0005B699847032801D109230FE068B94D4AF2
:10EBB000504B12684FF0300192B2D3185B00002224
:10EBC0001A604D4B1980062300E00823464A12685C
:10EBD0001372E3E0062D18D11A7812F07F0F40F07F
:10EBE00097809B78012B03D1414B1B68DB696EE05A
:10EBF000022B03D13E4B1B681B6A68E0032B40F0DD
:10EC000087803B4B1B685B6A61E0002D3CD15988D3
:10EC100000297DD15A6822F47F42B2F5003F77D1B6
:10EC20001A7812F07F0203D19B88002B70D129E063
:10EC3000012A0BD158792E4B1B689B6998470028F5
:10EC400066D123689B7A002B62D01BE0022A5FD139
:10EC50005B7913F0800F03F00F0205D0274951F8BC
:10EC6000221001F0300104E0244951F8221001F48F
:10EC700040512348007882424AD213F0700F47D1A6
:10EC8000002945D01F4B23E0082D05D11B7813F038
:10EC90007F0F3DD11C4B1BE00A2D39D11A7802F0B1
:10ECA0007F02012A34D19A7A002A31D0598800296A
:10ECB0002ED15A6822F47F42B2F5803F28D158798C
:10ECC0000B4B1B689B69984710BB104B00E0FBB1D6
:10ECD000054A4FF000011268002093615182984765
:10ECE000002020E0505C0040240D00200430002073
:10ECF000BC0C002002300020880D0020005C004089
:10ED000004010020F1E5000821E5000881E5000884
:10ED1000244C254B22681B6850781B6998470328B0
:10ED200001D1236806E01F4B4FF6FF711B681A8A5A
:10ED30008A4201D1092203E0022800D012B9082238
:10ED40001A722BE093F90010002921DAD988019179
:10ED50000198824202D9019A1A8211E08A420FD2A6
:10ED60001149096891F82C108A4201D2002105E06E
:10ED700092FBF1F001FB102212B901210B4A117034
:10ED8000094A126892F82C209A82FFF799FD05E053
:10ED900003221A72064B4FF440521A80FFF706FD09
:10EDA000FEBD00BF240D0020BC0C0020E4060020A6
:10EDB000860D0020074A022108B50748117207494D
:10EDC000074B086007490A60074A13601B689847A9
:10EDD00008BD00BFC40C002008010020E00C00208A
:10EDE00080000020240D0020BC0C002008B529E084
:10EDF00047F6FF700860198801F00F018B0003F1DE
:10EE00008043117003F5B843196889B211F4004FBB
:10EE100009D0186840F68F7100EA01011960127874
:10EE20000E4B013A0BE011F0800F0BD0186848F63A
:10EE30000F7100EA010119601278094B013A53F889
:10EE4000223098470749084B0868084A80B2188062
:10EE5000188800B20028CBDB08BD00BFE800002006
:10EE6000CC000020445C0040BA0C0020C00C002004
:10EE7000F8B59AE047F6FF761E601688564F06F002
:10EE80000F06B30003F1804303F5B8433E70002E34
:10EE900064D127682668236807F4405C03EA000011
:10EEA00080F400502060236806F0300003EA01017E
:10EEB00081F0200121601388484A13F0100F108060
:10EEC000A5F800C004D023689BB213F0800F08D0CF
:10EED000226848F60F7302EA03032360FFF746FD3A
:10EEE00016E013F4006F08D0226840F68F7302EA30
:10EEF00003032360FFF7DAFD0AE013F4004F54D058
:10EF0000226840F68F7302EA03032360FFF770FC68
:10EF100021682A884BF68F7301EA030312F4805F9D
:10EF200018BF83F4805312F4005F2D4A18BF83F496
:10EF300000531360294B11681A8848F6BF7301EA21
:10EF4000030312F0100F18BF83F0100312F0200F0C
:10EF5000234A18BF83F0200313603BE01C68A4B26F
:10EF600014F4004F0BD0196840F68F7201EA0202C8
:10EF70001A603A781B4B013A53F82230984714F044
:10EF8000800F12D0144948F60F720B789B0003F1E2
:10EF9000804303F5B843186800EA02021A600A7851
:10EFA000114B013A53F822309847104B104A1D6814
:10EFB0000B4C1FFA85FCA2F800C0B2F800C04BF65B
:10EFC0008F700FFA8CFCBCF1000F48F6BF71094D31
:10EFD000FFF650AFF8BD00BFC00C0020880D002028
:10EFE000005C0040E8000020CC000020445C0040B1
:10EFF000BA0C0020860D002001F10051013201F50C
:10F00000405110B549005208002308E010F803C031
:10F010006478013A4CEA042C21F813C00233C41876
:10F02000002AF3D110BD00BF01F10051013201F5FA
:10F03000405110B549005208002304E031F8134054
:10F04000013AC4520233002AF8D110BD014B1860B6
:10F05000704700BF405C0040014B186880B27047A9
:10F06000405C0040014B1860704700BF445C0040AA
:10F07000014B186880B27047445C0040014B18682F
:10F0800080B27047485C0040014B1860704700BF79
:10F090004C5C0040014B186880B270474C5C0040EB
:10F0A0004FF6F873024A00EA03031360704700BF8B
:10F0B000505C0040014B186880B27047505C0040C3
:10F0C000014B43F820107047005C0040024B53F89E
:10F0D000200080B2704700BF005C0040054B10B5B7
:10F0E00053F8204048F68F1204EA02020A4343F81C
:10F0F000202010BD005C0040024B53F8200000F4BB
:10F10000C0607047005C00400A4B10B553F82020E7
:10F1100048F6BF7402EA040411F0100F18BF84F01F
:10F12000100411F0200F18BF84F0200443F8204091
:10F1300010BD00BF005C00400A4B10B553F8202002
:10F140004BF68F7402EA040411F4805F18BF84F454
:10F15000805411F4005F18BF84F4005443F8204039
:10F1600010BD00BF005C004038B50D460446FFF7F7
:10F17000ADFF012D02D120F4805003E0022D04D117
:10F1800020F01000014B43F8240038BD005C004023
:10F19000024B53F8200000F030007047005C004044
:10F1A000024B53F8200000F440507047005C0040D0
:10F1B000054B48F6BF7253F8201001EA020282F0B4
:10F1C000300243F820207047005C0040054B4BF6AE
:10F1D0008F7253F8201001EA020282F4405243F881
:10F1E00020207047005C0040054B48F68F6253F8C2
:10F1F000201001EA020242F4807243F82020704796
:10F20000005C0040044B48F68F6253F8201001EA7E
:10F21000020243F820207047005C0040044B48F68F
:10F220008F6253F8201001EA020243F82020704751
:10F23000005C0040054B48F68F6253F8201001EA4D
:10F24000020242F4807243F820207047005C0040C4
:10F25000054B48F68F6253F8201001EA020242F48F
:10F26000807243F820207047005C0040044B48F651
:10F270008F6253F8201001EA020243F82020704701
:10F28000005C0040044B53F8200000F030001028D0
:10F2900014BF002001207047005C0040054B53F86C
:10F2A000200000F44050B0F5805F14BF0020012022
:10F2B000704700BF005C0040044B40F68F7253F86B
:10F2C000201001EA020243F820207047005C004051
:10F2D000044B48F60F7253F8201001EA020243F87B
:10F2E00020207047005C0040054B48F68F7253F8B1
:10F2F000201001EA020242F4804243F820207047C5
:10F30000005C0040054B48F68F7253F8201001EA6C
:10F31000020242F0400243F820207047005C0040A7
:10F32000084B53F8202012F4804F09D053F82010D6
:10F3300048F68F7201EA020242F4804243F820202C
:10F34000704700BF005C0040084B53F8202012F0CB
:10F35000400F09D053F8201048F68F7201EA0202DC
:10F3600042F0400243F82020704700BF005C00409C
:10F37000054B10B553F8204048F68F7204EA02029C
:10F380000A4343F8202010BD005C0040024B53F8B4
:10F39000200000F00F007047005C0040064B490859
:10F3A0001B6849009BB203EBC00303F1005303F554
:10F3B00040535B0019607047505C0040054A064BA3
:10F3C0001268490892B202EBC002D3185B004900F0
:10F3D00019607047505C004004300020054B1B68EA
:10F3E0009BB203EBC00303F1005303F540535B00F2
:10F3F00018887047505C0040044A054B126892B26E
:10F4000002EBC002D3185B0018887047505C0040C4
:10F4100004300020044A054B126892B202EBC0028D
:10F42000D3185B0019607047505C00400230002028
:10F430003E2909D94B0911F01F0F01D1013B9BB2A5
:10F440009B0243F4004305E04B0811F0010F18BF85
:10F4500001339B02036070470D4A0E4B126892B253
:10F46000D31803EBC0035B003E2909D94A0911F008
:10F470001F0F01D1013A92B2920242F4004205E01C
:10F480004A0811F0010F18BF013292021A6070474A
:10F49000505C004006300020054A064B126892B2CC
:10F4A00002EBC002D3185B0018688005800D70471E
:10F4B000505C004002300020054A064B126892B2B0
:10F4C00002EBC002D3185B0018688005800D7047FE
:10F4D000505C0040063000200C4B30B51D681C68A5
:10F4E000C0001FFA85FC8444A4B2094B00190CF13A
:10F4F000005CC3180CF5405C490852084FEA4C0008
:10F5000049005B00520001601A6030BD505C004051
:10F5100004300020064B49081B6849009BB203EBEE
:10F52000C00303F1005303F540535B0019607047BB
:10F53000505C0040054A064B1268490892B202EB43
:10F54000C002D3185B00490019607047505C00404E
:10F5500004300020054B1B689BB203EBC00303F192
:10F56000005303F540535B0018887047505C00401F
:10F57000044A054B126892B202EBC002D3185B003A
:10F5800018887047505C004004300020012910B5F5
:10F5900024D1254B25491B68C0009BB25918091876
:10F5A0004B003E2A09D9510912F01F0F01D1013930
:10F5B00089B2890241F4004105E0510812F0010FBF
:10F5C00018BF0131890219601749194B096889B2BE
:10F5D000CB18181840003E2A1ED913E0022922D168
:10F5E000114BC0001C681B68A4B21FFA83FC0F49B2
:10F5F0000F4B844400194118634449005B000A60C2
:10F600001A6010E0530912F01F0F01D1013B9BB2A9
:10F610009B0243F4004305E0530812F0010F18BFAA
:10F6200001339B02036010BD505C0040023000209B
:10F630000630002001291BD11349144B096889B2F7
:10F64000CB1803EBC00040003E2A09D9530912F041
:10F650001F0F01D1013B9BB29B0243F4004305E025
:10F66000530812F0010F18BF01339B0203600AE038
:10F67000022908D10449054B096889B201EBC00091
:10F68000C3185B001A607047505C004002300020D5
:10F6900001291BD11349144B096889B2CB1803EB1C
:10F6A000C00040003E2A09D9530912F01F0F01D1B2
:10F6B000013B9BB29B0243F4004305E0530812F068
:10F6C000010F18BF01339B0203600AE0022908D131
:10F6D0000449054B096889B201EBC000C3185B00FF
:10F6E0001A607047505C004006300020054A064B07
:10F6F000126892B202EBC002D3185B001868800552
:10F70000800D7047505C004002300020054A064BD7
:10F71000126892B202EBC002D3185B001868800531
:10F72000800D7047505C0040063000200D4BC0003B
:10F7300019680D4A89B241188A185200128812F4C9
:10F740007C4F01D001200CE01A68084B92B280185F
:10F75000C3185B0018888005800D002814BF0220A4
:10F7600000207047505C004006300020023000202E
:10F77000012909D10B4A48F68F7352F8201001EA8B
:10F78000030343F040030AE002290AD1054A48F680
:10F790008F7352F8201001EA030343F4804342F8C8
:10F7A00020307047005C004041EA0020704700BFF5
:10F7B000030AC0B243EA0020704700BF08B5002228
:10F7C0000A2300F045F808BD08B500210A2200F020
:10F7D000DFF808BDF0B40378002B2DD040F23412CE
:10F7E000C2F20002156802E010F8013FEBB15A19AD
:10F7F00003F12004527812F001070A7808BF1C4672
:10F8000001F10101561C9446AE5D16F0010F18BFC0
:10F8100002F1200C6445E7D007B1203316F0010F48
:10F8200018BF2032981AF0BC70470A786F78561CBF
:10F8300007F00107AE5DEFE740F234100A78C2F23C
:10F840000000561C05686F78AE5D07F00107E3E71E
:10F850002DE9F04F40F23415C2F2000583B00C469A
:10F860001F46D5F800800E460190009216F8015B05
:10F8700008EB050393F801B01BF0080BF6D12D2D12
:10F8800065D02B2D08BF16F8015BD7F1010338BFF7
:10F890000023102F14BF1A4643F0010232B1302D5D
:10F8A00066D01BB1302D0CBF08270A27BBF1000F13
:10F8B000394614BF4FF000496FF00049484600F048
:10F8C00059FC48468A46394600F026FB00218C4602
:10F8D00008EB0502A5F13003527812F0040F08D1AD
:10F8E00012F0030F20D012F0010F14BF372357235B
:10F8F000EB1A9F4218DD844594BF0022012252EA90
:10F90000D1714FF0FF310CD1844514BF0022012288
:10F910005345D4BF002202F0010212B907FB0C3C90
:10F92000012116F8015BD3E7B1F1FF3F14D0BBF121
:10F93000000F09D16046009B1BB101B1741E009AF3
:10F94000146003B0BDE8F08FCCF10000F3E716F8C7
:10F95000015B4FF0010B98E7019ABBF1000F4FF0EC
:10F96000220314BF4FF000406FF000401360E2E745
:10F970003278782A14BF00210121582A14BF0A4680
:10F9800041F00102002A8CD07578102702368DE7ED
:10F9900010B540F23814C2F200048C4613460146FA
:10F9A00062462068FFF754FF10BD00BF2DE9F04309
:10F9B0008BB006460F4600F07BF840F22C24C2F2D2
:10F9C000000494F90030B3F1FF3F8046894638D0F7
:10F9D0003046394600F084FA0546002831D13046D9
:10F9E00039460022002301F01DF8002829D124788F
:10F9F00041F63033C0F6010308950193CDE9026763
:10FA0000CDE90467002C21D040F200030022CFF69C
:10FA1000F0733046CDE9062339460022002300F07A
:10FA2000D9FF002822D0022300939C4234D068469C
:10FA300000F064FA00282FD0089B002B27D1DDE9C5
:10FA40000689404649460BB0BDE8F0834FF6FF7388
:10FA50004FF06042CCF2EF733046CDE906233946D1
:10FA60000022002300F0B6FF0028DCD10123022C85
:10FA7000009316D0684600F041FA90B141F6343058
:10FA8000C0F6010000F03CFACDE90601D4E700F031
:10FA90003DFA089B0360D2E700F038FA22230360A6
:10FAA000CAE700F033FA21230360E7E70000000013
:10FAB000B1F5801F0B462DE9F04F804687B089468F
:10FAC00004460D463EDB4FF6FF720026C7F6EF7286
:10FAD000934251DC23F07F4445F6647C24F47004A7
:10FAE000C0F2090CA44440F20002A6F57E760CF4A4
:10FAF000801C073EC3F6F0728CEA020206EB235626
:10FB000040F20003404642EA0401C3F6F0730022CB
:10FB100006EB1C5600F042FBA31C23F07F4323F4AA
:10FB20007003022B804689462FDC0022002300F060
:10FB300051FF002800F0CA80002E40F07C81002098
:10FB400000211FE021F00043034300F0B5800029AD
:10FB5000C0F2468140F200030022C4F250336FF03D
:10FB6000350600F0CFFC4FF6FF72C7F6EF720B467A
:10FB7000804693428946ADDD4046494642464B4663
:10FB800000F00EFB07B0BDE8F08F00224FF080437D
:10FB900000F006FB4EF68635CFF6F975651902467C
:10FBA0000B464046494600F0D7FDCDE902013046FC
:10FBB00000F042FCCDE90401DDE9020102460B46FA
:10FBC00000F0A0FC02460B46CDE9000100F09AFCD3
:10FBD000A7A3D3E9002382468B4600F093FCA6A39B
:10FBE000D3E9002300F0DCFA52465B4600F08AFCC1
:10FBF000A3A3D3E9002300F0D3FA52465B4600F0FA
:10FC000081FCA1A3D3E9002300F0CAFADDE90023B7
:10FC100000F078FC9EA3D3E90023CDE90001504613
:10FC2000594600F06FFC9CA3D3E9002300F0B8FA1A
:10FC300052465B4600F066FC99A3D3E9002300F02E
:10FC4000AFFA52465B4600F05DFC0B460246DDE92A
:10FC5000000100F0A5FA4BF65103C0F206031B1B8E
:10FC600043EA0505002D82468B4656DD40F200032F
:10FC70000022C3F6E0734046494600F043FC42468A
:10FC80004B4600F03FFC04460D46002E75D152460F
:10FC90005B4600F085FADDE9022300F033FC024602
:10FCA0000B462046294600F079FA02460B464046AC
:10FCB000494600F073FA65E740F200010020002297
:10FCC0000023CCF2503100F047FD5BE742464B4643
:10FCD0004046494600F016FC73A3D3E900230446CE
:10FCE0000D464046494600F00DFC40F2000300225C
:10FCF000C3F6E07300F054FA02460B46204629464C
:10FD000000F000FC04460D46002E72D140464946E4
:10FD100022462B4600F042FA34E7002E00F0D48051
:10FD200063A3D3E90023DDE9040100F0EBFB5246B5
:10FD30005B4606460F464046494600F02FFADDE98D
:10FD4000022300F0DFFB5CA3D3E9002304460D4649
:10FD5000DDE9040100F0D6FB02460B4620462946A9
:10FD600000F01EFA42464B4600F018FA02460B46D7
:10FD70003046394600F012FA04E74DA3D3E90023D8
:10FD8000DDE9040100F0BEFB52465B46CDE900010F
:10FD90002046294600F004FADDE9022300F0B2FB18
:10FDA00047A3D3E9002306460F46DDE9040100F02E
:10FDB000A9FB02460B463046394600F0F1F90246EF
:10FDC0000B462046294600F0E9F942464B4600F032
:10FDD000E5F902460B46DDE9000100F0DFF9D1E666
:10FDE00002460B4600F0DAF90022002300F0B4FCD2
:10FDF000C8E6304600F020FB2DA3D3E900230646D9
:10FE00000F4600F07FFB2CA3D3E9002382468B46EC
:10FE10003046394600F076FB22462B4600F0C0F90A
:10FE200042464B4600F0BAF902460B465046594648
:10FE300000F0B4F9A6E6304600F0FEFA1CA3D3E9C0
:10FE4000002306460F4600F05DFB1DA3D3E9002307
:10FE500004460D463046394600F054FB02460B4638
:10FE60002046294600F09CF98CE600BFAFF30080E5
:10FE700044523EDF12F1C23FDE03CB966446C73FD9
:10FE8000599322942449D23F935555555555E53FF2
:10FE90009FC678D0099AC33FAF788E1DC571CC3FFD
:10FEA00004FA97999999D93F555555555555D5BF48
:10FEB0000000E0FE422EE63F763C7935EF39EABDA0
:10FEC000763C7935EF39EA3D02460B4640464946D5
:10FED00000F064F9DDE9022300F014FBE5E600BF61
:10FEE00002464042104321F0004141EAD070C0F187
:10FEF000FE4000F57000C00F704700BF0020704743
:10FF000040F200010020C7F6F871704740F2381344
:10FF1000C2F20003186870474A1E08BF7047C0F05D
:10FF20002481884240F21681114200F01781B0FA14
:10FF300080F3B1FA81F2A2EB0303C3F11F0304A221
:10FF400002EB03134FF000029F4600BFAFF30080A7
:10FF5000B0EBC17F00BF42EB020228BFA0EBC17033
:10FF6000B0EB817F00BF42EB020228BFA0EB8170A3
:10FF7000B0EB417F00BF42EB020228BFA0EB417013
:10FF8000B0EB017F00BF42EB020228BFA0EB017083
:10FF9000B0EBC16F00BF42EB020228BFA0EBC16013
:10FFA000B0EB816F00BF42EB020228BFA0EB816083
:10FFB000B0EB416F00BF42EB020228BFA0EB4160F3
:10FFC000B0EB016F00BF42EB020228BFA0EB016063
:10FFD000B0EBC15F00BF42EB020228BFA0EBC150F3
:10FFE000B0EB815F00BF42EB020228BFA0EB815063
:10FFF000B0EB415F00BF42EB020228BFA0EB4150D3
:020000040801F1
:10000000B0EB015F00BF42EB020228BFA0EB015042
:10001000B0EBC14F00BF42EB020228BFA0EBC140D2
:10002000B0EB814F00BF42EB020228BFA0EB814042
:10003000B0EB414F00BF42EB020228BFA0EB4140B2
:10004000B0EB014F00BF42EB020228BFA0EB014022
:10005000B0EBC13F00BF42EB020228BFA0EBC130B2
:10006000B0EB813F00BF42EB020228BFA0EB813022
:10007000B0EB413F00BF42EB020228BFA0EB413092
:10008000B0EB013F00BF42EB020228BFA0EB013002
:10009000B0EBC12F00BF42EB020228BFA0EBC12092
:1000A000B0EB812F00BF42EB020228BFA0EB812002
:1000B000B0EB412F00BF42EB020228BFA0EB412072
:1000C000B0EB012F00BF42EB020228BFA0EB0120E2
:1000D000B0EBC11F00BF42EB020228BFA0EBC11072
:1000E000B0EB811F00BF42EB020228BFA0EB8110E2
:1000F000B0EB411F00BF42EB020228BFA0EB411052
:10010000B0EB011F00BF42EB020228BFA0EB0110C1
:10011000B0EBC10F00BF42EB020228BFA0EBC10051
:10012000B0EB810F00BF42EB020228BFA0EB8100C1
:10013000B0EB410F00BF42EB020228BFA0EB410031
:10014000B0EB010F00BF42EB020228BFA0EB0100A1
:10015000104670470CBF012000207047B1FA81F2B1
:10016000C2F11F0220FA02F0704708B14FF0FF30D1
:1001700000F00EB80029F8D02DE90340FFF7CCFEBF
:10018000BDE8064002FB00F3A1EB0301704700BF8E
:10019000704700BF81F0004102E000BF83F00043E0
:1001A00030B54FEA41044FEA430594EA050F08BF12
:1001B00090EA020F1FBF54EA000C55EA020C7FEAD6
:1001C000645C7FEA655C00F0E2804FEA5454D4EB53
:1001D0005555B8BF6D420CDD2C4480EA020281EA1D
:1001E000030382EA000083EA010180EA020281EA55
:1001F0000303362D88BF30BD11F0004F4FEA0131A7
:100200004FF4801C4CEA113102D0404261EB4101B5
:1002100013F0004F4FEA03334CEA133302D052423B
:1002200063EB430394EA050F00F0A780A4F10104F7
:10023000D5F1200E0DDB02FA0EFC22FA05F2801831
:1002400041F1000103FA0EF2801843FA05F3594117
:100250000EE0A5F120050EF1200E012A03FA0EFC96
:1002600028BF4CF0020C43FA05F3C01851EBE371C0
:1002700001F0004507D54FF0000EDCF1000C7EEBDD
:1002800000006EEB0101B1F5801F1BD3B1F5001F1B
:100290000CD349085FEA30004FEA3C0C04F101043A
:1002A0004FEA445212F5800F80F09A80BCF1004F63
:1002B00008BF5FEA500C50F1000041EB045141EAE5
:1002C000050130BD5FEA4C0C404141EB010111F4E6
:1002D000801FA4F10104E9D191F0000F04BF014691
:1002E0000020B1FA81F308BF2033A3F10B03B3F16F
:1002F00020020CDA0C3208DD02F1140CC2F10C02FF
:1003000001FA0CF021FA02F10CE002F11402D8BF5C
:10031000C2F1200C01FA02F120FA0CFCDCBF41EA28
:100320000C019040E41AA2BF01EB0451294330BDF7
:100330006FEA04041F3C1CDA0C340EDC04F11404D4
:10034000C4F1200220FA04F001FA02F340EA0300AB
:1003500021FA04F345EA030130BDC4F10C04C4F1F1
:10036000200220FA02F001FA04F340EA03002946D1
:1003700030BD21FA04F0294630BD94F0000F83F41B
:10038000801306BF81F480110134013D4EE77FEAFE
:10039000645C18BF7FEA655C29D094EA050F08BF4A
:1003A00090EA020F05D054EA000C04BF194610462B
:1003B00030BD91EA030F1EBF0021002030BD5FEA6F
:1003C000545C05D14000494128BF41F0004130BD97
:1003D00014F580043CBF01F5801130BD01F00045EB
:1003E00045F0FE4141F470014FF0000030BD7FEA5E
:1003F000645C1ABF194610467FEA655C1CBF0B4659
:10040000024650EA013406BF52EA033591EA030F6F
:1004100041F4002130BD00BF90F0000F04BF002167
:10042000704730B54FF4806404F132044FF000059A
:100430004FF0000150E700BF90F0000F04BF002113
:10044000704730B54FF4806404F1320410F0004579
:1004500048BF40424FF000013EE700BF42004FEA74
:10046000E2014FEA31014FEA02701FBF12F07F43F1
:1004700093F07F4F81F06051704792F0000F14BFEE
:1004800093F07F4F704730B54FF4607401F0004532
:1004900021F0004120E700BF50EA010208BF704789
:1004A00030B54FF000050AE050EA010208BF70477E
:1004B00030B511F0004502D5404261EB41014FF4E7
:1004C000806404F132045FEA915C3FF4DCAE4FF0EB
:1004D00003025FEADC0C18BF03325FEADC0C18BFD2
:1004E000033202EBDC02C2F1200300FA03FC20FA23
:1004F00002F001FA03FE40EA0E0021FA02F1144470
:10050000C1E600BF70B54FF0FF0C4CF4E06C1CEA84
:1005100011541DBF1CEA135594EA0C0F95EA0C0FF9
:1005200000F0DEF82C4481EA030621EA4C5123EA6C
:100530004C5350EA013518BF52EA033541F480119B
:1005400043F4801338D0A0FB02CE4FF00005E1FB4E
:1005500002E506F00042E0FB03E54FF00006E1FB98
:1005600003569CF0000F18BF4EF0010EA4F1FF04DB
:10057000B6F5007F64F5407404D25FEA4E0E6D411B
:1005800046EB060642EAC62141EA55514FEAC5202C
:1005900040EA5E504FEACE2EB4F1FD0C88BFBCF5A8
:1005A000E06F1ED8BEF1004F08BF5FEA500E50F159
:1005B000000041EB045170BD06F0004646EA01011F
:1005C00040EA020081EA0301B4EB5C04C2BFD4EB51
:1005D0000C0541EA045170BD41F480114FF0000E4A
:1005E000013C00F3AB8014F1360FDEBF002001F0B8
:1005F000004170BDC4F10004203C35DA0C341BDC32
:1006000004F11404C4F1200500FA05F320FA04F003
:1006100001FA05F240EA020001F0004221F0004137
:1006200010EBD37021FA04F642EB06015EEA430EAA
:1006300008BF20EAD37070BDC4F10C04C4F12005DA
:1006400000FA04F320FA05F001FA04F240EA02008D
:1006500001F0004110EBD37041F100015EEA430E5E
:1006600008BF20EAD37070BDC4F1200500FA05F27E
:100670004EEA020E20FA04F301FA05F243EA0203FD
:1006800021FA04F001F0004121FA04F220EA02000C
:1006900000EBD3705EEA430E08BF20EAD37070BD52
:1006A00094F0000F0FD101F00046400041EB010132
:1006B00011F4801F08BF013CF7D041EA060195F014
:1006C000000F18BF704703F00046520043EB0303CE
:1006D00013F4801F08BF013DF7D043EA06037047BB
:1006E00094EA0C0F0CEA135518BF95EA0C0F0CD0C6
:1006F00050EA410618BF52EA4306D1D181EA03010C
:1007000001F000414FF0000070BD50EA410606BF05
:100710001046194652EA430619D094EA0C0F02D14A
:1007200050EA013613D195EA0C0F05D152EA03368F
:100730001CBF104619460AD181EA030101F00041AD
:1007400041F0FE4141F470014FF0000070BD41F0F6
:10075000FE4141F4780170BD70B54FF0FF0C4CF4D0
:10076000E06C1CEA11541DBF1CEA135594EA0C0FEF
:1007700095EA0C0F00F0A7F8A4EB050481EA030E3C
:1007800052EA03354FEA013100F088804FEA033323
:100790004FF0805545EA131343EA12634FEA0222F1
:1007A00045EA111545EA10654FEA00260EF00041B2
:1007B0009D4208BF964244F1FD0404F5407402D204
:1007C0005B084FEA3202B61A65EB03055B084FEA95
:1007D00032024FF480104FF4002CB6EB020E75EB92
:1007E000030E22BFB61A754640EA0C005B084FEABA
:1007F0003202B6EB020E75EB030E22BFB61A754637
:1008000040EA5C005B084FEA3202B6EB020E75EB81
:10081000030E22BFB61A754640EA9C005B084FEAF9
:100820003202B6EB020E75EB030E22BFB61A754606
:1008300040EADC0055EA060E18D04FEA051545EAF5
:1008400016754FEA06164FEAC30343EA52734FEA9E
:10085000C2025FEA1C1CC0D111F4801F0BD141EA17
:1008600000014FF000004FF0004CB6E711F4801F7C
:1008700004BF01430020B4F1FD0C88BFBCF5E06F5C
:100880003FF6AFAEB5EB030C04BFB6EB020C5FEA6C
:10089000500C50F1000041EB045170BD0EF0004EC1
:1008A0004EEA113114EB5C04C2BFD4EB0C0541EAF3
:1008B000045170BD41F480114FF0000E013C90E6F0
:1008C00045EA060E8DE60CEA135594EA0C0F08BFB4
:1008D00095EA0C0F3FF43BAF94EA0C0F0AD150EAB3
:1008E00001347FF434AF95EA0C0F7FF425AF104646
:1008F00019462CE795EA0C0F06D152EA03353FF46E
:10090000FDAE1046194622E750EA410618BF52EAEA
:1009100043067FF4C5AE50EA41047FF40DAF52EABE
:1009200043057FF4EBAE12E74FF0FF3C06E000BF5B
:100930004FF0010C02E000BF4FF0010C4DF804CD68
:100940004FEA410C7FEA6C5C4FEA430C18BF7FEA28
:100950006C5C1BD001B050EA410C0CBF52EA430C56
:1009600091EA030F02BF90EA020F0020704710F1D6
:10097000000F91EA030F58BF994208BF90422CBF65
:10098000D8176FEAE37040F0010070474FEA410C5E
:100990007FEA6C5C02D150EA013C07D14FEA430C7C
:1009A0007FEA6C5CD6D152EA033CD3D05DF8040BED
:1009B000704700BF8446104662468C46194663461F
:1009C00000E000BF01B5FFF7B7FF002848BF10F1F6
:1009D000000F01BD4DF808EDFFF7F4FF0CBF01203B
:1009E00000205DF808FB00BF4DF808EDFFF7EAFFB7
:1009F00034BF012000205DF808FB00BF4DF808ED72
:100A0000FFF7E0FF94BF012000205DF808FB00BF66
:100A10004DF808EDFFF7CEFF94BF012000205DF8F0
:100A200008FB00BF4DF808EDFFF7C4FF34BF0120FD
:100A300000205DF808FB00BF4FEA410212F50012EA
:100A400015D211D56FF47873B3EB625212D94FEA15
:100A5000C12343F0004343EA505311F0004F23FAFF
:100A600002F018BF404270474FF00000704750EA54
:100A7000013005D111F0004008BF6FF00040704711
:100A80004FF00000704700BF4FEA4102B2F1E0436F
:100A900024BFB3F5001CDCF1FE5C0DD901F0004C65
:100AA0004FEAC0024CEA5070B2F1004F40EB8300B5
:100AB00008BF20F00100704711F0804F21D113F1E1
:100AC0003872BCBF01F00040704741F480114FEA1A
:100AD0005252C2F11802C2F1200C10FA0CF320FAA3
:100AE00002F018BF40F001004FEAC1234FEAD323C0
:100AF00003FA0CFC40EA0C0023FA02F34FEA43032A
:100B0000CCE77FEA625307D150EA01331EBF4FF0B2
:100B1000FE4040F44000704701F0004040F0FE40CD
:100B200040F40000704700BF80F0004002E000BFCA
:100B300081F0004142001FBF5FEA410392EA030FC8
:100B40007FEA226C7FEA236C6AD04FEA1262D2EB12
:100B50001363C1BFD218414048404140B8BF5B4217
:100B6000192B88BF704710F0004F40F4000020F0B0
:100B70007F4018BF404211F0004F41F4000121F0C6
:100B80007F4118BF494292EA030F3FD0A2F1010210
:100B900041FA03FC10EB0C00C3F1200301FA03F14E
:100BA00000F0004302D5494260EB4000B0F5000F71
:100BB00013D3B0F1807F06D340084FEA310102F130
:100BC0000102FE2A51D2B1F1004F40EBC25008BFE2
:100BD00020F0010040EA03007047490040EB0000AC
:100BE00010F4000FA2F10102EDD1B0FA80FCACF1DB
:100BF000080CB2EB0C0200FA0CF0AABF00EBC250DA
:100C000052421843BCBFD0401843704792F0000FC7
:100C100081F4000106BF80F400000132013BB5E71A
:100C20004FEA41037FEA226C18BF7FEA236C21D090
:100C300092EA030F04D092F0000F08BF08467047F5
:100C400090EA010F1CBF0020704712F07F4F04D1C3
:100C5000400028BF40F00040704712F100723CBFD6
:100C600000F50000704700F0004343F0FE4040F400
:100C7000000070477FEA226216BF08467FEA2363BE
:100C80000146420206BF5FEA412390EA010F40F4A9
:100C9000800070474FF0000304E000BF10F00043F5
:100CA00048BF40425FEA000C08BF704743F09643DC
:100CB00001464FF000001CE050EA010208BF7047F7
:100CC0004FF000030AE000BF50EA010208BF70477E
:100CD00011F0004302D5404261EB41015FEA010C93
:100CE00002BF84460146002043F0B64308BFA3F18B
:100CF0008053A3F50003BCFA8CF2083AA3EBC2536D
:100D000010DB01FA02FC634400FA02FCC2F120028B
:100D1000BCF1004F20FA02F243EB020008BF20F0C2
:100D20000100704702F1200201FA02FCC2F1200228
:100D300050EA4C0021FA02F243EB020008BF20EA1D
:100D4000DC7070474FF0FF0C1CEAD0521EBF1CEA4B
:100D5000D15392EA0C0F93EA0C0F6FD01A4480EA39
:100D6000010C400218BF5FEA41211ED04FF0006322
:100D700043EA501043EA5111A0FB01310CF000404E
:100D8000B1F5000F3EBF490041EAD3715B0040EA74
:100D9000010062F17F02FD2A1DD8B3F1004F40EB44
:100DA000C25008BF20F00100704790F0000F0CF017
:100DB000004C08BF49024CEA502040EA51207F3ADB
:100DC000C2BFD2F1FF0340EAC250704740F40000B6
:100DD0004FF00003013A5DDC12F1190FDCBF00F0A7
:100DE00000407047C2F10002410021FA02F1C2F155
:100DF000200200FA02FC5FEA310040F1000053EAF1
:100E00004C0308BF20EADC70704792F0000F00F03E
:100E1000004C02BF400010F4000F013AF9D040EA44
:100E20000C0093F0000F01F0004C02BF490011F4D8
:100E3000000F013BF9D041EA0C018FE70CEAD153D6
:100E400092EA0C0F18BF93EA0C0F0AD030F0004C56
:100E500018BF31F0004CD8D180EA010000F000400A
:100E6000704790F0000F17BF90F0004F084691F0C8
:100E7000000F91F0004F14D092EA0C0F01D1420202
:100E80000FD193EA0C0F03D14B0218BF084608D1CB
:100E900080EA010000F0004040F0FE4040F4000015
:100EA000704740F0FE4040F4400070474FF0FF0CA8
:100EB0001CEAD0521EBF1CEAD15392EA0C0F93EAEF
:100EC0000C0F69D0A2EB030280EA010C49024FEA41
:100ED000402037D04FF0805343EA111143EA1013FA
:100EE0000CF000408B4238BF5B0042F17D024FF4B2
:100EF000000C8B4224BF5B1A40EA0C00B3EB510F8D
:100F000024BFA3EB510340EA5C00B3EB910F24BF75
:100F1000A3EB910340EA9C00B3EBD10F24BFA3EBFA
:100F2000D10340EADC001B0118BF5FEA1C1CE0D1C2
:100F3000FD2A3FF650AF8B4240EBC25008BF20F075
:100F4000010070470CF0004C4CEA50207F32C2BFC9
:100F5000D2F1FF0340EAC250704740F400004FF066
:100F60000003013A37E792F0000F00F0004C02BF97
:100F7000400010F4000F013AF9D040EA0C0093F061
:100F8000000F01F0004C02BF490011F4000F013BBB
:100F9000F9D041EA0C0195E70CEAD15392EA0C0F23
:100FA00008D142027FF47DAF93EA0C0F7FF470AF5B
:100FB000084676E793EA0C0F04D14B023FF44CAF9E
:100FC00008466EE730F0004C18BF31F0004CCAD133
:100FD00030F000427FF45CAF31F000437FF43CAF6F
:100FE0005FE700BF4FF0FF3C06E000BF4FF0010C91
:100FF00002E000BF4FF0010C4DF804CD4FEA400273
:101000004FEA41037FEA226C18BF7FEA236C11D0BC
:1010100001B052EA530C18BF90EA010F58BFB2EB6F
:10102000030088BFC81738BF6FEAE17018BF40F0EF
:10103000010070477FEA226C02D15FEA402C05D1A3
:101040007FEA236CE4D15FEA412CE1D05DF8040B28
:10105000704700BF844608466146FFE70FB5FFF7BB
:10106000C9FF002848BF10F1000F0FBD4DF808ED73
:10107000FFF7F4FF0CBF012000205DF808FB00BF64
:101080004DF808EDFFF7EAFF34BF012000205DF8BE
:1010900008FB00BF4DF808EDFFF7E0FF94BF01200B
:1010A00000205DF808FB00BF4DF808EDFFF7D2FF08
:1010B00094BF012000205DF808FB00BF4DF808ED4B
:1010C000FFF7C8FF34BF012000205DF808FB00BF18
:1010D00042000ED2B2F1FE4F0BD34FF09E03B3EBA2
:1010E000126209D44FEA002343F0004323FA02F0CE
:1010F00070474FF00000704712F1610F01D14202BA
:1011000002D14FF0FF3070474FF00000704700BF32
:1011100073B96AB9002908BF0028BCBF00204FF08E
:101120000041C4BF6FF000414FF0FF30FFF730B80F
:1011300082B0EC462DE9005000F01CF8DDF804E028
:1011400002B00CBC704700BFF8B514461D460646F9
:101150000F4600F0D3F900FB05F5A0FB042304FBC8
:101160000154E318B61A67EB0307069BC3E900674F
:10117000F8BD00BFF8B514461D4606460F4600F000
:101180000FF800FB05F5A0FB042304FB0154E31852
:10119000B61A67EB0307069BC3E90067F8BD00BFFB
:1011A00000292DE9F04F85B0C0F2C9800026002B40
:1011B000C0F2C0808946144605469B46002B4BD1A1
:1011C0008A4258D9B2FA82F353B1C3F1200001FA2E
:1011D00003F925FA00F812FA03F49D4048EA0909D8
:1011E000270C484639461FFA84FBFEF795FE394620
:1011F00082464846FEF7BEFF4FEA15420BFB0AF354
:1012000042EA01494B4509D919EB04090AF1FF3AB1
:1012100004D24B4584BF0AF1FF3AA144C3EB09094C
:1012200039464846ADB2FEF777FE39468046484615
:10123000FEF7A0FF0BFB08FB45EA0145AB4507D9CC
:101240002D1908F1FF3803D2AB4588BF08F1FF38EC
:1012500048EA0A48002703E08B4257D90027B846DE
:1012600042463B4616B1524263EB430319461046D1
:1012700005B0BDE8F08F22B911460120FEF74CFE03
:101280000446B4FA84F8B8F1000F5ED1C4EB090843
:10129000270C1FFA84F90121029139464046FEF7D6
:1012A0003BFE394682464046FEF764FF4FEA15484A
:1012B00009FB0AF348EA014B5B4509D91BEB040B18
:1012C0000AF1FF3A04D25B4584BF0AF1FF3AA34416
:1012D000C3EB0B0B39465846ADB2FEF71DFE39463F
:1012E00080465846FEF746FF09FB08F945EA0145E6
:1012F000A94507D92D1908F1FF3803D2A94588BFA0
:1013000008F1FF3848EA0A48029FA9E7B3FA83F7D1
:10131000002F67D18B422CBF4FF000094FF001091D
:1013200082428CBF4C4649F00104002C96D04FF00D
:10133000010895E7524263EB4303F6433AE7404224
:1013400061EB41014FF0FF3631E704FA08F4C8F1D0
:10135000200735FA07F329FA07FA270C09FA08FBE0
:101360003946504643EA0B020292FEF7D5FD394654
:101370001FFA84F983465046FEF7FCFE029809FBEB
:101380000BF2030C43EA01439A4204D91B190BF1F7
:10139000FF3BC0F0AD809B1A394618460193FEF71B
:1013A000BBFD0199824608463946FEF7E3FE0298E6
:1013B00009FB0AF31FFA80FC4CEA0142934208D968
:1013C00012190AF1FF3A04D2934284BF0AF1FF3A9C
:1013D000121905FA08F54AEA0B4EC3EB0208CDF8DC
:1013E00008E05AE7C7F1200003FA07FAC24035FACD
:1013F00000F342EA0A0B21FA00F801FA07F9404625
:101400004FEA1B4A43EA0901029151461FFA8BF247
:101410000392FEF781FD514681464046FEF7AAFE43
:101420000398029B00FB09F2180C14FA07F340EA38
:101430000144A24204D914EB0B0409F1FF3951D342
:10144000A41A514620460193FEF766FD5146804698
:101450002046FEF78FFE039C019B04FB08F2029CD2
:101460001FFA84FC4CEA0140824204D910EB0B00C5
:1014700008F1FF3830D348EA09481FFA83FC1B0CF7
:10148000801A1FFA88FE4FEA184A0CFB0EF90CFB73
:101490000AF203FB0E2103FB0AF301EB19418A4216
:1014A00088BF03F5803303EB114E704510D31FFA4C
:1014B00089F905FA07F709EB014014BF0022012260
:1014C00087422CBF002702F00107002F3FF4C8AE6F
:1014D00008F1FF380027C3E6824284BF584408F170
:1014E000FF38C8E7A24284BF09F1FF395C44A7E78F
:1014F0009A4284BF0BF1FF3B1B194CE72DE9F04FDB
:101500000C4683B08046164689461F4615468A46D5
:10151000002B4BD18A425CD9B2FA82F35BB1C3F1A2
:10152000200001FA03FA28FA00F216FA03F508FA85
:1015300003F842EA0A0A2E0C50463146AFB2FEF7D3
:10154000EBFC31464FEA184481465046FEF712FE46
:1015500007FB09F344EA014A534509D91AEB050A86
:1015600009F1FF3904D2534584BF09F1FF39AA4478
:10157000C3EB0A0A314650461FFA88F8FEF7CCFC46
:10158000314604465046FEF7F5FD07FB04F748EAEE
:101590000148474506D9013C18EB050802D24745EA
:1015A00088BF013C44EA094400265CE08B4258D8DD
:1015B000B3FA83F6002E5BD18B422CBF00220122AE
:1015C00085428CBF154642F00105002D49D001240B
:1015D00049E022B911460120FEF79EFC0546B5FA06
:1015E00085F6002E40F0BB80641B2F0C1FFA85FA95
:1015F000012639462046FEF78FFC39464FEA184B44
:1016000081462046FEF7B6FD0AFB09F34BEA014B83
:101610005B4509D91BEB050B09F1FF3904D25B458A
:1016200084BF09F1FF39AB44C3EB0B0B3946584675
:101630001FFA88F8FEF770FC394604465846FEF754
:1016400099FD0AFB04FA48EA0148C24506D9013C63
:1016500018EB050802D2C24588BF013C44EA0944A0
:1016600001E0002634463146204603B0BDE8F08F45
:10167000C6F12000B34032FA00F721FA00FB1F4305
:1016800014FA06F228FA00F158464FEA174A1143B5
:1016900000915146BBB20193FEF73EFC5146B54066
:1016A00081465846FEF766FD019C009804FB09F34D
:1016B0004FEA104C4CEA014B5B4505D91BEB070B7D
:1016C00009F1FF39C0F08F80C3EB0B0B5146584630
:1016D000FEF722FC514604465846FEF74BFD0198A2
:1016E000009A00FB04F31FFA82FC4CEA0142934289
:1016F00006D9013CD21903D2934201D9D219013C37
:1017000044EA0944A8B2D21A2D0C1FFA84FC4FEA0D
:10171000144300FB0CF700FB03FE05FB0CE105FB8B
:1017200003F501EB17418E4588BF05F5803505EBC4
:101730001145AA4210D3BFB208FA06F607EB0142E0
:1017400014BF4FF0000E4FF0010E96422CBF002642
:101750000EF00106002E86D0013C002683E7B5403E
:10176000C6F1200124FA01F928FA01F22F0CB44045
:101770003946484622430092FEF7CEFB39461FFA0F
:1017800085FA83464846FEF7F5FC009B1A0C0AFBD7
:101790000BF342EA0144A34203D964190BF1FF3B66
:1017A00027D3E41A39462046FEF7B6FB3946814670
:1017B0002046FEF7DFFC00980AFB09F31FFA80FCC5
:1017C0004CEA0144A34208D9641909F1FF3904D253
:1017D000A34284BF09F1FF39641908FA06F8E41A34
:1017E00049EA0B4605E75B4584BF09F1FF39BB4475
:1017F0006AE7A34284BF0BF1FF3B6419D1E700BF46
:101800000000000000000000010003E800000000EC
:1018100000000003E800000000000200FA060003D8
:10182000000000000037060000000000000000007B
:10183000F4010000640000000180080800000000BE
:10184000006400000000000000000000C80000006C
:101850001201100102000040D016A105011B010277
:101860000301000009024300020100C03209040024
:1018700000010202010005240010010524010001FD
:10188000042402020524060001070582030800FF64
:1018900009040100020A00000007050302400000DD
:1018A00007058102400000000403090426035400D8
:1018B000720069006E0061006D00690063004D00F8
:1018C0006F00740069006F006E0020004300740018
:1018D0006C000000320354004D0043004D002D0009
:1018E0003100310036003100200028007600690008
:1018F00072007400750061006C00200043004F000E
:101900004D00290020000000524F520000010652F5
:101910004F4C000002064D5354000003024D565038
:1019200000000407534150000005074741500000E4
:10193000060353544150000703525341500008031B
:101940005347500000090747475000000A0353540B
:101950004750000B0352534750000C0352465300AC
:10196000000D0353494F00000E0747494F00000F79
:101970000353414300001D0753434F00001E074718
:10198000434F00001F0343434F0000200341434FD8
:10199000000027035546300000400755463100003F
:1019A00041075546320000420755463300004307C1
:1019B0005546340000440755463500004507554656
:1019C00036000046075546370000470752554E007F
:1019D00000810553544F5000800042494E00008B57
:1019E00000000000000000000000000001020304ED
:1019F000010203040607080902040608002020204B
:101A000020202020202028282828282020202020AE
:101A1000202020202020202020202020208810107E
:101A200010101010101010101010101010040404DA
:101A30000404040404040410101010101010414198
:101A40004141414101010101010101010101010186
:101A5000010101010101010110101010101042429A
:101A60004242424202020202020202020202020256
:101A700002020202020202021010101020000000F6
:101A80000000000000000000000000000000000056
:101A90000000000000000000000000000000000046
:101AA0000000000000000000000000000000000036
:101AB0000000000000000000000000000000000026
:101AC0000000000000000000000000000000000016
:101AD0000000000000000000000000000000000006
:101AE00000000000000000000000000000000000F6
:101AF00000000000000000000000000000000000E6
:101B00003131363156313237004142530052454C63
:101B100000434F4F52440053544152540053544FCA
:101B2000500053544154555300000000430000003E
:081B30006C6F6700000000006B
:081B380068F6FF7F01000000C8
:101B4000001B010800010000000102000008000065
:101B50000100000002000000000000000000000082
:101B60000000000000000000000000000000000075
:101B70000000000000000000000000000000000065
:101B8000000000000000000000C20100000008008A
:101B9000A818010804000000AC1801082600000085
:101BA000D418010832000000B00000201A00000024
:101BB00064180108430000005018010812000000DA
:101BC000E1930008ED910008FD8F000811900008D6
:101BD000159000087590000899900008DD910008A4
:101BE000CD910008A991000800000000400000000D
:101BF0001A0354004D00430031003100360031001B
:101C0000000000000000000000000000FD8E000841
:101C1000A9E70008A9E70008A9E70008A9E7000864
:101C2000A9E70008A9E70008A9E70008A9E7000854
:101C30003D930008A9E70008A9E70008A9E7000804
:101C4000A9E7000804010000A9E70008D98F0008EF
:101C5000A9E70008A9E70008A9E70008A9E7000824
:101C6000A9E70008A9E70008F18F000801000000BB
:101C7000FD190108FC1901083C01002000000000CA
:101C80000000000000000000000000000000000054
:101C90000000000000000000000000002C1B0108F4
:101CA0000000000000000000000000000000000034
:101CB0000000000000000000000000000000000024
:101CC0000000000000000000000000000000000014
:101CD0000000000000000000000000000000000004
:101CE00000000000000000000000000000000000F4
:101CF00000000000000000000000000000000000E4
:101D000000000000000000000000000000000000D3
:101D100000000000000000000000000000000000C3
:101D200000000000000000000000000000000000B3
:101D300000000000000000000000000000000000A3
:101D40000000000000000000000000000000000093
:101D50000000000000000000000000000000000083
:101D60000000000000000000000000000100000072
:04000005080041109E
:00000001FF
